:100000000C9426060C944E060C944E060C944E0648
:100010000C944E060C944E060C944E060C944E0610
:100020000C94F5120C944E060C944E060C944E064D
:100030000C944E060C944E060C944E060C944E06F0
:100040000C944E060C944E060C94F34E0C944E06F3
:100050000C94E7500C9475510C944E060C944E067B
:100060000C944E060C944E060C94BB6B0C944E06EE
:100070000C941C510C94B0510C944E064E545020CC
:1000800053796E63696E672E2E2E005D0D0A002C6B
:1000900000222C00302C22002C002C005B002E743F
:1000A000787400446574656374696E6720755344A1
:1000B0002E2E2E00302E2054657374202831206D92
:1000C000696E29002E20002000486F6C64204233A6
:1000D00020746F20737461727400436C69636B20C9
:1000E000423320746F206C6973740052756E206106
:1000F0002050726F6772616D3A00286C73776329C4
:100100000028656970290020286F73697029003AFA
:10011000002867776970290066777600747A006E28
:100120007470006468637000697031006970320037
:100130006970330069703400677731006777320087
:10014000677733006777340068703000687031007B
:1001500068777600657874005F00736474006D6181
:1001600073006D746F6E006D746F6600757273004E
:1001700072736F00776C0064656E00697061730064
:10018000646576696400636F6E006C69740064690D
:100190006D005F00757774006E747031006E74705E
:1001A00032006E747033006E747034006C67006DD2
:1001B000617332006D746F6E32006D746F66320061
:1001C00072657365740046573A00545A6F6E653A0B
:1001D000004E54503F00444843503F004F532E6957
:1001E00070313A002E6970323A002E6970333A004D
:1001F0002E6970343A0047572E6970313A002E69E3
:1002000070323A002E6970333A002E6970343A0029
:10021000506F72743A000048573A20004578702EAB
:1002200020626F6172643A000053746E2064656CE2
:1002300061793A004D6173313A004D61733120208C
:100240006F6E2061646A3A004D617331206F66669B
:100250002061646A3A005261696E2073656E736F43
:10026000723A004E6F726D616C6C79206F70656EC2
:100270003F0025205761746572696E673A004465D6
:10028000762E20656E61626C653F0049676E207056
:1002900077643F004465762E2049443A004C43443D
:1002A00020636F6E2E3A004C4344206C69742E3AE2
:1002B000004C43442064696D2E3A0000557365205C
:1002C000776561746865723F004E54502E697031D5
:1002D0003A002E6970323A002E6970333A002E6966
:1002E00070343A004C6F673F004D6173323A004DF5
:1002F00061733220206F6E2061646A3A004D617331
:1003000032206F66662061646A3A005265736574D4
:1003100020616C6C3F004D6F6E0054756500576531
:100320006400546875004672690053617400537527
:100330006E00207365630025004E6F0059657300E1
:100340002B002B0020474D54003030003A002D0088
:100350002B000020202020002D44697361626C6511
:1003600064212D003A0045004D433A0020284D41BC
:100370004329002D002E002D0020002020003A00EF
:100380002000486F6C6420423320746F20736176C4
:10039000650042312F42323A2B2F2D2C2042333A26
:1003A0002D3E003D3D536574204F7074696F6E7330
:1003B0003D3D00506C6561736520576169742E2E58
:1003C0002E00526573657474696E672E2E2E00437D
:1003D0006F6E6E656374696E672E2E2E0050726F9D
:1003E0006772616D20006C6F630077746B657900D4
:1003F000747474006376006A630064700063700054
:100400006372007570006A7000636F006A6F00733A
:1004100070006A7300636D006373006A6E006A6C3B
:1004200000646C007375006375003C7363726970DF
:10043000743E77696E646F772E6C6F636174696F59
:100440006E3D222F223B3C2F7363726970743E0A0B
:10045000007B22726573756C74223A24447D007BA4
:1004600022726573756C74223A24447D0024460020
:10047000222446223A24447D00485454502F312EE1
:100480003120323030204F4B0D0A004361636865E4
:100490002D436F6E74726F6C3A206D61782D6167B9
:1004A000653D3630343830302C207075626C6963AD
:1004B0000D0A00436F6E74656E742D547970653A41
:1004C00020746578742F6373733B6368617273651E
:1004D000743D7574662D380D0A436F6E74656E74C5
:1004E0002D456E636F64696E673A20677A69700D97
:1004F0000A00436F6E74656E742D547970653A20EE
:10050000746578742F6A6176617363726970743B85
:10051000636861727365743D7574662D380D0A43A6
:100520006F6E74656E742D456E636F64696E673AA5
:1005300020677A69700D0A000D0A002446002446DF
:10054000002446244600646179005D002C24530099
:100550002453005B007479706500656E64007374E9
:100560006172740068697374007400656E00736969
:1005700064005D2C226E73746174696F6E73223A2D
:1005800024447D002C0024440022736E223A5B0038
:10059000637077006E7077007474740077746B65A5
:1005A00079006C6F63006A737000726400656E009E
:1005B0007262740072736E003C6D657461206E61CE
:1005C0006D653D2276696577706F72742220636F66
:1005D0006E74656E743D2277696474683D646576F7
:1005E0006963652D77696474682C696E69746961E3
:1005F0006C2D7363616C653D312E302C6D696E69B5
:100600006D756D2D7363616C653D312E302C757386
:1006100065722D7363616C61626C653D6E6F223E25
:100620000D0A003C736372697074207372633D221B
:1006300024452F686F6D652E6A73223E3C2F7363CD
:10064000726970743E0A3C2F626F64793E0A3C2FD7
:1006500068746D6C3E00766172207665723D24444C
:100660002C697061733D24443B3C2F736372697045
:10067000743E0A003C21444F43545950452068744D
:100680006D6C3E0A3C68746D6C3E0A3C6865616442
:100690003E0A24463C2F686561643E0A3C626F64F2
:1006A000793E0A3C7363726970743E005B302C3093
:1006B0005D5D2C226C72756E223A5B24442C2444BE
:1006C0002C24442C244C5D7D005B24442C244C2C95
:1006D000244C5D2C00305D2C227073223A5B002488
:1006E000442C002264657674223A244C2C226E62DB
:1006F0007264223A24442C22656E223A24442C222D
:100700007264223A24442C227273223A24442C220A
:1007100072647374223A244C2C226C6F63223A2246
:100720002445222C2277746B6579223A22244522B3
:100730002C2273756E72697365223A24442C2273DD
:10074000756E736574223A24442C22656970223ACE
:10075000244C2C226C7763223A244C2C226C737725
:1007600063223A244C2C227362697473223A5B0030
:100770003C6872202F3E3C666F726D206E616D6525
:100780003D6F6620616374696F6E3D6375206D65B2
:1007900074686F643D6765743E3C703E3C623E53D6
:1007A00063726970742055524C3A3C2F623E3C692A
:1007B0006E70757420747970653D746578742073FB
:1007C000697A653D3332206D61786C656E67746857
:1007D0003D3132372076616C75653D2224452220FB
:1007E0006E616D653D6A73703E3C2F703E3C703E9D
:1007F00044656661756C742069732024533C627291
:10080000202F3E4966206C6F63616C206F6E2075EF
:10081000534420636172642C20757365202E2F3C35
:100820002F703E3C703E3C623E50617373776F7236
:10083000643A3C2F623E3C696E7075742074797026
:10084000653D70617373776F72642073697A653D7B
:100850003332206E616D653D70773E3C696E707518
:100860007420747970653D7375626D69743E3C2FB8
:10087000703E3C6872202F3E3C2F666F726D3E3C8E
:10088000736372697074207372633D6874747073FB
:100890003A2F2F75692E6F70656E737072696E6B6B
:1008A0006C65722E636F6D2F6A732F686173686554
:1008B000722E6A733E3C2F7363726970743E005DE2
:1008C0007D00225D00225D2C00245300244C5D2C11
:1008D0002200244C2C0024445D2C5B0024442C007A
:1008E0005B24442C24442C24442C5B00226E707224
:1008F0006F6773223A24442C226E626F61726473B4
:10090000223A24442C226D6E70223A24442C226D0B
:100910006E7374223A24442C22706E73697A6522B5
:100920003A24442C227064223A5B002C22646578BD
:1009300070223A24442C226D657870223A24447D3A
:10094000002C00222446223A2444006E616D65008A
:100950007069640070696400706964005D2C226DC8
:1009600061786C656E223A24447D002C0022245369
:10097000220022736E616D6573223A5B0073746EA0
:100980005F73657100726673746E0073746E5F647A
:100990006973006D61736F70320069676E6F7265A5
:1009A0005F7261696E006D61736F70005D2C002C69
:1009B00000244400222446223A5B00707700436FF3
:1009C0006E74656E742D547970653A206170706C28
:1009D00069636174696F6E2F6A736F6E0D0A436F7E
:1009E0006E6E656374696F6E3A20636C6F73650D2C
:1009F0000A004163636573732D436F6E74726F6C8D
:100A00002D416C6C6F772D4F726967696E3A202AA1
:100A10000D0A0043616368652D436F6E74726F6CDD
:100A20003A206D61782D6167653D302C206E6F2D09
:100A300063616368652C206E6F2D73746F72652C13
:100A4000206D7573742D726576616C69646174656F
:100A50000D0A0024462446244624460D0A7B002421
:100A6000462446244624460D0A00436F6E74656E84
:100A7000742D547970653A20746578742F68746D9C
:100A80006C0D0A0024462446244624460D0A000024
:100A9000010800060400014500008200004000201B
:100AA00000504F535420244620485454502F312E88
:100AB000300D0A486F73743A2024460D0A244624E8
:100AC000534163636570743A202A2F2A0D0A436FDD
:100AD0006E74656E742D4C656E6774683A2024449C
:100AE0000D0A436F6E74656E742D547970653A20EB
:100AF0006170706C69636174696F6E2F782D7777A0
:100B0000772D666F726D2D75726C656E636F64659F
:100B1000640D0A0D0A2453004745542024462453EB
:100B200020485454502F312E300D0A486F73743AB8
:100B30002024460D0A24460D0A0D0A004163636510
:100B400070743A20746578742F68746D6C00E300DB
:100B500004FA000100000001776561746865722E77
:100B60006F70656E737072696E6B6C65722E636FF9
:100B70006D002F776561746865720024442E70796A
:100B80003F6C6F633D2445266B65793D24452666A1
:100B900077763D24440065697000747A0073636160
:100BA0006C650073756E7365740073756E7269732E
:100BB000650000002100240027002A000000220018
:100BC000250028002B00000020002300260029001B
:100BD00002020202020202020404040404040404E5
:100BE00003030303030303030101010101010101E5
:100BF00001020408102040800102040810204080F7
:100C000001020408102040808040201008040201E6
:100C100000000001020000000000000004030706BD
:100C200000000000000000000000000000000000C4
:100C30007C3C3E5E2B3D3F2F5B5D3B2C2A225C00C3
:100C4000160D25139E1F90528F547B6711241FBED3
:100C5000CFEFD0E1DEBFCDBF13E0A0E0B1E0E0E731
:100C6000FCED02C005900D92A438B107D9F71EE043
:100C7000A4E8B3E001C01D92A43DB107E1F71CE078
:100C8000CCE4DCE004C02297FE010E94326EC03446
:100C9000D107C9F70E9426530C9495060C940000C6
:100CA000FC0188279927E89421912032E9F3293023
:100CB00010F02E30C8F32B3241F02D3239F4689405
:100CC00004C00E947807820F911D219120532A3081
:100CD000C0F31EF4909581959F4F08951F93FC01DA
:100CE00099278827BC01E89411911032E9F3193053
:100CF00010F01E30C8F31B3251F01D3249F46894D5
:100D000006C00E946307610F711D811D911D119125
:100D100010531A30B0F33EF490958095709561951C
:100D20007F4F8F4F9F4F1F910895F8940C94366E0C
:100D3000FB01DC0102C005900D9241505040D8F7F4
:100D40000895FB01DC010D900020E9F71197059053
:100D50000D920020E1F70895FB01DC0105900D9252
:100D60000020E1F70895FB01DC0104C08D910190A2
:100D7000801921F441505040C8F7881B990B089501
:100D8000FB01DC0102C001900D9241505040D8F7A8
:100D90000895DC0101C06D9341505040E0F7089583
:100DA000FB01DC010D900020E9F7119701900D92F5
:100DB0000020E1F70895FC018191861721F0882336
:100DC000D9F7992708953197CF010895FB01DC01E8
:100DD00001900D920020E1F70895FB01DC014150E4
:100DE000504030F08D910190801919F40020B9F72E
:100DF000881B990B0895FB01DC014150504048F0DD
:100E000001900D920020C9F701C01D924150504041
:100E1000E0F70895A0E0B0E0E0E1F7E00C94036EA5
:100E20007C01EB018A01690109C0CE012196F6011E
:100E30000995F70181937F010150104001151105BB
:100E4000A1F7CDB7DEB7E8E00C941F6EA0E0B0E0EC
:100E5000ECE2F7E00C94036EEC017B018A0169017E
:100E600009C0CE012196F70161917F01F601099534
:100E70000150104001151105A1F7CDB7DEB7E8E02C
:100E80000C941F6EFB019F01E8944230C4F0453280
:100E9000B4F44A3029F497FB1EF4909581959F4F46
:100EA000642F77270E94956D805D8A330CF0895DF1
:100EB0008193CB010097A1F716F45DE25193108264
:100EC000C9010C94A507592F482F372F262F660FDD
:100ED000771F881F991F660F771F881F991F620F42
:100EE000731F841F951F660F771F881F991F089512
:100EF0007AE0979F902D879F802D910D1124089562
:100F0000FA01CF93FF93EF932230CCF02532BCF45B
:100F1000C22F2C2F332744275527FF93EF930E948E
:100F2000BC6DEF91FF91605D6A330CF0695D619378
:100F3000B901CA01605070408040904051F7108262
:100F40008F919F91CF910C94A507DC01FC01672F35
:100F500071917723E1F7329704C07C916D93708390
:100F60006291AE17BF07C8F30895DF93CF9300D007
:100F700000D000D0CDB7DEB7DE011196E8EFF2E089
:100F800086E001900D928150E1F786E191E0EAEE72
:100F9000F3E0DF019C011D9221503040E1F7809188
:100FA0008403833019F46AED73E003C0BE016F5F00
:100FB0007F4F84E490E043E450E00E94CE42809171
:100FC0008403833039F08AEE93E0BE016F5F7F4F78
:100FD0000E94574E81E0809314048093150486E0AC
:100FE000809316048091910390919203A0919303B2
:100FF000B09194038093180490931904A0931A0459
:10100000B0931B0480918403833039F484E194E02D
:101010000C966AEC73E00E945F4E80E394E064EC0F
:1010200073E00E94574EA0E0B5E0EDE8F1E002C0A9
:1010300081918D9331E0E339F307D1F790918403E7
:10104000992311F083E001C081E0809306058DE3D0
:101050008093070587E08093080581E08093090568
:10106000AAE0B5E0E4ECF3E002C081918D9383E067
:10107000EA3CF807D1F78CE08093100585E0809377
:101080001105E7E8F1E0A2E1B5E002C081918D939E
:1010900021E0EC38F207D1F727E135E030939903EE
:1010A00020939803913069F582E38093170584E0DB
:1010B00080931805D9011296EAECF3E002C0819101
:1010C0008D9333E0EE3CF307D1F786E380931D0563
:1010D00084E080931E058FE195E0909399038093BF
:1010E0009803DC01EAEDF3E002C081918D9383E087
:1010F000EE3DF807D1F783E295E090939903809352
:10110000980320919703222311F094E001C093E00B
:10111000A0919803B0919903FD0187E38193119603
:101120009C93DF01119681E08183FD01319683E07C
:1011300011968C93DF01119686E08183CD01019693
:101140009093990380939803222339F011962C935E
:1011500001969093990380939803E0919803F091FE
:1011600099038FEF8193F0939903E0939803CF0154
:10117000845194400E94BD4426960FB6F894DEBF79
:101180000FBECDBFCF91DF910895EF92FF920F93E5
:101190001F93CF93DF938C0180918403823009F4F5
:1011A000F8C0833030F4882351F1813009F066C1F2
:1011B0004BC0833021F0843009F060C1EAC00E9446
:1011C0003B4F2091890330918A0340918B035091CA
:1011D0008C03E0908503F0908603009187031091C3
:1011E00088032E0D3F1D401F511F62177307840790
:1011F000950708F443C10E94B50784E018C00E9417
:101200003B4F609391037093920380939303909369
:1012100094031092CA031092CB031092CC03109245
:10122000CD030E94B50781E00E94B80D81E0809354
:1012300084030E943B4F60938D0370938E038093D1
:101240008F03909390031AC10634110508F4D5C09A
:1012500080910D04833409F0D0C02091180430919E
:10126000190440911A0450911B04809191039091AC
:101270009203A0919303B0919403281739074A076A
:101280005B0709F0BAC0C4E0D5E0FE01A8014651F1
:101290005C4FDF01119691819D012F5F3F4F80814F
:1012A000853329F411968C91823009F4C5C0F90177
:1012B000E90FF11DE417F50760F39FC0FE0191915E
:1012C000E980EF0121969333D9F0943340F49330C1
:1012D00089F0963091F0913009F046C008C09A33F9
:1012E00079F09F3F09F451C09633F1F537C08EEC89
:1012F00093E036C086ED93E033C08EED93E030C0CE
:10130000618170E080E090E0982F872F762F66272C
:101310002981620F711D811D911D982F872F762FB6
:1013200066272A81620F711D811D911D982F872FBD
:10133000762F66272B81620F711D811D911D28EE6E
:1013400033E040E050E00E946A6D6093890370933F
:101350008A0380938B0390938C0389C08AED93E07A
:10136000BE010E945F4E83C0E0919503F091960309
:10137000309709F47CC080919703981709F077C0E3
:10138000892FBE014E2D099572C00E94B50782E0DB
:101390004ECF0634110588F180910D04833469F530
:1013A000209118043091190440911A0450911B04A3
:1013B0008091910390919203A0919303B091940333
:1013C000281739074A075B07C1F4E4E0F5E0A801F4
:1013D00046515C4FDF01119691819D012F5F3F4F78
:1013E0008081853321F411968C91853071F1F9015A
:1013F000E90FF11DE417F50768F30E943B4F2091B8
:101400008D0330918E0340918F0350919003205FA4
:10141000384D4F4F5F4F261737074807590748F099
:101420002DC086ED93E00E94344383E080938403D3
:1014300025C01092840322C08AEC93E064E274E039
:101440000E945F4E06511C4F39CF81E00E94A70DCC
:101450000E943B4F609385037093860380938703BC
:10146000909388038091D6038823F9F2DACFCE0DCA
:10147000D11DC017D10708F421CF87CFDF91CF91BD
:101480001F910F91FF90EF900895CF93DF9381E02C
:101490008093E6039091C903892F82958F70805DB8
:1014A00080938A019F70905D90938B0110928403CA
:1014B0000E943B4FEB0104C00E94080E0E94C50829
:1014C00080918403833061F00E943B4F6C1B7D0B45
:1014D0006053754728F40E94C90D882389F3ECCF27
:1014E0000E944A421092E9031092E80390E0809132
:1014F0008403833009F491E0892FDF91CF9108951F
:10150000FF920F931F93CF93DF938C01F62E0E94CF
:101510003B4FEB010CC00E94080E0E948A450E94BE
:101520003B4F6C1B7D0B6053754708F0EFC00E946A
:10153000C90D882381F30E943B4FEB010CC00E9430
:10154000080E0E948A450E943B4F6C1B7D0B605326
:10155000754708F0DBC00E944442882381F710924F
:10156000E2031092E3031092E4031092E5038091EA
:101570009A038F5F80939A038091DE03882361F43E
:1015800088E098E0A8E0B8E08093DE039093DF0362
:10159000A093E003B093E10380919A0390E0906EF2
:1015A0006EED73E045E350E00E94CE42E4E1F4E0EA
:1015B0008CE0DF011D928A95E9F7DF011C9690E02F
:1015C000FF2019F0F801808102C0F80184910F5FBB
:1015D0001F4F8E3241F0882331F09F5FFD01E90FEC
:1015E000F11D8083EDCFFD019193DF01A90FB11DA6
:1015F000882329F7FD01119211961C92DF011196A3
:1016000041E04183FD01319611961C92418386EDA4
:101610002AEE33E0821B32968E0F80931404909151
:101620009A0390931504409316044093190490E094
:101630000E94BD440E943B4F8B0161C00E943B4F02
:10164000601B710B6053754708F060C00E94080E64
:10165000EC01009709F453C00E948A45892B09F0D8
:101660004EC0C634D10508F44AC080910D048533BC
:1016700009F045C080910E04803E09F040C0909171
:101680000F0480919A039817D1F58091150489175A
:10169000B1F58091170490E08F709070892BB1F5AF
:1016A00080911404E82FF0E0EC5EFB4F9E01265180
:1016B0003C4F8081807C39F0329609C0808188233C
:1016C00011F4319604C03196E217F307B8F3CF0155
:1016D0000E962817390798F08181813051F4818561
:1016E000843039F43A9682EE93E0BF010E945F4E57
:1016F00006C0818590E00A96E80FF91FDACF809145
:10170000E203882309F49ACF81E001C080E0DF91F1
:10171000CF911F910F91FF900895482F6AE00E948A
:10172000896D282F30E084E0220F331F8A95E1F77E
:10173000842F0E94896D892F820F0895CF93DF93A4
:10174000EC0180919B0390919C038836910559F59B
:1017500085E49CE068E670E00E94555485E49CE0D6
:1017600060E00E94D75488810E948D0B682F70E042
:101770006F77707085E49CE00E94D75489810E9445
:101780008D0B682F85E49CE00E94D7548A810E94CB
:101790008D0B682F85E49CE00E94D7548B810E94BA
:1017A0008D0B682F2DC08F36910509F04AC085E456
:1017B0009CE06FE670E00E94555485E49CE060E098
:1017C0000E94D75488810E948D0B682F606885E441
:1017D0009CE00E94D75489810E948D0B682F85E47C
:1017E0009CE00E94D7548A810E948D0B682F85E46B
:1017F0009CE00E94D7548B810E948D0B682F6860FB
:1018000085E49CE00E94D7548C810E948D0B682F48
:1018100085E49CE00E94D7548D810E948D0B682F37
:1018200085E49CE00E94D7548E818E510E948D0BDE
:10183000682F85E49CE00E94D75485E49CE00E94D8
:101840001A55DF91CF91089588E690E090939C031C
:1018500080939B0385E49CE068E670E00E94555409
:1018600085E49CE060E00E94D75485E49CE00E94FF
:101870001A558823D9F08FE690E090939C038093CB
:101880009B0385E49CE06FE670E00E94555485E47C
:101890009CE060E00E94D75485E49CE00E941A55C9
:1018A000882321F010929C0310929B0308951F93AC
:1018B000CF93DF93EC0160919B0370919C036115C2
:1018C000710509F46FC085E49CE00E94555485E4DD
:1018D0009CE060E00E94D75485E49CE00E941A5589
:1018E00060919B0370919C0385E49CE047E050E08D
:1018F0000E942B5585E49CE00E946854282F2F7786
:1019000022952F701AE0219F900111248F70820F71
:10191000888385E49CE00E946854282F22952F70CC
:10192000219F900111248F70820F898385E49CE0B0
:101930000E946854282F2F7322952F70219F9001A9
:1019400011248F70820F8A8385E49CE00E94685482
:1019500087708B8385E49CE00E946854282F229531
:101960002F70219F900111248F70820F8C8385E44A
:101970009CE00E946854282F22952F70219F90018F
:1019800011248F70820F8D8385E49CE00E9468543F
:10199000282F2F70225E82958F70819FC0011124A5
:1019A000280F2E83DF91CF911F9108950F931F93DE
:1019B000DF93CF93CDB7DEB727970FB6F894DEBF8E
:1019C0000FBECDBF8E010F5F1F4FA8010E941E49A1
:1019D000C8010E949E0B27960FB6F894DEBF0FBE7B
:1019E000CDBFCF91DF911F910F9108950F931F935A
:1019F000DF93CF93CDB7DEB727970FB6F894DEBF4E
:101A00000FBECDBF8E010F5F1F4FC8010E94570C44
:101A1000C8010E94644A27960FB6F894DEBF0FBE35
:101A2000CDBFCF91DF911F910F91089585E49CE088
:101A30000E942F5508958091A00361E00E943F50BD
:101A400078940895FF920F931F93082F162FF42E6A
:101A5000F8948091A00360E00E943F501F71102B0A
:101A60001EBD0DB407FEFDCFFEBC0DB407FEFDCFBD
:101A70000E941B0D1F910F91FF9008951F93182F27
:101A8000282F30E0207630708091A10390E0281755
:101A9000390799F080EA6FE143E00E94220D412F5F
:101AA00040764093A10350E085E0559547958A958F
:101AB000E1F780E86FE10E94220D1F9108950F93D6
:101AC0001F93182F062F0E943E0D80E4612F402F98
:101AD0000E94220D1F910F9108950F931F93182FAD
:101AE000072F0E945F0D812F8F5F602F0E945F0D77
:101AF0001F910F9108950F931F93182F062FF8949D
:101B00008091A00360E00E943F50802F8F71812B55
:101B10008EBD0DB407FEFDCF1EBC0DB407FEFDCF7C
:101B200007FF04C01EBC0DB407FEFDCF1EB50E940A
:101B30001B0D812F1F910F9108951F93182F0E9445
:101B40003E0D80E0612F0E947B0D1F910895882338
:101B500011F410929F0380919F03882341F488E33E
:101B60000E949D0D682F6E7F88E30E945F0D08958F
:101B70001F93182F88E30E949D0D682F616088E3F2
:101B80000E945F0D112319F481E080939F031F9140
:101B9000089584ED61E10E945F0D82ED61E00E9495
:101BA0005F0D8AEE0E949D0D80FDFBCF82ED60E00F
:101BB0000E945F0D89ED0E949D0D90E0969587959E
:101BC00096958795817008950F931F93CF93DF9318
:101BD000EC018B01F8948091A00360E00E943F50DB
:101BE0008AE38EBD0DB407FEFDCF09C01EBC0DB447
:101BF00007FEFDCF8EB5F80181938F0121972097C5
:101C0000A9F70E941B0DDF91CF911F910F910895AD
:101C10000F931F93DF93CF9300D000D000D0CDB7A8
:101C2000DEB789E30E949D0D882319F400E010E0DF
:101C300048C06091A2037091A30380E00E946D0DE3
:101C400086E090E0BE016F5F7F4F0E94E40D8981C6
:101C50009A819093A3038093A2032B813C81E0910E
:101C60009D03F0919E038D8187FD03C000E010E08D
:101C70000EC0245030408F01015010402017310712
:101C800008F48901C8016AEE73E00E94E40DF801CE
:101C9000E651FC4F10826091A2037091A3038CE087
:101CA0006130780724F08CE06FEF7BE003C0615077
:101CB00070408CE00E946D0D80E86EE140E40E946F
:101CC000220DC80126960FB6F894DEBF0FBECDBF19
:101CD000CF91DF911F910F9108950F931F93CF9391
:101CE000DF938C01EB01F8948091A00360E00E94E7
:101CF0003F508AE78EBD0DB407FEFDCF08C0888136
:101D00008EBD0DB407FEFDCF219601501040011588
:101D10001105A9F70E941B0DDF91CF911F910F9123
:101D20000895CF93DF93EC018CE10E949D0D81FF1C
:101D30000FC080E86FE140E80E94220D80EA6FE169
:101D400040E80E94220D80EA6CE142E00E94220DF0
:101D500082E060E07CE00E946D0DBE016050744F37
:101D600086E00E946D0D8AE760E040E00E94220D4F
:101D7000CE016AEE73E00E946D0E80E86FE148E0EC
:101D80000E94220DDF91CF91089584E061E00E94CE
:101D9000005084E061E00E943F5085E061E00E94D5
:101DA000005087E061E00E94005086E060E00E9401
:101DB000005085E061E00E943F5085E060E00E94B5
:101DC0003F5087E060E00E943F5080E58CBD8DB5BC
:101DD00081608DBD0895EF92FF920F931F93CF9373
:101DE000DF93EB01142F90939E0380939D030CB41B
:101DF00006FC02C00E94C50E1093A003812F61E073
:101E00000E9400500E941B0D8FEF60E04FEF0E9478
:101E1000220D62E070E080E090E00E94494F0E9455
:101E20003B4F7B018C0180E395E7A0E0B0E0E80E3A
:101E3000F91E0A1F1B1F09C00E943B4FE616F7063A
:101E40000807190710F480E084C080E06DE10E946B
:101E50007B0D882389F31092A3031092A20388E0DC
:101E600060E070E00E946D0D8CE060E070E00E9428
:101E70006D0D8AE06FEF7BE00E946D0D84E060E005
:101E80007CE00E946D0D86E06FEF71E10E946D0DA8
:101E900080E00E94B80D88E26FE370E30E946D0D50
:101EA00080E369EF77EF0E946D0D80EC6DE00E949A
:101EB0005F0D81EC60E00E945F0D80E862EC42E320
:101EC0000E94220D86EC62E17CE00E946D0D84ECA4
:101ED00062E10E945F0D8AEC6AEE75E00E946D0D72
:101EE00084EE68810E945F0D85EE69810E945F0D1E
:101EF00082EE6A810E945F0D83EE6B810E945F0D0E
:101F000080EE6C810E945F0D81EE6D810E945F0DFD
:101F100084ED60E10E945F0D86ED60E071E00E945B
:101F20006D0D8AEE0E949D0D80FDFBCF8FE10E941A
:101F30003E0D80E86BE140EC0E94220D80E86FE1ED
:101F400044E00E94220D82E70E949D0D863008F039
:101F50008F5FDF91CF911F910F91FF90EF900895C8
:101F6000EF92FF920F931F93CF93DF93FC01EB014E
:101F70008A0179011092E603009729F08AEC93E038
:101F8000BF010E945F4E209719F0CE010E9434439A
:101F90000115110529F08EED93E0B8010E945F4E06
:101FA000E114F10429F08EEC93E0B7010E945F4E3A
:101FB0000E944A421092E9031092E80381E0DF9107
:101FC000CF911F910F91FF90EF900895AF92BF9224
:101FD000CF92DF92FF920F931F93CF93DF938C01E9
:101FE000EB01F42E1092E60338E341E050E060E0AC
:101FF00070E018C0832F90E0FC01B3E0F595E79501
:10200000BA95E1F7EC55FC4F877090705A016B015F
:1020100004C0AA0CBB1CCC1CDD1C8A95D2F7208105
:102020002A292083315031F784EC93E0BE010E94CD
:10203000574EC80164EC73E04F2D0E94EB0EDF9108
:10204000CF911F910F91FF90DF90CF90BF90AF90F5
:102050000895CF92DF92EF92FF920F931F93DF9339
:10206000CF93CDB7DEB7EB84FC84CD84DE84DE0174
:102070001F9601C0D801F6018491882309F4BCC0E1
:102080000894C11CD11C843209F099C0F60108944F
:10209000C11CD11C8491863409F45FC0873434F4A8
:1020A000843469F0853409F08AC06EC08C34C9F17B
:1020B000833509F445C0883409F081C00DC08D0115
:1020C0000E5F1F4FF701668177818D919C914AE0E9
:1020D00050E00E9442077EC02C91822F992787FDF5
:1020E000909514E0959587951A95E1F78F702F706C
:1020F0002A300CF0295F8A300CF0895F8D010E5F69
:102100001F4FF701A681B781805DFD018193205D9E
:1021100011962C933196D7011796FC93EE93169750
:10212000A9CF8D010C5F1F4F6D917D918D919C9179
:10213000F701468157812AE030E00E9480074AC0BB
:102140008D010E5F1F4F6D917C91D70116968D9179
:102150009C9117970E94E6063DC08D010E5F1F4FB0
:102160002D913C910AC0D7011696ED91FC911797DD
:1021700081931796FC93EE931697F9012F5F3F4FCB
:102180008491882381F776CF8D010E5F1F4F2D91AB
:102190003C910AC0D7011696ED91FC911797819357
:1021A0001796FC93EE931697F999FECF32BD21BD99
:1021B000F89A80B52F5F3F4F882361F75BCFF70117
:1021C00026813781F90181939F01F70137832683A7
:1021D0008D0150CFD70116968D919C911797FC01D8
:1021E00001900020E9F73197E81BF90B8E0F9F1F34
:1021F000F701978386833ECFCF91DF911F910F9197
:10220000FF90EF90DF90CF9008950F931F938C0174
:10221000FC01868160E00E943F5081E090E00E94D6
:10222000B94FF801868161E00E943F5081E090E063
:102230000E94B94FF801868160E00E943F5084E619
:1022400090E00E94B94F1F910F910895CF92DF92B5
:10225000EF92FF920F931F93CF93DF93D82EC92E47
:10226000282F392FC9018C01C0E0D0E0E62EFF24D1
:10227000F801878161E00E940050B7010C2E02C076
:10228000759567950A94E2F76170F80187810E945D
:102290003F5021960F5F1F4FC830D10549F78D2D54
:1022A0009C2D0E940511DF91CF911F910F91FF90FE
:1022B000EF90DF90CF900895CF92DF92EF92FF9250
:1022C0000F931F93CF93DF93D82EC92E282F392F2A
:1022D000C9018C01C0E0D0E0E62EFF24F80187811F
:1022E00061E00E940050B7010C2E02C07595679501
:1022F0000A94E2F76170F80187810E943F502196AD
:102300000F5F1F4FC430D10549F78D2D9C2D0E94C2
:102310000511DF91CF911F910F91FF90EF90DF900A
:10232000CF9008951F93CF93DF93EC01162F8C81EC
:10233000642F0E943F508D818F3F19F060E00E9412
:102340003F508F8584FF05C0CE01612F0E9426116A
:102350000EC0612F70E084E0759567958A95E1F76E
:10236000CE010E945C11CE01612F0E945C11DF91B1
:10237000CF911F91089541E00E94921181E090E079
:10238000089540E00E9492110895EF92FF920F93FA
:102390001F93CF93DF938C017A016770660F660FEE
:1023A000660F60640E94C111C0E0D0E0D801ED91D9
:1023B000FC91D701AC0FBD1F0190F081E02DC80149
:1023C0006C9109952196C830D10581F7DF91CF91A5
:1023D0001F910F91FF90EF900895FC0160896E7F2F
:1023E000608B68600E94C1110895FC016089862F8E
:1023F0008460808B6C60CF010E94C1110895DF93CF
:10240000CF93CDB7DEB728970FB6F894DEBF0FBED7
:10241000CDBF9C01FE013196A6E0B3E088E00D90AF
:1024200001928150E1F7F9018389481710F0482F94
:102430004150E42FF0E0EE0FFF1FEC0FFD1F8181F4
:10244000680F6068C9010E94C11128960FB6F89400
:10245000DEBF0FBECDBFCF91DF91089561E00E9436
:10246000C11180ED97E00E94B94F0895CF93DF939B
:10247000EC01423018F08F8588608F874B8B1C8A67
:10248000222329F0413019F48F8584608F8780E5FD
:1024900093EC0E94B94F8C8160E00E943F508E8186
:1024A00060E00E943F508D818F3F19F060E00E94F4
:1024B0003F506F8564FD1DC0CE0163E00E945C113A
:1024C00084E991E10E94B94FCE0163E00E945C1162
:1024D00084E991E10E94B94FCE0163E00E945C1152
:1024E00086E990E00E94B94FCE0162E00E945C1143
:1024F00016C06062CE010E94C11184E991E10E9480
:10250000B94F6F856062CE010E94C11186E990E0EB
:102510000E94B94F6F856062CE010E94C1116F8524
:102520006062CE010E94C11184E0888BCE010E94BE
:10253000F511CE010E942E1282E0898BCE0166E059
:102540000E94C111DF91CF9108956F927F928F9277
:10255000AF92CF92EF920F931F93DF93CF93CDB7AC
:10256000DEB73C01162F842FF301448325830683B5
:10257000E782C086A18682869D8593879E85948703
:102580009F8595879889968761E00E940050F301A6
:1025900085818F3F19F061E00E940050F301868130
:1025A00061E00E940050112319F0F301178603C067
:1025B00080E1F3018787C30160E141E020E00E94F0
:1025C0003612CF91DF911F910F91EF90CF90AF9086
:1025D0008F907F906F900895FC01A681B7816D93D5
:1025E000B783A68381E090E008951F920F920FB603
:1025F0000F9211242F933F934F935F936F937F9389
:102600008F939F93AF93BF93EF93FF9380917F0737
:102610008F5F80937F0780917F07803128F0E09162
:102620007D07F0917E070995FF91EF91BF91AF91E2
:102630009F918F917F916F915F914F913F912F91DA
:102640000F900FBE0F901F90189589E180933D0762
:10265000109240071092540710925B0710925D078A
:10266000109278071092770782E193E090937607B3
:102670008093750708950E948229AB01BC01909157
:10268000A20720E014C0A22FB0E0FD01EC5FF54FDF
:102690008081882359F0AA0FBB1FAA0FBB1FAC5B18
:1026A000B64F4D935D936D937C9313972F5F2917CE
:1026B00050F30895EF92FF920F931F938091B00112
:1026C000882309F44FC080919A0782958F7009F092
:1026D00049C08091990783FD45C08091D9079091A9
:1026E000DA07A091DB07B091DC070097A105B105DF
:1026F00099F00E9482292091D9073091DA07409100
:10270000DB075091DC072D573E4A4E4F5F4F26178F
:1027100037074807590730F50E9482296093D90787
:102720007093DA078093DB079093DC078091800732
:10273000882329F48CE790E061E00E9409210E943F
:10274000B52E7B018C01611571058105910551F054
:102750000E94444B8091990784FF04C0C801B701CF
:102760000E94D60C1F910F91FF90EF900895AF92A9
:10277000BF92CF92DF92EF92FF920F931F938091BF
:10278000990783FDBDC08091E5079091E607A09170
:10279000E707B091E8070097A105B10511F40E9481
:1027A000422A80919A0782958F7091E0E92EF12C50
:1027B00002C0EE0CFF1C8A95E2F70027F7FC00959B
:1027C000102F0E94714B5B016C01C801B70125E31A
:1027D00030E040E050E00E946A6D2091E5073091C2
:1027E000E6074091E7075091E807260F371F481F7B
:1027F000591F2A153B054C055D0508F081C08091E5
:102800008007882359F48BE698E06FE041E00E944E
:10281000FF118BE698E064E00E94BB110E94714BAF
:102820006093E5077093E6078093E7079093E807C6
:1028300086ED93E00E943D450E943B4F7B018C0159
:102840000E94080E0E948A4586ED93E00E94FF4791
:10285000882361F40E943B4F6E197F09800B910B16
:10286000683C71058105910558F336C080919A073F
:102870008F7002C08F70806680939A0780919A074C
:1028800082958F7090E003979CF40E94714B209189
:10289000E9073091EA074091EB075091EC072F567A
:1028A0003E4A4E4F5F4F261737074807590740F5F6
:1028B0000E94714B6093E9077093EA078093EB07DE
:1028C0009093EC070E94422A8823D1F080919A07C6
:1028D0008F7080939A0714C080919A07282F2295B1
:1028E0002F702F5F2F70922F9295907F8F70892B72
:1028F00080939A0730E0273031050CF0BBCFBECF74
:102900001F910F91FF90EF90DF90CF90BF90AF900D
:102910000895EF92FF920F931F938C018CE397E041
:1029200060E071E040E00E946C6220E6E22E28E068
:10293000F22EC701B8010E94E60602EF17E0C801B7
:1029400065E971E00E94E606C801B7010E94D00661
:10295000C8016EE970E00E94A1061F910F91FF90DF
:10296000EF900895CF93DF93EC0180917C02882350
:1029700061F18091990785FF28C0CE0162E071E086
:1029800043E050E00E94ED06009771F48CE397E07D
:1029900065E971E040E00E946C628823B1F08BE54C
:1029A00097E00E94185B11C0CE010E9489148CE34D
:1029B00097E062EF77E00E946862882331F08CE351
:1029C00097E062EF77E00E944562DF91CF91089532
:1029D0008F929F92AF92BF92CF92DF92EF92FF922F
:1029E0000F931F93DF93CF93CDB7DEB76E970FB6DC
:1029F000F894DEBF0FBECDBFE82E4A015B01809187
:102A00007C02882309F416C1CB01BA0120E831E524
:102A100041E050E00E94BC6DCA01B90142EF57E0AD
:102A20002AE030E00E94800782EF97E00E9489143C
:102A30008091990785FFFEC08CE397E060E071E02C
:102A400040E00E946C628CE397E065E971E040E051
:102A50000E946C62882351F48CE397E065E971E091
:102A600041E00E944962882309F4E4C01D821F826C
:102A70001C821B8287E793E09A8389838E010B5F18
:102A80001F4F42EFC42E47E0D42EC801B60142E4E6
:102A90000E94B060F82E4F89588D698D7A8DC801DB
:102AA0000E943756FF2009F4C5C0C6016CE970E0EA
:102AB0000E94AC06EE20D1F5F60101900020E9F766
:102AC0003197EC19FD09EC0DFD1D8091350A90E060
:102AD000BF014AE050E00E944207C6016AE970E087
:102AE0000E94A106F60101900020E9F73197EC1948
:102AF000FD09EC0DFD1D8091340A90E0BF014AE014
:102B000050E00E944207C60168E970E00E94A106F9
:102B1000F60101900020E9F73197EC19FD09EC0D61
:102B2000FD1D8091360A9091370A5AC0C60164E9AA
:102B300070E00E94A106EE2DF0E0EE0FFF1FE456BC
:102B4000FE4F60817181C6010E94D006C60161E915
:102B500070E00E94A10622E0E216B9F033E0E3162D
:102B600099F141E0E41609F040C0F601019000201F
:102B7000E9F73197E25FF7408091CD079091CE075A
:102B8000A091CF07B091D0070FC0F60101900020AF
:102B9000E9F73197E25FF7408091D1079091D20732
:102BA000A091D307B091D407A5019401281B390B3C
:102BB0004A0B5B0BCA01B901EE50F84FAF012AE096
:102BC00030E00E94800711C0F60101900020E9F773
:102BD0003197E25FF740EE50F84F8091F10790E0B7
:102BE000BF014AE050E00E94420702EF17E0C8012F
:102BF0006FE870E00E94A106F80101900020E9F75B
:102C00003197E01BF10BE00FF11FC501B401AF01DB
:102C10002AE030E00E948007C8016BE870E00E9463
:102C2000A106CE010196B8010E940D63CE01059662
:102C30000E949F586E960FB6F894DEBF0FBECDBFB0
:102C4000CF91DF911F910F91FF90EF90DF90CF9088
:102C5000BF90AF909F908F900895CF92DF92EF92A8
:102C6000FF921F936B017C018091810790918207F5
:102C7000A0918307B09184078C579C4FAF4FBF4FF3
:102C80008C159D05AE05BF0578F5C0928107D092E1
:102C90008207E0928307F09284072091F10730E0E9
:102CA00040E050E010918507612F70E080E090E0F7
:102CB0000E946A6D20912E02620F711D811D911D6F
:102CC0001F5F10938507212F30E040E050E00E9405
:102CD000BC6D2093F107103639F483E0B701A601EB
:102CE0000E94E814109285071F91FF90EF90DF90EB
:102CF000CF9008950E94911F0E9410280E94332BAC
:102D000008952F923F924F925F926F927F928F928F
:102D10009F92AF92BF92CF92DF92EF92FF920F936A
:102D20001F93DF93CF93CDB7DEB72C970FB6F894F0
:102D3000DEBF0FBECDBF7B018C014B015C0108944F
:102D4000811C911CA11CB11C80910A020E94F44CB0
:102D50006C0120913C0A30913D0A40913E0A50910D
:102D60003F0AE216F3060407150718F085017401FF
:102D700009C07C010027F7FC0095102FE20EF31E1E
:102D8000041F151F4090A20780919B07282F30E059
:102D90003A83298380919C07282E332460919907D8
:102DA0006695669566956170552481E0682E712C54
:102DB000C601AA2797FDA095BA2F8B839C83AD836C
:102DC000BE8380C0E52DF0E0A981BA81A615B705C4
:102DD00009F474C02614370409F470C0CF01880FB9
:102DE000991F880F991FA4E4CA2EA9E0DA2EC80EF5
:102DF000D91ED6012D913D914D915C912115310542
:102E00004105510509F45AC0DC01AC57B74FB887EA
:102E1000AF838D919D910D90BC91A02D0097A10540
:102E2000B10509F04BC0DF0173E0B695A7957A951F
:102E3000E1F7752D7770FD01ED55F84F808190E039
:102E4000072E02C0959587950A94E2F780FD36C05B
:102E5000A953B84F8C9190E002C0959587957A95CB
:102E6000E2F780FF1AC0EF81F885E082F1820283E9
:102E70001383DA01C9018E0D9F1DA01FB11FF6013A
:102E800080839183A283B383EB80FC800D811E81BC
:102E9000E80EF91E0A1F1B1F10C0AF81B8858D9266
:102EA0009D92AD92BC921397280D391D4A1D5B1D52
:102EB000F601208331834283538361E05394089465
:102EC000611C711C541408F47DCF6170660F660F8D
:102ED000660F80919907877F862B809399072C96A0
:102EE0000FB6F894DEBF0FBECDBFCF91DF911F911B
:102EF0000F91FF90EF90DF90CF90BF90AF909F9099
:102F00008F907F906F905F904F903F902F9008959B
:102F1000AF92BF92CF92DF92EF92FF920F931F93E7
:102F2000DF93CF93CDB7DEB7C754D0400FB6F89438
:102F3000DEBF0FBECDBFE82E0E947A168E2D8150C7
:102F40008E3F28F4BE016F5F7F4F0E942B2DDD2442
:102F5000FF244EEFC42E3CE0A32EB12CAC0EBD1EC0
:102F600041C00F2D10E08FEFE81629F442E050E049
:102F700060E070E012C0EE2009F440C0F501E00FFF
:102F8000F11F80810E94844C0E94B14CAB01BC01B6
:102F9000411551056105710521F1F80123E0F69510
:102FA000E7952A95E1F7E554F84F808190E02F2DC1
:102FB000277002C0959587952A95E2F780FD11C08C
:102FC000F801EE0FFF1FEE0FFF1FEC5BF64F408383
:102FD0005183628373830C5F154FF801C082DD2437
:102FE000D394F3948091A207F81608F4BACFDD20A9
:102FF00051F00E9482290E94811605C04CE350E0E6
:1030000060E070E0CACFC95BDF4F0FB6F894DEBF57
:103010000FBECDBFCF91DF911F910F91FF90EF9029
:10302000DF90CF90BF90AF900895DF92EF92FF9224
:103030000F931F93CF93DF93D82E7A018B01C82F64
:10304000D0E060E00E946D1FFE01EE0FFF1FEE0F4B
:10305000FF1FEC57F74F20813181428153812115A9
:1030600031054105510509F45EC02E153F054007A5
:10307000510708F042C0BE016F5F7F4F80919B07F0
:1030800090E08617970711F180919C0790E08617D2
:103090009707E1F0D092340AFE01EC5FF54F808192
:1030A0008093350AC701821B930B9093370A809354
:1030B000360AE092380AF092390A00933A0A1093DD
:1030C0003B0A80E0B801A7010E94E814FE0163E01A
:1030D000F695E7956A95E1F7EF53F84F808190E018
:1030E0002D2D277002C0959587952A95E2F780FFD0
:1030F00004C08D2D60E00E94A827FE01EE0FFF1F87
:10310000EE0FFF1FDF01AC57B74F1D921D921D92AE
:103110001C921397EC5BF64F10821182128213827D
:10312000CC5FD54F1882DF91CF911F910F91FF9007
:10313000EF90DF9008954F925F926F927F928F92FF
:103140009F92AF92BF92CF92DF92EF92FF920F9336
:103150001F93CF93DF935B016C01909199074424F7
:103160004394492291FD0CC080912202882311F4DE
:10317000FF2408C0F92EF694F69481E0F82211F0AD
:10318000FF24F394EE2459C08E2D90E0FC01E1550C
:10319000F84F3081FC01ED55F84F20815E2C550C25
:1031A000550C550C00E010E0622E7724832E9924F4
:1031B000252D200FC22FD0E0FE01EC5FF54FE081FE
:1031C000E336A0F5442059F0FF2081F1C401002E20
:1031D00002C0959587950A94E2F780FD27C0C30148
:1031E000002E02C0959587950A94E2F780FF06C0ED
:1031F000822FB601A5010E94151818C0EE23B1F068
:10320000FE01EE0FFF1FEE0FFF1FDF01AC57B74FA0
:103210001D921D921D921C921397EC5BF64F10822B
:10322000118212821382CC5FD54F18820F5F1F4F1D
:103230000830110509F0BCCFE3948091A107E8168E
:1032400008F4A2CFDF91CF911F910F91FF90EF90E3
:10325000DF90CF90BF90AF909F908F907F906F90B6
:103260005F904F900895EF92FF920F931F9380917C
:103270009A0782958F7009F054C08091990783FD59
:1032800050C00E9482297B018C012091E10730917E
:10329000E2074091E3075091E4072115310541050C
:1032A0005105F1F08091DD079091DE07A091DF07D5
:1032B000B091E0070097A105B10591F02F553E4A66
:1032C0004E4F5F4F2E153F054007510748F41092AF
:1032D000E5071092E6071092E7071092E80721C071
:1032E0008091DD079091DE07A091DF07B091E007A4
:1032F0000097A105B10549F0875F984FAF4FBF4FC9
:103300008E159F05A007B10760F40E948229609383
:10331000DD077093DE078093DF079093E0070E943C
:10332000094D1F910F91FF90EF90089584B7877F0B
:1033300084BF0E9451280E94C9250E94092B6CE37A
:1033400070E080E090E00E943B4B8091990784FD03
:1033500003C080E090E002C086EF9CE00E94E44B56
:1033600064EF71E080E090E00E94494F0E94822962
:103370000E94BC298091600088618093600081E296
:10338000809360008091600080648093600083EA95
:1033900090E061E00E9409218CE397E060E044E066
:1033A0000E94C862882329F08091990780628093E7
:1033B00099070E94422A882321F080919A078F70F2
:1033C00004C080919A078F70806180939A0764EFA0
:1033D00071E080E090E00E94494F0E9410280E9416
:1033E000714B6093D5077093D6078093D70790935E
:1033F000D8070895EF92FF920F931F93DF93CF9317
:10340000CDB7DEB7C754D0400FB6F894DEBF0FBEBD
:10341000CDBFE090D507F090D6070091D707109167
:10342000D807E114F1040105110511F10E94714B57
:103430002FE030E040E050E0E20EF31E041F151FC5
:10344000E616F7060807190798F4809152026FEF05
:1034500070E0681B71098CE00E94934E1092D507B2
:103460001092D6071092D7071092D80710928007B3
:1034700082E00E94FD1FF82E082F10E086FF1CC17D
:103480000E94714B6093D5077093D6078093D7073E
:103490009093D80780914C026FEF70E0681B710920
:1034A0008CE00E94934E80918007833020F481301D
:1034B00008F0BEC004C0833009F0FEC0ADC0C80132
:1034C0008F7090708230910509F449C08430910565
:1034D00009F483C0019709F0EFC0F7FE1FC08DE12A
:1034E0000E949350892B21F48FEF0E948817E4C02B
:1034F0008EE10E949350892B71F486ED93E060E099
:103500000E9409238BE698E060E041E00E94FF11F1
:1035100081E191E01EC00E943B13CEC08AEC93E093
:1035200060E00E9409238BE698E060E041E00E94A1
:10353000FF118FE091E00E94B7206091930170919C
:1035400094018BE698E04AE050E00E94EE5387E059
:1035500091E00E94B72081E080938007ADC0F7FE24
:1035600032C08FE10E949350892B71F48DEE97E069
:1035700061E00E9409238BE698E060E041E00E9450
:10358000FF1181E091E0E5CF8DE10E949350892BFE
:10359000B9F48BE698E00E942E126091E1077091D9
:1035A000E2078091E3079091E4070E94BC298BE633
:1035B00098E060E041E00E94FF118AEF90E0C9CFFF
:1035C0000E94451F79C08BE698E00E942E1284EC81
:1035D00093E00E94C72082E0BFCFF7FE0CC08BEEC5
:1035E00090E060E00E9409218AED90E061E00E9495
:1035F000092183E0B1CF20919A07822F8F7090E04C
:103600006091A107019670E00E94A96D8F70207FE4
:10361000282B20939A0750C00F70107004301105AA
:1036200009F04AC0F7FE07C0809190070E948817F2
:103630001092800741C08091900790E060918308CC
:1036400070E06F5F7F4F01960E94A96D8093900795
:1036500089EC90E060E00E94092180919007882326
:1036600031F18150BE016F5F7F4F0E942B2D87EC9F
:1036700090E061E00E9409218BE698E060E041E083
:103680000E94FF11609190078BE698E070E04AE09D
:1036900050E00E943F5484EC90E00E94B7208BE6FB
:1036A00098E0BE01645C7F4F0E94525405C084EBD9
:1036B00090E061E00E940921C95BDF4F0FB6F894EA
:1036C000DEBF0FBECDBFCF91DF911F910F91FF9055
:1036D000EF9008952F923F924F925F926F927F9258
:1036E0008F929F92AF92BF92CF92DF92EF92FF9212
:1036F0000F931F93DF93CF93CDB7DEB7C854D0405D
:103700000FB6F894DEBF0FBECDBF8091100280933C
:103710009B078091820280939C070E9482294B0123
:103720005C010E94080E0E948A459093870780934F
:103730008607009721F086519C4F0E949939A895E1
:1037400010927F070E94FA1980918C0790918D0743
:10375000A0918E07B0918F0788159905AA05BB0522
:1037600009F464C380928C0790928D07A0928E0713
:10377000B0928F0780918007882321F40E948229CC
:103780000E94BC298091990781FF10C08091950704
:1037900090919607A0919707B0919807881699067F
:1037A000AA06BB0690F00E944F240FC08091950797
:1037B00090919607A0919707B0919807881699065F
:1037C000AA06BB0610F40E945F240E944620909136
:1037D00099079695917080919D07869581708917BC
:1037E000C9F0992349F08092D1079092D207A09214
:1037F000D307B092D40705C082E0B501A4010E94AE
:10380000E81490919907927080919D078D7F892B84
:1038100080939D07909199079695969591708091C8
:103820009D078695869581708917C9F0992349F07F
:103830008092CD079092CE07A092CF07B092D0078A
:1038400005C081E0B501A4010E94E8149091990798
:10385000947080919D078B7F892B80939D07C50174
:10386000B4012CE330E040E050E00E94BC6D7901EF
:103870008A018091880790918907A0918A07B09169
:103880008B07E816F9060A071B0709F4C5C0E09282
:103890008807F092890700938A0710938B075524B5
:1038A00044241E010894211C311CABC0852DB1019C
:1038B0000E942B2DC101B501A4010E943B2C88233D
:1038C00009F49EC000E0852D8F5F29968FAF299760
:1038D00092C0602E772493012F5F3F4F80919B070A
:1038E00090E08217930709F485C080919C0790E0CF
:1038F0008217930709F47EC0D30113E0B695A7950C
:103900001A95E1F7202F2770FD01ED55F84F8081C2
:1039100090E0022E02C0959587950A94E2F780FD0B
:1039200069C0A554B84F8C9190E002C095958795D9
:103930002A95E2F780FD5EC0ECE0F0E0EC0FFD1FA1
:10394000E60DF71D2081222309F454C0F301EE0F88
:10395000FF1FEE0FFF1FEC5BF64F80819181A2816C
:10396000B3810097A105B10509F044C0822F0E94E0
:10397000844C0E94B14C6B017C01898181FF1FC086
:1039800010912E02212F30E040E050E0C701B60137
:103990000E946A6D24E630E040E050E00E94BC6D79
:1039A000C901DA016C017D01143148F49AE0C916AD
:1039B000D104E104F10418F4CC24DD247601F301F0
:1039C000EE0FFF1FEE0FFF1FEC5BF64FC082D182A0
:1039D000E282F382C114D104E104F10459F0E4E07D
:1039E000FAE06E0E7F1E29968FAD2997F301808332
:1039F000442443940F5F8091A207081708F469CF0D
:103A0000539480918308581608F450CF442021F035
:103A1000C501B4010E9481168091990783FFF7C008
:103A2000772486C0872D90E0FC01ED55F84F20816A
:103A3000672C660C660C660CEE24FF24222E3324C1
:103A400061EC462E67E0562E480E591ED62CDE0C31
:103A50000D2D10E098012F5F3F4F80919B0790E064
:103A60008217930709F45BC080919C0790E082174E
:103A7000930709F454C0F801EC5FF54F8081882367
:103A8000A9F0F801EE0FFF1FEE0FFF1FEC5BF64FE2
:103A900080819181A281B38188169906AA06BB060E
:103AA00028F08D2DB501A4010E941518C1010E2C1E
:103AB00002C0959587950A94E2F780FD30C0980181
:103AC000220F331F220F331FF901EC57F74F80816C
:103AD0009181A281B38188169906AA06BB06F8F0E7
:103AE0002C5B364FF90180819181A281B3818816C8
:103AF0009906AA06BB0698F48D2D61E00E946D1F01
:103B0000F201808190E00E2C02C0959587950A9471
:103B1000E2F780FF04C08D2D61E00E94A827089481
:103B2000E11CF11CF8E0EF16F10409F08FCF73945B
:103B30008091A107781608F475CFC501B4010E94E1
:103B40009B180E94102810923C0A10923D0A109275
:103B50003E0A10923F0A7091A20760E080E03FC0E9
:103B6000A62FB0E0FD01EE0FFF1FEE0FFF1FEC5B75
:103B7000F64FE080F180028113818E149F04A0062D
:103B8000B10660F593E0B695A7959A95E1F7A9532C
:103B9000B84F8C9190E0262F277002C0959587959D
:103BA0002A95E2F780FF19C020913C0A30913D0A26
:103BB00040913E0A50913F0AD801C701E216F30630
:103BC0000407150710F4DA01C90180933C0A9093A9
:103BD0003D0AA0933E0AB0933F0A81E06F5F6717EA
:103BE00008F4BECF882399F40E94911F0E941028E8
:103BF0000E94332B80919907877F8093990780914A
:103C0000100280939B078091820280939C07D09042
:103C10009B07DD2009F470C08091160290911C0270
:103C2000C090A207FF2401E010E02D2C3324482E81
:103C3000552466247724492F50E060E070E04C530F
:103C400050406040704050C02F2D30E020163106AB
:103C500009F447C0D90183E0B695A7958A95E1F7A5
:103C6000F7E0EF2EEF20FD01ED55F84F808190E059
:103C70000E2C02C0959587950A94E2F780FF31C01B
:103C8000A755B84F8C9190E002C095958795EA941E
:103C9000E2F780FF26C0220F331F220F331FF901E6
:103CA000EC57F74F80819181A281B381840D951DDE
:103CB000A61DB71D88169906AA06BB0690F02C5BB8
:103CC000364FF90180819181A281B381840F951FC4
:103CD000A61FB71F88159905AA05BB0510F061E05E
:103CE00007C0F3940F5F1F4FFC1408F4ADCF60E0E2
:103CF0008D2D81500E946D1FD0909C07DD2009F40E
:103D000070C08091880290918E02C090A207FF241B
:103D100001E010E02D2C3324482E5524662477240E
:103D2000492F50E060E070E04C53504060407040DC
:103D300050C02F2D30E02016310609F447C0D901BC
:103D400093E0B695A7959A95E1F787E0E82EEF20E6
:103D5000FD01ED55F84F808190E00E2C02C0959545
:103D600087950A94E2F780FF31C0AB54B84F8C912D
:103D700090E002C095958795EA94E2F780FF26C00F
:103D8000220F331F220F331FF901EC57F74F8081A9
:103D90009181A281B381840D951DA61DB71D881642
:103DA0009906AA06BB0690F02C5B364FF90180817C
:103DB0009181A281B381840F951FA61FB71F88151B
:103DC0009905AA05BB0510F061E007C0F3940F5FE9
:103DD0001F4FFC1408F4ADCF60E08D2D81500E9480
:103DE0006D1FC501B4010E949B180E94102880918C
:103DF0008007882389F4C501B40123E030E040E066
:103E000050E00E94BC6D9B01AC012A5E3C4F81E0FA
:103E1000F90160810E946F220E945A130E94B71319
:103E20000E943319C501B4010E942D16C85BDF4FF3
:103E30000FB6F894DEBF0FBECDBFCF91DF911F91BB
:103E40000F91FF90EF90DF90CF90BF90AF909F9039
:103E50008F907F906F905F904F903F902F9008953C
:103E60009C01F999FECF32BD21BDF89A80B5089525
:103E70009C01F999FECF1FBA32BD21BD60BD0FB6BE
:103E8000F894FA9AF99A0FBE0895E0918008F0919B
:103E9000810809950895FC0124EF33E084E0243182
:103EA000380711F440E009C0F999FECFC901019625
:103EB00032BD21BDF89A40B59C019081442331F078
:103EC000992349F0491739F43196E8CF80E09923D6
:103ED00019F481E0089580E00895282F27708695D1
:103EE0008695869590E0662369F0FC01ED55F84FC4
:103EF00081E090E002C0880F991F2A95E2F72081A7
:103F0000282B0DC0FC01ED55F84F81E090E002C078
:103F1000880F991F2A95E2F7809520812823208316
:103F200008951092A3071092A4071092A50710926B
:103F3000A6071092A7071092A807089510926E087E
:103F400010926D0882E093E090936C0880936B0868
:103F5000089580914C026FEF70E0681B71098CE04E
:103F60000E94934E0895609146028DE070E00E9499
:103F7000934E0895EF92FF920F931F93CF93DF9389
:103F8000E82E162F042FF22E662321F0623081F4E2
:103F9000222371F08E2D0E949350892B11F000E0A6
:103FA00024C0FF2011F480E001C080E8082B1DC070
:103FB000C0E0D0E08E2D0E949350892B81F4113007
:103FC00031F0123061F483E0C83ED80744F461E078
:103FD00070E080E090E00E94494F2196EBCFFF20F7
:103FE00019F4C85ED3400CF00068802FDF91CF91A8
:103FF0001F910F91FF90EF9008950F931F93082F3B
:1040000010918208107861E070E080E090E00E94FA
:10401000494F8FE10E949350892B21F48FE1602F4B
:1040200041E013C08EE10E949350892B21F48EE170
:10403000602F42E00AC08DE10E949350892B11F05D
:1040400040E007C08DE1602F44E0212F0E94BA1F9D
:10405000482F8091820890E08F709070242F30E07C
:10406000892B39F42F703070232B71F0842F8064EA
:1040700006C02F703070232B39F4842F8062409358
:1040800082081F910F910895842FF9CF8BE00E9431
:10409000935040E02091280230E08217930709F006
:1040A00041E0440F440F809199078B7F842B8093CC
:1040B000990708951F93182F843690F064E60E94A4
:1040C000896D682F8BE698E070E04AE050E00E942E
:1040D0003F548BE698E060E171E00E94525402C0C8
:1040E0008A30A0F0812F6AE00E94896D0E94896D5C
:1040F000692F8BE698E070E04AE050E00E943F5460
:104100008BE698E060E171E00E945254812F6AE0F2
:104110000E94896D692F8BE698E070E04AE050E0DC
:104120000E943F541F910895EF92FF920F931F93A7
:104130008C018BE6E82E88E0F82EC8016AE070E07A
:104140000E94A96DC7014AE050E00E943F54C80197
:104150006AE070E00E94A96DBC01C7014AE050E02E
:104160000E943F541F910F91FF90EF900895CF93BD
:10417000DF93EC0104C08BE698E00E945F53FE01E0
:10418000219664916623B9F7DF91CF9108950F933B
:104190001F93CF93DF93182F092F8BE698E060E0F1
:1041A00040E00E94FF11212F302FC901EC0110E0E7
:1041B00005C083E793E00E94B7202196688170E0F4
:1041C00094E0759567959A95E1F78BE698E040E164
:1041D00050E00E943F54688170E06F7070708BE611
:1041E00098E040E150E00E943F54143031F48BE6F7
:1041F00098E060E041E00E94FF111F5F1630C9F6B1
:104200008CE693E00E94B720DF91CF911F910F9130
:1042100008950F931F93CF93DF938C01462F8BE666
:1042200098E060E00E94FF11E80104C08BE698E08E
:104230000E945F539E01201B822FFE0121966491F4
:104240006623A1F7992787FD9095C0E1D0E0C81BB0
:10425000D90B05C080E893E00E94B7202197D7FFD3
:10426000F9CFDF91CF911F910F9108950F931F9375
:10427000CF93DF938C01FC01EE0FFF1FE80FF91FB6
:10428000EE0FFF1FEA55FE4F8081918160E00E9492
:10429000092182E593E061E00E9409218BE698E024
:1042A00060E041E00E94FF110331110509F487C06D
:1042B00004311105BCF40C30110509F4AFC00D3008
:1042C000110544F40115110561F10130110509F0E2
:1042D000CCC034C00E301105F1F00131110509F0E8
:1042E000C4C0AAC00C31110509F4BAC00D311105C2
:1042F0004CF40431110509F471C00B31110509F0BA
:10430000B4C0A2C00632110509F459C00732110524
:1043100009F0ABC063C08BE698E062E171E00E94F7
:104320005254F801EE0FFF1FE00FF11FEE0FFF1FB9
:10433000EC55FE4F80810E945A20B5C08091AA01A1
:10434000C82FD0E0E097D7FD05C080E593E00E943C
:10435000B72007C08EE493E00E94B720D095C195A6
:10436000DF4FCE0164E070E00E94A96D8BE698E01B
:104370004AE050E00E943F548CE493E00E94B72052
:10438000CE0164E070E00E94A96D9C01BC0184E054
:10439000660F771F8A95E1F7621B730B29F489E496
:1043A00093E00E94B72006C08BE698E04AE050E018
:1043B0000E943F5484E493E00E94B7207AC082E4D4
:1043C00093E00E94B720F801EE0FFF1FE00FF11FEE
:1043D000EE0FFF1FEC55FE4F60815EC0F801EE0F3F
:1043E000FF1FE00FF11FEE0FFF1FEC55FE4F808106
:1043F0008C3320F080E493E00E94B720F801EE0FA8
:10440000FF1FE00FF11FEE0FFF1FEC55FE4F608105
:1044100070E06C5370408BE698E041C07091F201FF
:1044200060E08091EC01680F711D8BE698E04AE036
:1044300050E00E94EE533DC080910A020E94F44C6D
:10444000BC018BE698E007C00E94B31F6091460252
:104450008BE698E070E04AE050E00E943F5429C0AB
:104460000E94A91F60914C02F3CFF801EE0FFF1FCD
:10447000E00FF11FEE0FFF1FEC55FE4F81816081B1
:10448000813051F4662319F489E393E002C08CE390
:1044900093E00E94B72007C08BE698E070E04AE006
:1044A00050E00E943F540731110519F487E393E06F
:1044B0000FC0C8014397029748F00632110531F04A
:1044C0000732110519F00131110521F482E393E05F
:1044D0000E94B720DF91CF911F910F910895FF9215
:1044E0000F931F93482FF62E8BE698E060E00E9412
:1044F000FF1180919A078F7019F488E693E010C03D
:1045000086E693E00E94B72060919A076F708BE671
:1045100098E070E04AE050E00E943F5484E693E067
:104520000E94B7208091990780FD06C088E593E03E
:1045300061E00E9409212EC0E0919A07EF70F0E03F
:10454000ED55F84F008110E090919A079F70990FF8
:10455000990F990F9F5F910F80911002981721F486
:1045600000FD0EC06DE40DC080918202981721F409
:1045700000FD06C06EE405C000FD02C06FE501C08D
:104580006F2D8BE698E00E945F531F5F183011F08B
:104590000695DACF83E593E00E94B7208BE698E09A
:1045A0006DE041E00E94FF118091990781FD06C0F6
:1045B00082FF09C080912202882329F08BE698E0CF
:1045C00063E00E94BB118BE698E06EE041E00E9440
:1045D000FF118091990785FF05C08BE698E062E0A6
:1045E0000E94BB118BE698E06FE041E00E94FF1152
:1045F00060E080919A0782958F7090E003970CF0AD
:1046000061E08BE698E00E94BB111F910F91FF9033
:104610000895DF92EF92FF920F931F93CF93DF9352
:104620007C01D62E8BE698E00E942E128BE698E055
:1046300060E040E00E94FF118701C0E0D0E0DD2093
:1046400019F0F801638104C0F701EC0FFD1F6081D0
:104650008BE698E070E04AE050E00E943F54C3309F
:1046600021F085E793E00E94B72021960150104089
:10467000C430D10521F7DF91CF911F910F91FF90A9
:10468000EF90DF900895E4E9F2E0AAE1B8E08081DC
:104690008C933697119781E0EE39F807C1F782ECD9
:1046A00097E062EF77E049E250E028E33FE10E94C3
:1046B00026078091FE018F5F8093A10790E053E071
:1046C000880F991F5A95E1F78093A20790913402C1
:1046D0009170809199078E7F892B80939907089517
:1046E0000F931F93CF93DF93EC010AEA82E00E94BD
:1046F000FD1F482F50E09A012F7030702230310595
:1047000041F12430310509F443C02130310509F06D
:1047100093C0209709F493C0CE30D10509F48FC01F
:10472000CC30D10509F48BC0CD30D10509F487C058
:10473000FE01EE0FFF1FEC0FFD1FEE0FFF1FEC55EC
:10474000FE4F90818181891709F479C09F5F908322
:1047500076C0209709F470C0CE30D10509F46CC042
:10476000CC30D10509F468C0CD30D10509F464C05E
:10477000FE01EE0FFF1FEC0FFD1FEE0FFF1FEC55AC
:10478000FE4F9081992309F457C09150908354C0F3
:1047900086FF52C087FF0AC080919402882311F0DF
:1047A000009394020E94432311E04AC0C330D10514
:1047B00039F48091B601882339F1CCE0D0E02BC0E8
:1047C000CC30D10519F4CEE0D0E025C0C531D105FB
:1047D00039F4809122028823B9F4C7E1D0E01BC0EC
:1047E000C231D10539F480911002882369F4C5E102
:1047F000D0E011C0C532D10539F4809182028823FE
:1048000019F4C8E2D0E007C0CE01019669E270E079
:104810000E94A96DEC01FE01EE0FFF1FEC0FFD1FC2
:10482000EE0FFF1FEC55FE4F0480F581E02DE49163
:10483000EF3529F4219603C0882309F457CF10E0FF
:10484000CE010E943621112309F450CF8BE698E067
:104850000E94ED11DF91CF911F910F9108958091EA
:1048600099078E7F80939907109234020E94432308
:1048700008958091990781608093990781E08093E2
:1048800034020E94432308958CEE93E061E977E0BF
:1048900048E050E028E33FE10E9426070895809118
:1048A00099078D7F8093990710929507109296072C
:1048B00010929707109298070E94442408958091BF
:1048C00099078260809399070E944424089546E0E6
:1048D00050E028E33FE10E9426070895FB01108A7B
:1048E00090E024E0880F991F2A95E1F78C559B4FA3
:1048F00040E150E028E33FE10E942607089582EF5F
:1049000097E062EC77E049E250E020E33FE10E946B
:104910000A07A2EFB7E0E4EAF1E08D9180833696D2
:1049200088E0AB31B807C9F78091FE018F5F8093B3
:10493000A10790E033E0880F991F3A95E1F7809343
:10494000A207909134029170809199078E7F892BF4
:1049500080939907089581E997E06CEE73E048E051
:1049600050E020E33FE10E940A078091990790916F
:104970009A07A0919B07B0919C0780939D07909305
:104980009E07A0939F07B093A00708959C01CB01B9
:10499000B90146E050E020E33FE10E940A07089594
:1049A000FB01108A682F70E044E0660F771F4A957C
:1049B000E1F76C557B4FCF0140E150E020E33FE150
:1049C0000E940A070895DF92EF92FF920F931F93C0
:1049D0009C01D62E82EF97E0B9014D2D50E020E3E7
:1049E0003FE10E940A07E2EFF7E020E030E040E01C
:1049F00050E060E038C0908179018A0154E0EE0C0B
:104A0000FF1C001F111F5A95D1F7892F80538A3040
:104A100030F4892F992787FD9095C09719C0892F69
:104A20008154863030F4892F992787FD9095C79758
:104A30000FC0892F8156863028F020E030E040E01A
:104A400050E013C0892F992787FD90958755904096
:104A50009C01442737FD4095542F2E0D3F1D401FCC
:104A6000511F6F5F31966D1530F2B901CA011F9168
:104A70000F91FF90EF90DF900895EF92FF920F93C8
:104A80001F93CF93DF938B017A01C82FD0E064E0AE
:104A9000CC0FDD1F6A95E1F7CC55DB4FCE0166E008
:104AA0000E94E324611571058105910521F101152D
:104AB000110529F0F8016083718382839383CE010D
:104AC000069666E00E94E324611571058105910553
:104AD00091F0E114F10429F0F7016083718382837E
:104AE0009383CE010C9664E00E94E3246115710566
:104AF0008105910511F460E070E0CB01DF91CF9169
:104B00001F910F91FF90EF900895AF92BF92DF92A7
:104B1000EF92FF920F931F93CF93DF9301EC17E077
:104B2000EE24FF2471E0A72EB12CF8011082DE2CB8
:104B3000DD0CDD0CDD0CC0E0D0E08D2D8C2B60E0B9
:104B400070E040E050E00E943D25892B59F095012E
:104B50000C2E02C0220F331F0A94E2F7F801808165
:104B6000822B80832196C830D10539F70894E11C47
:104B7000F11C0F5F1F4FF6E0EF16F104B1F6DF9165
:104B8000CF911F910F91FF90EF90DF90BF90AF906A
:104B90000895EF92FF920F931F93CF93DF9364EFEB
:104BA00071E080E090E00E94494FF999FECF82ECDD
:104BB00097E092BD81BDF89A80B5863D59F4F99988
:104BC000FECF8AEE97E092BD81BDF89A80B58A3A11
:104BD00009F0B4C082EC93E060E00E94092183EB0D
:104BE00093E061E00E940921E2EFF7E0119288E092
:104BF000EA36F807D9F7C0E0D0E000E018E0A801F5
:104C00004C1B5D0B4937510514F048E750E0CE01CD
:104C100062EF77E028E33FE10E942607C858DF4FA4
:104C200088E0C037D80759F70E94442484EF93E006
:104C300064E171E049E050E028E33FE10E9426078B
:104C400084E194E06DE171E04AE050E028E33FE167
:104C50000E94260784E494E067E271E040E250E0BD
:104C600028E33FE10E94260784E894E067E471E0CE
:104C700041E050E028E33FE10E94260783E580936E
:104C8000F2071092F50704EA14E0C1E0D0E0E2EF89
:104C9000EE2EE7E0FE2ECE016AE070E00E94A96DE4
:104CA000605D6093F307CE016AE070E00E94A96D39
:104CB000805D8093F407F70101900020E9F7E25F3F
:104CC000F740C80162EF77E0AF0128E33FE10E94BF
:104CD0002607005F1F4F219687E0043A1807D9F690
:104CE0008FEF8093F2078093F3078093F40780930C
:104CF000F5078093F6078093F70784EA97E062EF61
:104D000077E046E050E028E33FE10E9426078CEB85
:104D100097E062EF77E046E050E028E33FE10E9451
:104D200026070E94432364EF71E080E090E00E9438
:104D3000494FE0918008F091810809950E947F24F5
:104D400084EA97E069EA77E00E94C6248AEA97E05D
:104D50006FEA77E00E94C62480EB97E065EB77E08E
:104D60000E94C62486EB97E06BEB77E00E94C62496
:104D70008CEB97E067EC77E00E94C6240E948525C3
:104D80000E94AB2480E00E94FD1F90E08F70907025
:104D90008130910519F0049779F503C088E290E01D
:104DA00020C083EA93E060E00E94092160ED77E093
:104DB00080E090E00E94494F82E993E060E00E9429
:104DC000092182E893E061E00E94092180E00E94CD
:104DD000FD1F86FFFBCF8BE698E00E942E1280E03D
:104DE00090E00E94702380919402882329F0E09142
:104DF0008008F091810809958CE061E00E940050E4
:104E00008DE061E00E9400500E94A91F0E94B31F24
:104E1000DF91CF911F910F91FF90EF900895EF9246
:104E2000FF920F931F93DC01CB0179018A01139A42
:104E30000E94B94F1398C7010E94B94F1F910F915B
:104E4000FF90EF9008952F923F924F925F926F9252
:104E50007F928F929F92AF92BF92CF92DF92EF920A
:104E6000FF920F931F93DF93CF9300D00F92CDB794
:104E7000DEB74B015C0179018A01DA01C901880FB3
:104E8000991FAA1FBB1F8E0D9F1DA01FB11F582E5B
:104E9000692E7A2ECB2ED801C701F5E0880F991F15
:104EA000AA1FBB1FFA95D1F78E199F09A00BB10B52
:104EB0008983292E3A2E4B2EDD242FC0D501C40123
:104EC0000A8004C0B695A795979587950A94D2F75E
:104ED00080FF07C0652D762D872D9C2DA801970199
:104EE00006C0C801B701252D362D472D5C2D0E9427
:104EF0000F278A819B8101979B838A838F5F9F4FB6
:104F0000E9F6C801B7012981322D432D542D0E94A5
:104F10000F27D394F8E1DF1629F087E190E09B8317
:104F20008A83CCCF0F900F900F90CF91DF911F917C
:104F30000F91FF90EF90DF90CF90BF90AF909F9038
:104F40008F907F906F905F904F903F902F9008953B
:104F50001F93DF93CF93CDB7DEB728970FB6F894A2
:104F6000DEBF0FBECDBF162FBE016F5F7F4FAE01FC
:104F70004B5F5F4F0E943D25AC01112329F06981F1
:104F80007A818B819C8104C06D817E818F8198851F
:104F90009A01369527955695479556954795240F2E
:104FA000351F40E050E00E94232728960FB6F89462
:104FB000DEBF0FBECDBFCF91DF911F91089584E07A
:104FC0000E94714E9C0183E02E3B380718F020E0D0
:104FD00030E024C083E02734380718F021E030E0C7
:104FE0001DC082E02B3E380718F022E030E016C0EA
:104FF00082E0223A380718F023E030E00FC082E068
:105000002536380718F024E030E008C0235332403A
:1050100018F025E030E002C02FEF3FEFC9010895FE
:10502000EF92FF920F931F93CF93DF9383E060E0A3
:105030000E943F5008EA17E08091990780FD02C066
:1050400060E002C0F8016081C7E0D0E0E62EFF24F6
:1050500086E160E00E943F50B7010C2E02C07595BA
:1050600067950A94E2F7617085E10E943F5086E1FE
:1050700061E00E943F502197FFEFCF3FDF0741F7EC
:105080000150104087E0023A1807B1F683E061E072
:105090000E943F50DF91CF911F910F91FF90EF90B1
:1050A00008958F92AF92CF92EF920F931F93DF9359
:1050B000CF93CDB7DEB7A0970FB6F894DEBF0FBE83
:1050C000CDBF81E061E00E94005081E061E00E947C
:1050D0003F5083E061E00E94005083E061E00E9465
:1050E0003F5086E161E00E94005085E161E00E944E
:1050F00000501092A3071092A4071092A5071092D7
:10510000A6071092A7071092A8070E94102881E016
:1051100060E00E943F508BE060E00E9400508BE016
:1051200061E00E943F5080919907816080939907C8
:105130008091990790919A07A0919B07B0919C0745
:1051400080939D0790939E07A0939F07B093A0071D
:1051500088E691E0909392078093910788E394E02A
:10516000909394078093930711E01093A10788E030
:105170008093A2078CE161E00E9400508CE160E026
:105180000E943F5080E061E00E94005080E061E0BA
:105190000E943F50109381008CE061E00E9400501B
:1051A0008DE061E00E9400500E94A91F0E94B31F81
:1051B00000D000D0EDB7FEB73196ADB7BEB71196AF
:1051C0001C921182128213828BE698E061E043E127
:1051D0002FEF02E134E1E32E15E1C12EB6E1AB2E53
:1051E000A7E18A2E0E94A5120F900F900F900F90AA
:1051F0008BE698E060E142E020E00E94361285E410
:105200009CE00E942F55DE011196E1E3F3E088E077
:1052100001900D928150E1F7DE011996E9E2F3E089
:1052200088E001900D928150E1F7DE015196E1E2B4
:10523000F3E088E001900D928150E1F7DE0159968C
:10524000E9E1F3E088E001900D928150E1F78BE60F
:1052500098E061E08E010F5F1F4FA8010E94C51109
:105260001A821B8281E08C838BE698E060E0A801C3
:105270000E94C5118BE698E062E0AE01475F5F4F88
:105280000E94C5118BE698E063E0AE014F5E5F4F70
:105290000E94C5118BE698E064E0AE01475E5F4F67
:1052A0000E94C5118FE160E00E9400508EE160E035
:1052B0000E9400508DE160E00E9400508FE161E0AB
:1052C0000E943F508EE161E00E943F508DE161E01D
:1052D0000E943F500E94240C882329F48091990752
:1052E000806180939907A0960FB6F894DEBF0FBE39
:1052F000CDBFCF91DF911F910F91EF90CF90AF90E5
:105300008F900895EF92FF920F931F930E94714B1D
:105310007B018C016091AA0170E080E090E024E8BC
:1053200033E040E050E00E946A6D9B01AC01205CDC
:10533000384A404050402E0D3F1D401F511FB901BB
:10534000CA011F910F91FF90EF9008950E9482294A
:1053500020E831E541E050E00E94BC6D2D5F3F4FF9
:105360004F4F5F4FCA01B90127E030E040E050E005
:105370000E94BC6D862F0895EF92FF920F931F93AA
:105380007B018C018BE698E060E040E00E94FF1119
:10539000C801B7010E945E4A0E9494208EE793E004
:1053A0000E94B720C801B7010E94584A0E94942069
:1053B0008BE793E00E94B7200E94A629E82FF0E037
:1053C000EE0FFF1FE656FD4F808191810E94B720AE
:1053D00089E793E00E94B720C801B7010E94464ABE
:1053E0000E94942087E793E00E94B720C801B7018C
:1053F0000E94524A0E9494201F910F91FF90EF90BB
:105400000895CF93DF9385E49CE060E570E00E940F
:10541000555485E49CE060E00E94D75485E49CE00C
:105420000E941A55882311F080E029C085E49CE091
:1054300060E570E00E94555485E49CE06AEF0E94AC
:10544000D75485E49CE00E941A5585E49CE060E511
:1054500070E046E050E00E942B5585E49CE00E94FD
:105460005F54892BD1F3C2EFD7E085E49CE00E9422
:105470006854899387E0C83FD807B9F781E0DF9186
:10548000CF910895DF93CF93CDB7DEB728970FB6AE
:10549000F894DEBF0FBECDBF8FEC93E061E00E94B9
:1054A00009210E94714B6093E5077093E607809392
:1054B000E7079093E8076093E9077093EA07809302
:1054C000EB079093EC070E94012A882391F4109235
:1054D000F20789E68093F3078093F4078DE28093C7
:1054E000F50781E38093F607809140028093F707E8
:1054F00005C08091990780688093990782E593E0C1
:1055000062EF77E044E00E94E60F882309F461C06F
:105510009091F20180E02091EC01820F911D909317
:105520009401809393018091B601882349F10E94F0
:10553000450A882309F44DC08091CA038093BC01B9
:105540008091CB038093C2018091CC038093C801EA
:105550008091CD038093CE018091D6038093D401B6
:105560008091D7038093DA018091D8038093E00182
:105570008091D9038093E6010E94432391E02AC0E1
:105580008091BC0189838091C2018A838091C80186
:105590008B838091CE018C838091D4018D83809107
:1055A000DA018E838091E0018F838091E601888704
:1055B000AE014B5F5F4FCE010196BA0120E030E0B3
:1055C0000E94B00F90E0882309F491E081E09827D1
:1055D00001C090E0892F28960FB6F894DEBF0FBE69
:1055E000CDBFCF91DF9108959C01F999FECF32BDD7
:1055F00021BDF89A80B508959C01F999FECF1FBA94
:1056000032BD21BD60BD0FB6F894FA9AF99A0FBE6B
:105610000895A4E0BAE080E090E0FC01EC57F74F79
:105620001082118212821382FC01EC5BF64F108211
:105630001182128213821D920496803C910569F7B3
:1056400010923C0A10923D0A10923E0A10923F0AB4
:10565000F999FECF89E090E092BD81BDF89A80B5BE
:10566000809383080895A4E0BAE080E090E0FC0114
:10567000EC57F74F1082118212821382FC01EC5B0F
:10568000F64F10821182128213821D920496803C82
:10569000910569F710923C0A10923D0A10923E0A59
:1056A00010923F0A089510928308F999FECF1FBA0D
:1056B00089E090E092BD81BD10BC0FB6F894FA9AD3
:1056C000F99A0FBE0895982F80918308981708F0D3
:1056D00041C0992309F43EC0892F90E0019727E447
:1056E00030E0AC01429FC001439F900D529F900D4E
:1056F00011249C01265F3F4F8F5A9F4F24C0F99978
:10570000FECF32BD21BDF89A50B5F999FECF72BDDA
:1057100061BDF89A40B5F999FECF1FBA32BD21BDDF
:1057200040BD0FB6F894FA9AF99A0FBEF999FECFD8
:105730001FBA72BD61BD50BD0FB6F894FA9AF99ABE
:105740000FBE2F5F3F4FB901695B7F4F28173907A5
:1057500009F0D5CF089577FF03C06FEF7FEF22C028
:10576000CB01977074FF03C0909581959F4F76FF92
:105770000BC06091910770919207680F791F77FFB6
:1057800011C060E070E00EC075FF0CC0609193071F
:1057900070919407680F791F85E0603A780714F0DC
:1057A0006FE975E0CB010895BF92CF92DF92EF923F
:1057B000FF920F931F936C01FC01B080E1800E9467
:1057C000822920E831E541E050E00E94BC6D2B0DBC
:1057D000311D411D511DFF2400E010E0CA01B90137
:1057E000A80197010E94BC6DF60160831F910F9183
:1057F000FF90EF90DF90CF90BF9008958F929F928F
:10580000AF92BF92CF92DF92EF92FF920F931F93CE
:105810004C01FC01A180E080FF24EA0CF11C002770
:10582000F7FC0095102F0E948229BB24CC24DD2494
:1058300020E831E541E050E00E94BC6DCA01B901A9
:10584000A60195010E94BC6DE61AF70A080B190B18
:10585000C801B701A60195010E94BC6DF4016083E7
:105860001F910F91FF90EF90DF90CF90BF90AF907E
:105870009F908F9008957F928F929F92AF92BF9248
:10588000CF92DF92EF92FF920F931F93CF93DF930C
:105890006C017A018B01CB01BA010E945E4A4C0176
:1058A000C801B7010E94584AEC01C801B7010E9423
:1058B0004C4AA82EC801B7010E94524AB82EC8010E
:1058C000B7010E94464A782ED6018C9180FFB4C061
:1058D0008295837090E082309105B9F08330910514
:1058E00009F1892BE1F5F601218130E08A2D90E064
:1058F000059667E070E00E94A96D02C03595279576
:105900008A95E2F720FD2BC097C02B2D30E0D60101
:1059100011968C9190E08F7190702817390709F0DB
:105920008BC01DC0C801B70120E831E541E050E05F
:105930000E94BC6DCA01B901F601228130E040E04D
:1059400050E00E94BC6DD60111962C9130E040E0F1
:1059500050E0621773078407950709F06DC0F601E0
:105960008081869586958370A1F0823019F4B0FE0F
:1059700010C062C0813069F4FFE1BF1609F45CC059
:105980008DE1B81621F492E0791609F455C0B0FE05
:1059900053C08CE390E0889E8001899E100D989EF4
:1059A000100D11240C0F1D1FD6018C9186FD30C0E7
:1059B00013966D917C911497C6010E94AB2BF60152
:1059C000C581D6810780F085E02D9C010817190755
:1059D00098F1209729F480E00217130771F526C08B
:1059E000309751F1C801821B930B9C01BF010E94AB
:1059F000956D6E9FC0016F9F900D7E9F900D11243D
:105A000082179307C9F480E0C617D707B4F00EC019
:105A1000E60188E0E82EF12CEC0CFD1C6B817C810A
:105A2000C6010E94AB2B0817190711F481E005C0CD
:105A30002296CE15DF0591F780E0DF91CF911F917F
:105A40000F91FF90EF90DF90CF90BF90AF909F901D
:105A50008F907F900895982F9B01809183089817CD
:105A600068F467E4969FB0011124665F7F4FC90117
:105A700047E450E024EF3AE20E940A070895DF92DB
:105A8000EF92FF920F931F93DF93CF93CDB7DEB7C3
:105A9000C754D0400FB6F894DEBF0FBECDBF2091E3
:105AA0008308821708F046C0222309F443C090E01F
:105AB000019627E430E0829F8001839F100D929F22
:105AC000100D1124065F1F4F97E4D92E7E01089414
:105AD000E11CF11C14C0C701B80147E450E024EFF9
:105AE0003AE20E940A07C80187549040B70147E490
:105AF00050E02CEF3AE20E942607095B1F4F2091ED
:105B000083082D9DC00111240A960817190718F360
:105B1000215020938308F999FECF1FBA89E090E0C5
:105B200092BD81BD20BD0FB6F894FA9AF99A0FBEC6
:105B300081E001C080E0C95BDF4F0FB6F894DEBFA3
:105B40000FBECDBFCF91DF911F910F91FF90EF90CE
:105B5000DF900895982F80918308981710F080E0C7
:105B6000089587E4989FC00111240A9647E450E005
:105B70002CEF3AE20E94260781E00895BC01909143
:105B800083089E3010F080E0089587E4989FC0015C
:105B900011240A9647E450E02CEF3AE20E942607CF
:105BA000209183082F5F20938308F999FECF1FBAB5
:105BB00089E090E092BD81BD20BD0FB6F894FA9ABD
:105BC000F99A0FBE81E008959C01F999FECF1FBAA2
:105BD00032BD21BD60BD0FB6F894FA9AF99A0FBE96
:105BE0000895EF92FF920F93CF93DF93DC01EB01C7
:105BF000722F532F002331F4822F932F9C01F90130
:105C000060E03EC0822F932FFC0160E019C08491B8
:105C1000332727FD309590E02817390769F431962E
:105C20008491882361F411968C918D3329F4872F08
:105C3000952FFC0161E003C0872F952FFC01119681
:105C40002C91222339F1203229F12A3019F16623CF
:105C5000F1F224C08081981771F4319680818823F5
:105C600071F411968C918D3331F4872F952F9C010F
:105C7000F90161E004C0872F952F9C01F90111966D
:105C80009C91992339F0903229F09A3019F06623CB
:105C900009F304C0613011F030E018C07A2F50E0F1
:105CA0004150504002C0299311963A2F371B2C9136
:105CB000222359F0203249F02A3039F0263229F0D7
:105CC000832F90E08417950774F31882E114F10490
:105CD00011F0F7016083832FDF91CF910F91FF9037
:105CE000EF900895CF93DF93FC01EC0137C08B3226
:105CF00011F480E231C0853279F5DF01119691818E
:105D0000392F30533A3070F0892F8156863010F495
:105D1000375208C0892F8154863010F030E002C01D
:105D2000392F3753FD01319611962C91922F9053B4
:105D30009A3070F0822F8156863010F4975208C046
:105D4000822F8154863010F090E002C0922F97533A
:105D5000832F8295807F892B899331968081882338
:105D600031F61882DF91CF9108956F927F928F92D2
:105D70009F92BF92CF92DF92EF92FF920F931F9369
:105D8000DF93CF93CDB7DEB728970FB6F894DEBF79
:105D90000FBECDBF80916402898380916A028A839D
:105DA000809170028B83809176028C83BB243E01AC
:105DB0000894611C711C85E0882E912C8C0E9D1E10
:105DC0006091F0026F5F6093F002C3010E94EC44A7
:105DD0000E943B4F6B017C0188EE93E0A0E0B0E0B5
:105DE000C80ED91EEA1EFB1E0E94080E8C010E94DE
:105DF0008A45012B71F1C4016091F0020E941F429B
:105E0000882339F12D813E814F81588520583E47A6
:105E10004A4A534808C0B39494E1B91689F620E081
:105E200030E040E050E0B901CA0128960FB6F8947E
:105E3000DEBF0FBECDBFCF91DF911F910F91FF90BD
:105E4000EF90DF90CF90BF909F908F907F906F905A
:105E500008950E943B4F6C157D058E059F0520F22D
:105E6000DACFAF92BF92DF92EF92FF920F931F9320
:105E7000CF93DF9300D000D005E717E0ADB7BEB7F2
:105E800012961C930E93119789E895E014969C93B3
:105E90008E9313970E942910FF240F900F900F905C
:105EA0000F90D02EE12E26E8A22E25E0B22EC4E8D7
:105EB000D5E04FC00F2D10E000D000D000D0ADB71E
:105EC000BEB71196EDB7FEB7D182E2821396BC92AF
:105ED000AE921297F80193E0F595E7959A95E1F760
:105EE000ED55F84F808190E098012770307002C026
:105EF000959587952A95E2F78170907015969C93F9
:105F00008E9314970E9429108091A20790E0019728
:105F10002DB73EB72A5F3F4F0FB6F8943EBF0FBE76
:105F20002DBF08171907A1F000D000D0ADB7BEB73C
:105F30001196DC9211971296EC9212971496DC93BC
:105F4000CE9313970E9429100F900F900F900F90EF
:105F5000F3942091A207F21608F4ACCF00D000D041
:105F600000D0EDB7FEB7319685E797E0ADB7BEB785
:105F700012969C938E93119782E795E09383828388
:105F8000248315820E942910EDB7FEB736960FB60E
:105F9000F894FEBF0FBEEDBFDF91CF911F910F911F
:105FA000FF90EF90DF90BF90AF9008958F929F92F7
:105FB000AF92BF92DF92EF92FF920F931F93CF9316
:105FC000DF93EB0100D000D000D0EDB7FEB73196E3
:105FD00005E717E0ADB7BEB712961C930E93119765
:105FE00024EB39E033832283958384830E94291034
:105FF000FF24EDB7FEB736960FB6F894FEBF0FBE7E
:10600000EDBFD02EE12E41EB842E49E0942E3FEAE5
:10601000A32E39E0B32E40C000D000D000D0ADB7E1
:10602000BEB71196EDB7FEB7D182E28213969C926D
:106030008E9212970F2D10E0FE01E00FF11F80816C
:1060400014968C93149715961C920E942910809197
:10605000A10790E001972DB73EB72A5F3F4F0FB6DB
:10606000F8943EBF0FBE2DBF08171907A1F000D04E
:1060700000D0ADB7BEB71196DC9211971296EC9294
:1060800012971496BC92AE9213970E9429100F900B
:106090000F900F900F90F3948091A107F81608F4D9
:1060A000BBCF00D000D085E797E0EDB7FEB7928375
:1060B00081838CEA99E0948383830E9429100F9056
:1060C0000F900F900F90DF91CF911F910F91FF9044
:1060D000EF90DF90BF90AF909F908F9008958DB715
:1060E0009EB70C970FB6F8949EBF0FBE8DBFEDB74D
:1060F000FEB7319685E797E0ADB7BEB712969C9391
:106100008E93119783E59AE09383828389E794E0E5
:10611000958384838EEB99E09783868382EF99E061
:106120009187808783E19AE0938782870E94291074
:106130008DB79EB70C960FB6F8949EBF0FBE8DBF5D
:1061400008950E946F300E94312F80E008958DB72E
:106150009EB70C970FB6F8949EBF0FBE8DBFEDB7DC
:10616000FEB7319685E797E0ADB7BEB712969C9320
:106170008E9311978FE59AE09383828389E794E069
:10618000958384838EEB99E09783868382EF99E0F1
:106190009187808783E19AE0938782870E94291004
:1061A0008DB79EB70C960FB6F8949EBF0FBE8DBFED
:1061B00008958DB79EB70C970FB6F8949EBF0FBE8B
:1061C0008DBFEDB7FEB7319685E797E0ADB7BEB7A7
:1061D00012969C938E93119784E89AE0938382831E
:1061E00089E794E0958384838AE69AE0978386839F
:1061F00083E19AE09187808782EF99E09387828795
:106200000E9429108DB79EB70C960FB6F8949EBFCA
:106210000FBE8DBF08950E94D9308DB79EB70897E5
:106220000FB6F8949EBF0FBE8DBFEDB7FEB7319687
:1062300085E797E0ADB7BEB712969C938E93119702
:1062400080E797E09383828384E494E0958384835A
:1062500088E491E0978386830E9429108DB79EB7CA
:1062600008960FB6F8949EBF0FBE8DBF80E00895CC
:10627000EF92FF920F9362EF77E048E726E435E074
:1062800001E0EE24FF240E94F12D882311F480E127
:1062900005C082EF97E00E94B21481E00F91FF9059
:1062A000EF9008950F931F930E9482290E94D93086
:1062B00000D000D000D0EDB7FEB7319605E717E06B
:1062C000ADB7BEB712961C930E93119784E796E074
:1062D0009383828388EB95E0958384830E942910C1
:1062E00000D0EDB7FEB73196ADB7BEB712961C938E
:1062F0000E93119786E596E09383828386ED90E076
:106300009583848380913A02868317820E942910A4
:106310000F900F90EDB7FEB73196ADB7BEB712969E
:106320001C930E93119783E296E09383828384E417
:1063300094E0958384830E9429108DB79EB70696BA
:106340000FB6F8949EBF0FBE8DBF80E01F910F91D6
:106350000895CF93DF939C011092F207FC01A08176
:10636000B181C0E0D0E00FC09C919D3231F09B32F2
:1063700021F0892F80538A3068F4FE01EE50F84FE7
:10638000908321961196F901808191810A96A81730
:10639000B90750F3CE50D84F18821196F901B18346
:1063A000A08382EF97E00E946E06CB01DF91CF9130
:1063B00008956F927F928F929F92AF92BF92CF92E9
:1063C000DF92EF92FF920F931F93DF93CF9300D052
:1063D0000F92CDB7DEB75C016A01DE011196EEE3E4
:1063E000F3E083E001900D928150E1F7698310E0C2
:1063F00052E0652E712C6C0E7D1E4E010894811C9E
:10640000911C1CC0812F90E0B3014AE050E00E9433
:106410004207C50162EF77E048E7940100E0EE240F
:10642000FF240E94F12D882341F082EF97E00E9423
:106430005006F601E10FF11D80831F5F8091A107D7
:10644000181700F30F900F900F90CF91DF911F91CD
:106450000F91FF90EF90DF90CF90BF90AF909F9003
:106460008F907F906F9008958F929F92AF92BF927E
:10647000CF92DF92EF92FF920F931F93CF93DF9310
:106480006C0162EF77E048E72EE635E001E0EE24AC
:10649000FF240E94F12D882309F488C082EF97E041
:1064A0000E945006EC0197FD7FC08091A20790E00A
:1064B000C817D9070CF078C0C60162EF77E048E74B
:1064C0002BE635E00E94F12D882309F46FC082EF9E
:1064D00097E00E945006182F0E9482294B015C0110
:1064E000112309F45AC0C60162EF77E048E729E6B4
:1064F00035E00E94F12D882309F458C082EF97E01F
:106500000E946E06CB01019780529D4F08F04CC04F
:106510009E012F5F3F4F80919B0790E0821793076A
:1065200009F446C080919C0790E08217930709F414
:106530003FC0FE01B3E0F595E795BA95E1F7F0E0CD
:10654000ED55F84F808190E0AE014770042E02C0F7
:10655000959587950A94E2F780FD2AC0FE01EE0F1B
:10656000FF1FEE0FFF1FEC5BF64F80819181A28130
:10657000B3810097A105B105D9F4CB01A0E0B0E04B
:1065800080839183A283B383CC5FD54F83E68883D6
:10659000C501B4010E94811605C08C2FB501A4016C
:1065A0000E94151881E005C081E103C080E101C0AF
:1065B00080E3DF91CF911F910F91FF90EF90DF90DB
:1065C000CF90BF90AF909F908F900895AF92BF9261
:1065D000CF92DF92EF92FF920F93DF93CF93CDB7DD
:1065E000DEB7C857D0400FB6F894DEBF0FBECDBFA0
:1065F0006C0102EFA02E07E0B02EB50148E724E9B8
:1066000035E001E0EE24FF240E94F12D882311F4EF
:1066100080E135C0C6016E010894C11CD11CB601D1
:1066200048E720E935E001E0EE24FF240E94F12D47
:10663000882321F1C501B60140E250E00E94ED0639
:106640000097E1F4C5010E94722E10921208F50124
:1066500001900020E9F73197E25FF7404E2F4F5F3E
:10666000403208F040E284EF93E062EF77E050E0E0
:1066700024EE3DE20E94260781E001C083E0C85875
:10668000DF4F0FB6F894DEBF0FBECDBFCF91DF91C5
:106690000F91FF90EF90DF90CF90BF90AF90089553
:1066A000EF92FF920F9362EF77E048E726EA35E03A
:1066B00001E0EE24FF240E94F12D882311F182EFE6
:1066C00097E00E94722E10923208A2EFB7E0FD010F
:1066D0008081803209F08D938081882311F031967A
:1066E000F7CFA2EFB7E0FD0101900020E9F7EA1B28
:1066F000FB0B84E494E0BD01AF0124EE3DE20E9477
:1067000026078FEF0F91FF90EF9008952F923F9201
:106710004F925F926F927F928F929F92AF92BF92B1
:10672000CF92DF92EF92FF920F931F93DF93CF935D
:10673000CDB7DEB727970FB6F894DEBF0FBECDBF3B
:106740004C0134EAC32E31E0D32E6624772455243D
:106750001F82AA24BB2422E0222E312C2C0E3D1EA7
:106760001A2D183209F47DC0183109F47AC0AA2014
:1067700009F477C01E3009F474C0103109F471C0F7
:106780002A2D9B2DF60140808181813009F41082F1
:10679000D101E9E3F3E085E001900D928150E1F74A
:1067A000822FBE016D5F7F4F4AE050E00E9442079A
:1067B000C40162EF77E048E7910100E0EE24FF2496
:1067C0000E94F12D882371F1F6018181813011F44D
:1067D000808328C082EF97E00E946E069B01AC0187
:1067E000143111F0173221F4245C3F4F4F4F5F4FAB
:1067F000113141F4C9010E94DF4C282F30E040E004
:1068000050E002C057FD0CC0F601818190E0A0E08D
:10681000B0E082179307A407B50714F0208302C0E5
:10682000F1E0FF83F60180818415D9F0812F81503A
:10683000823010F466246394812F8052843010F4E7
:1068400066246394812F83508B3010F45524539425
:106850001A3119F45524539404C01F3111F47724CC
:1068600073940894A11CB11C86E090E0C80ED91E58
:1068700099E2A916B10409F073CF92EFC92E97E0FF
:10688000D92EC401B60148E722EA35E001E0EE2442
:10689000FF240E94F12D8823E1F0C6010E94722E90
:1068A00010922208C60164E174E00E94474C8823DC
:1068B00081F0F60101900020E9F7EC19FD0984E16F
:1068C00094E0B601AF0124EE3DE20E942607772452
:1068D0007394198282EFC82E87E0D82EC401B601C6
:1068E00048E72CE935E001E07E010894E11CF11C49
:1068F0000E94F12D8823E9F0C6010E94722E1092A9
:106900001208C60164E874E00E94474C882321F114
:10691000F60101900020E9F7EC19FD0984E894E004
:10692000B601AF0124EE3DE20E942607772473945E
:1069300013C08981882381F01092F207F60101903B
:106940000020E9F7E25FF74084E894E0B601AF0188
:1069500024EE3DE20E9426078091B001882339F59C
:10696000C40162EF77E048E728E935E001E0EE2472
:10697000FF240E94F12D8823D1F082EF97E00E943E
:106980006E06162F072FF82EE92E0E947A16612F19
:10699000702F8F2D9E2D0E94444B8091990784FF6C
:1069A00006C0612F702F8F2D9E2D0E94D60CEF8177
:1069B000EE2311F081E121C00E944323662041F0C3
:1069C0001092D9071092DA071092DB071092DC07B9
:1069D000772041F01092DD071092DE071092DF075A
:1069E0001092E007552041F01092E5071092E6075B
:1069F0001092E7071092E80781E027960FB6F89407
:106A0000DEBF0FBECDBFCF91DF911F910F91FF90E1
:106A1000EF90DF90CF90BF90AF909F908F907F903E
:106A20006F905F904F903F902F900895AF92BF92DC
:106A3000CF92DF92EF92FF921F93CF93DF93C4EA3E
:106A4000D1E010E065E7E62E67E0F62E53E4A52ED0
:106A500059E0B52E41E4C42E49E0D42E8881282F78
:106A600030E040E050E0143111F0173221F42C53A3
:106A7000304040405040113141F4822F0E94F44C8C
:106A80009C01442737FD4095542F6C817D81FB018B
:106A900084918F35E9F11A3121F48091990787FDAE
:106AA00037C08DB79EB70A970FB6F8949EBF0FBE3A
:106AB0008DBFEDB7FEB73196ADB7BEB71296FC925B
:106AC000EE921197B382A282758364832683378303
:106AD000408751870E942910EDB7FEB73A960FB64E
:106AE000F894FEBF0FBEEDBF183291F000D000D079
:106AF000ADB7BEB71296FC92EE9211971496DC9247
:106B0000CE9213970E9429100F900F900F900F9024
:106B10001F5F2696193209F0A1CF0E94DF27EDB73B
:106B2000FEB738970FB6F894FEBF0FBEEDBF319693
:106B300025E737E0ADB7BEB712963C932E93119779
:106B40002BE239E0338322839583848385E090E0D0
:106B5000978386830E942910EDB7FEB738960FB64B
:106B6000F894FEBF0FBEEDBFDF91CF911F91FF9054
:106B7000EF90DF90CF90BF90AF9008950E946F305C
:106B80000E94163580E00895AF92BF92CF92DF92B7
:106B9000EF92FF920F931F93DF93CF93CDB7DEB7A2
:106BA000CB54D0400FB6F894DEBF0FBECDBF6C0102
:106BB00062EF77E048E720E539E001E0EE24FF24CA
:106BC0000E94F12D882309F4E5C082EF97E00E942E
:106BD00050065C018FEFA8168FEFB8060CF4DCC0EE
:106BE0008091830890E0A816B9060CF0D5C0C601C4
:106BF00062EF77E048E72BE439E00E94F12D8E0147
:106C0000025C1F4F882361F082EF97E00E94722E92
:106C1000C80162EF77E04CE050E00E94FB0617C02D
:106C2000C8016DED73E00E94AC069FEFA9169FEFBF
:106C3000B90621F48091830890E001C0C501019656
:106C4000BE016A5B7F4F4AE050E00E944207C601E6
:106C50000E94722EDA82C98286010C591F4F0EC023
:106C6000C70168E671E043E050E00E94ED0600973E
:106C700081F00894E11CF11CFA82E982E980FA8033
:106C8000F7018081882309F485C0E016F10640F3FE
:106C900081C083E090E0E80EF91EFA82E9827E016D
:106CA0000894E11CF11CC7010E94A9318B83C70124
:106CB0000E94A9318C83C7010E94A9318D838981EB
:106CC0009A8101969A838983C7010E94A9319F8383
:106CD0008E83C7010E94A93199878887C7010E94C6
:106CE000A9319B878A87C7010E94A9319D878C871C
:106CF00089819A8102969A83898310E02C96FFAE4F
:106D0000EEAE2C972B96DFAC2B972C960FAD2C97D5
:106D10007EE0E72EF12CEC0EFD1E0BC08D2D902F8A
:106D20000E94A9310E945F4CF701E10FF11D8083A1
:106D30001F5F8091A207181788F389819A810296B4
:106D40009A838983CE010E9605C0FC01E10FF11DE7
:106D500010821F5F1033C8F38B818295837083305C
:106D600039F48D81823020F0CE0104960E94D42B1C
:106D7000BE016D5F7F4F9FEFA9169FEFB90621F40B
:106D8000CB010E94BE2D03C08A2D0E94AA2D88230C
:106D900029F402C080E103C081E101C081E0C55B4C
:106DA000DF4F0FB6F894DEBF0FBECDBFCF91DF919E
:106DB0001F910F91FF90EF90DF90CF90BF90AF9019
:106DC0000895EF92FF920F9362EF77E048E724E592
:106DD00039E001E0EE24FF240E94F12D882311F414
:106DE00080E114C082EF97E00E9450069C011816C3
:106DF00019065CF48091830890E0281739072CF479
:106E0000822F0E94632B81E001C081E10F91FF90EE
:106E1000EF900895EF92FF920F9362EF77E048E7CB
:106E200028E539E001E0EE24FF240E94F12D8823BB
:106E300011F480E118C082EF97E00E9450069C0197
:106E40008FEF2F3F380719F40E94532B0BC080910E
:106E5000830890E02817390714F081E104C0822FDD
:106E60000E943F2D81E00F91FF90EF900895BF9217
:106E7000CF92DF92EF92FF920F931F93DF93CF9306
:106E800000D0CDB7DEB78C010E94722E1A83098321
:106E900084E6E82EF12CE00EF11E0DC0C8016CE670
:106EA00071E043E050E00E94ED06009779F00F5F3B
:106EB0001F4F1A83098309811A81F8018081882371
:106EC00009F44EC00E151F0548F34AC00D5F1F4F51
:106ED0001A8309830E947A16FF24EE246E01089417
:106EE000C11CD11CBEEFBB2E2FC0C6010E94A93110
:106EF000AC01009741F10F2D10E0EF2DE695E695DE
:106F0000E695F0E0E554F84F808190E02F2D277052
:106F100002C0959587952A95E2F780FD14C0CA01B5
:106F20000E94B14CF801EE0FFF1FEE0FFF1FEC5B4C
:106F3000F64F60837183828393830C5F154FF80152
:106F4000B082EE24E394F3948091A207F81668F2DD
:106F5000EE2031F00E9482290E94811681E001C05A
:106F600080E10F900F90CF91DF911F910F91FF90D3
:106F7000EF90DF90CF90BF9008958F929F92AF9245
:106F8000BF92CF92DF92EF92FF920F931F93DF9306
:106F9000CF9300D000D0CDB7DEB76C0183E78983F3
:106FA0001A821B821C8210E092E0892E912C8C0E9A
:106FB0009D1E5E010894A11CB11C1DC0812F90E094
:106FC000B4014AE050E00E944207C60162EF77E058
:106FD00048E7950100E0EE24FF240E94F12D88236C
:106FE00049F082EF97E00E94722E812F62EF77E0E6
:106FF0000E946E241F5F8091A2071817F8F2C60145
:107000006DE649EA57E00E94D93184EA97E069EADF
:1070100077E00E946724C60169E64FEA57E00E94C4
:10702000D9318AEA97E06FEA77E00E946724C601C7
:107030006EE645EB57E00E94D93180EB97E065EBB7
:1070400077E00E946724C60164E64BEB57E00E949C
:10705000D93186EB97E06BEB77E00E9467240E94C2
:107060008525C60161E747EC57E00E94D9318CEBDA
:1070700097E067EC77E00E94672481E00F900F9023
:107080000F900F90CF91DF911F910F91FF90EF9094
:10709000DF90CF90BF90AF909F908F900895EF9228
:1070A000FF920F939C0180913A028823B1F4C901A9
:1070B00062EF77E048E72BEB39E001E0EE24FF24B4
:1070C0000E94F12D882351F082EF97E00E94722EEA
:1070D00082EF97E00E944B1F811181E00F91FF909A
:1070E000EF900895882379F080917B0790917C0739
:1070F0002091790730917A07821B930B61E140E080
:107100000E945E43089580917B0790917C072091B7
:10711000790730917A07821B930B60E143E00E946C
:107120005E43109278071092770780E294E0909384
:107130007A078093790790937C0780937B07089563
:10714000CF92DF92EF92FF920F931F93DF93CF9333
:10715000CDB7DEB76E970FB6F894DEBF0FBECDBFCA
:107160007C018CE397E060E771E040E00E946C6294
:107170008CE397E0B7010E946862882309F4CAC0D3
:10718000CE010196B70141E00E9419638DB79EB709
:1071900008970FB6F8949EBF0FBE8DBFEDB7FEB730
:1071A000319625E7C22E27E0D22EADB7BEB7129694
:1071B000DC92CE92119781E495E09383828389E7F4
:1071C00094E0958384838BE894E0978386830E9480
:1071D0002910D7010D900020E9F78D010E191F0924
:1071E000055010400E0D1F1DEDB7FEB738960FB6B7
:1071F000F894FEBF0FBEEDBFC80162E771E044E046
:1072000050E00E94ED06009799F400D000D000D025
:10721000EDB7FEB73196ADB7BEB71296DC92CE92FF
:1072200011978EE395E09383828383EB94E01BC0F8
:10723000C80167E771E044E050E00E94ED06009766
:10724000F1F400D000D000D0EDB7FEB73196ADB765
:10725000BEB71296DC92CE9211978BE395E09383A2
:10726000828382EF94E0958384830E942910EDB796
:10727000FEB736960FB6F894FEBF0FBEEDBF00D036
:1072800000D085E797E0ADB7BEB712969C938E937A
:10729000119788E395E014969C938E9313970E9420
:1072A00029100F900F900F900F9080E00E9472387D
:1072B0008E010B5F1F4F13C0C80160E274E04CE108
:1072C00053E00E94C558AA2797FDA095BA2F8C516C
:1072D0009340A040B04080F080E00E9472382F8937
:1072E000388D498D5A8D8F859889A989BA89281733
:1072F00039074A075B0701F761E070E080E090E042
:107300000E94494F81E00E947238CE0105960E948A
:107310009F5881E06E960FB6F894DEBF0FBECDBFCA
:10732000CF91DF911F910F91FF90EF90DF90CF9061
:107330000895DF92EF92FF920F931F93CF93DF9305
:10734000EC010E94EA43109278071092770780E2DE
:1073500094E090937A078093790790937C078093C9
:107360007B07BE016B5F7F4FFD8080E2F81621F046
:10737000EC2EDD2EFE0104C0CB010E94523109C16A
:107380008581882359F0803249F08A3039F08F3373
:1073900029F031968F32A1F752E1AEC050E0ACC077
:1073A000C52FD0E0FE01EE0FFF1FEE0FFF1FE855C7
:1073B000FD4F0190F081E02D849190E080179107BE
:1073C00009F0EBC03196849190E04C91242F332743
:1073D00027FD30958217930709F0DFC093E7F91670
:1073E00071F4453709F041C0CC0FDD1FCC0FDD1F14
:1073F000C655DD4FE881F981CB01039647C0AAE667
:10740000FA1699F54F3689F58B010D5F1F4FC801AC
:107410000E944F38882389F50E946F308DB79EB740
:1074200008970FB6F8949EBF0FBE8DBFEDB7FEB79D
:10743000319685E797E0ADB7BEB712969C938E93D1
:10744000119780E794E0938382838091A8019091C3
:10745000A901958384838091A401868317820E9469
:1074600029108DB79EB708968FC08B010D5F1F4FF7
:10747000C8010E944F38882339F1CC0FDD1FCC0F93
:10748000DD1FC655DD4FE881F981C8010995182F28
:10749000882309F47EC08F3FC1F40E94D93000D008
:1074A00000D000D0EDB7FEB7319685E797E0ADB7D5
:1074B000BEB712969C938E9311978DE694E09383BA
:1074C00082838AE294E059C012E00E94A73000D083
:1074D00000D000D0EDB7FEB7319685E797E0ADB7A5
:1074E000BEB712969C938E9311978FE594E0938389
:1074F00082831483158243C00F2D112707FD109539
:10750000DB011196523109F04BCF8091990785FF2D
:1075100040C0C2EFD7E08E2D9D2D9C01D90101C046
:107520008993EA2FEE1915968C911597803229F0E0
:10753000119698E0C231D90799F7F0E0EE50F84F74
:10754000108282EF97E00E94A038882341F50E94C4
:10755000A73000D000D000D0EDB7FEB7319685E758
:1075600097E0ADB7BEB712969C938E93119781E5C5
:1075700094E09383828380E290E0958384830E94E9
:1075800029108DB79EB706960FB6F8949EBF0FBE12
:107590008DBF81E00E94723802C05F5FB3CFDF9180
:1075A000CF911F910F91FF90EF90DF9008952F9250
:1075B0003F924F925F926F927F928F929F92AF9283
:1075C000BF92CF92DF92EF92FF920F931F93DF93C0
:1075D000CF93CDB7DEB7A3970FB6F894DEBF0FBE3B
:1075E000CDBF4C018091990785FD02C080E267C143
:1075F000C40162EF77E048E724E635E001E0EE24DD
:10760000FF240E94F12D8823B9F082EF97E00E94B9
:1076100050067C0121E08E36920708F04DC10E9491
:10762000822920E831E541E050E00E94BC6D59011B
:107630006901CE18DF083EC0C40162EF77E048E779
:107640002EE535E001E0EE24FF240E94F12D882391
:1076500009F434C182EF97E00E946E065B016C0171
:10766000C40162EF77E048E72AE535E00E94F12D9A
:10767000882309F423C1C601B50120E831E541E0C2
:1076800050E00E94DE6D690182EF97E00E946E0675
:1076900020E831E541E050E00E94DE6D59012C15F3
:1076A0003D0508F409C1C9018C199D098E56914008
:1076B00008F002C119821A821B821C82C4012E01A9
:1076C0000894411C511CB20144E025E535E001E07D
:1076D000EE24FF240E94F12D8BA30E94A73000D03E
:1076E00000D005E717E0ADB7BEB712961C930E9316
:1076F000119783E595E014969C938E9313970E94BF
:1077000029107601DD24D3940F900F900F900F90E5
:1077100032EF632E37E0732E29E0822E912C8C0EEF
:107720009D1EC02E012F90E5292E95E0392EA6C072
:10773000C70162EF77E04AE050E00E94420782EF23
:1077400097E00E9489148CE397E062EF77E00E9453
:107750006862882309F48FC019861B8618861F82E9
:10776000E7E7F3E0FE83ED83C40162EF77E041E0F9
:107770000E94B06001C0DD24C40162EF77E047E7FA
:1077800050E020E030E00E94B75B1816190624F0A4
:10779000C4010E949F586FC0FC01EF50F84F8081D8
:1077A0008A3009F41082FBA1FF2351F0C20166EF79
:1077B00077E042E050E00E94ED060097E9F60AC04B
:1077C0008CE791E066EF77E042E050E00E94ED0642
:1077D000009791F2DD20E1F000D000D000D0EDB7AD
:1077E000FEB73196ADB7BEB71196CC9211971296EF
:1077F0000C9333822282758264820E942910EDB735
:10780000FEB736960FB6F894FEBF0FBEEDBF1DC093
:1078100000D000D000D0EDB7FEB73196ADB7BEB7FF
:107820001196CC92119712960C932CE435E0338389
:107830002283758264820E9429108DB79EB70696B6
:107840000FB6F8949EBF0FBE8DBF80917B079091BD
:107850007C072091790730917A07821B930BA2E570
:10786000B3E0A81BB90BA035B1050CF084CF80E0C4
:107870000E94723880CF0894E11CF11CAE14BF0442
:1078800008F056CF00D000D085E797E0EDB7FEB7FF
:10789000928381838AE495E0948383830E942910F4
:1078A0000F900F900F900F9061E070E080E090E0FB
:1078B0000E94494F80E003C081E101C080E1A396AE
:1078C0000FB6F894DEBF0FBECDBFCF91DF911F91F1
:1078D0000F91FF90EF90DF90CF90BF90AF909F906F
:1078E0008F907F906F905F904F903F902F90089572
:1078F000EF92FF920F931F93CF93DF93EC0162EF10
:1079000077E048E724EB35E001E0EE24FF240E9415
:10791000F12D882311F00E943B13CE0162EF77E036
:1079200048E720EB35E001E0EE24FF240E94F12D32
:10793000882371F082EF97E00E945006181619060E
:107940003CF40E94D93081E00E9472380E94451FA9
:10795000CE0162EF77E048E72DEA35E001E0EE2462
:10796000FF240E94F12D882399F08091F207813342
:1079700039F48091990780FD0BC00E94392408C01A
:10798000803331F48091990780FF02C00E942F2438
:10799000CE0162EF77E048E72AEA35E001E0EE2425
:1079A000FF240E94F12D882361F182EF97E00E946D
:1079B0005006EC0118161906F4F40E9482297B0186
:1079C0008C01BE01882777FD8095982F20E13EE04D
:1079D00040E050E00E946A6DE60EF71E081F191F76
:1079E000E0929507F09296070093970710939807F7
:1079F0000E945F2406C0009711F081E103C00E943D
:107A00004F2481E0DF91CF911F910F91FF90EF9074
:107A100008952F923F925F926F927F928F929F92E2
:107A2000AF92BF92CF92DF92EF92FF920F931F938C
:107A3000DF93CF930F92CDB7DEB70E9482295B010F
:107A40006C012DB73EB7285230400FB6F8943EBFB8
:107A50000FBE2DBFEDB7FEB7319605E717E0ADB706
:107A6000BEB712961C930E93119783EE96E0938304
:107A70008283A482B582C682D7828091A107808743
:107A8000118680919907817082871386809199076A
:107A9000869581708487158680919907869586954D
:107AA0008170868717868091950790919607A0919F
:107AB0009707B0919807808B918BA28BB38B84E151
:107AC00094E0958B848B84E894E0978B868B8091EF
:107AD000910790919207918F808F80919307909159
:107AE0009407938F828F8091ED079091EE07A0917C
:107AF000EF07B091F007848F958FA68FB78F809195
:107B0000DD079091DE07A091DF07B091E00780A329
:107B100091A3A2A3B3A38091E1079091E207A09162
:107B2000E307B091E40784A395A3A6A3B7A30E949B
:107B3000291090E0EDB7FEB7B8960FB6F894FEBFE7
:107B40000FBEEDBF78010FED16E023C000D000D0CE
:107B500000D0EDB7FEB73196ADB7BEB71196EC9237
:107B600011971296FC9213830283A92FB0E0AD55B2
:107B7000B84F8C918483158299830E942910998132
:107B80009F5FEDB7FEB736960FB6F894FEBF0FBEF7
:107B9000EDBF8091A107E5E76E2EE7E07E2E9817F6
:107BA000A8F200D000D0ADB7BEB712967C926E920C
:107BB000119785ED96E014969C938E9313970E94EF
:107BC000291099240F900F900F900F90C301562CFD
:107BD000892E79EC672E76E0772E62E5262E63E01B
:107BE000362E76C0A92DB0E0FD01EC5FF54F608127
:107BF000662329F420E030E040E050E025C0CD01CC
:107C0000880F991F880F991FFC01EC57F74FE080F0
:107C1000F18002811381FC01EC5BF64FAE14BF04CE
:107C2000C006D10648F020813181428153812A1952
:107C30003B094C095D0908C0208131814281538193
:107C40002E193F09400B510BEDB7FEB73E970FB60B
:107C5000F894FEBF0FBEEDBF0DB71EB70F5F1F4FED
:107C600051828282F8017382628264831582268344
:107C7000378340875187AA0FBB1FAA0FBB1FAC5782
:107C8000B74F8D919D910D90BC91A02D82879387C8
:107C9000A487B5870E94291080917B0790917C076B
:107CA0002091790730917A07821B930B9101281B51
:107CB000390BADB7BEB71E960FB6F894BEBF0FBE58
:107CC000ADBF203531051CF480E00E9472389394DA
:107CD0008091A207981608F485CFEDB7FEB73E97BE
:107CE0000FB6F894FEBF0FBEEDBF319685E797E063
:107CF000ADB7BEB712969C938E9311978CEA96E01F
:107D0000938382838091340A848315828091350A1B
:107D1000868317828091360A9091370A91878087EF
:107D20008091380A9091390AA0913A0AB0913B0AA1
:107D300082879387A487B5870E942910EDB7FEB785
:107D40003E960FB6F894FEBF0FBEEDBF61E070E047
:107D500080E090E00E94494F0F90CF91DF911F91FA
:107D60000F91FF90EF90DF90CF90BF90AF909F90DA
:107D70008F907F906F905F903F902F9008950E941A
:107D80006F300E94093D80E008952F923F924F92FC
:107D90005F926F927F928F929F92AF92BF92CF929B
:107DA000DF92EF92FF920F931F93DF93CF93CDB7A4
:107DB000DEB7C754D0400FB6F894DEBF0FBECDBFBC
:107DC0000E946F302DB73EB72E5030400FB6F8945A
:107DD0003EBF0FBE2DBFEDB7FEB7319605E717E0EA
:107DE000ADB7BEB712961C930E9311978CEE98E028
:107DF0009383828380918308848315828091A10775
:107E0000868317828EE090E09187808784E090E0FF
:107E1000938782878CE090E0958784870E94291061
:107E2000EE24EDB7FEB73E960FB6F894FEBF0FBE38
:107E3000EDBFF02E012F8CEDC82E88E0D82E1CE06F
:107E4000812E912C8C0E9D1EAF2CB02EB2EC2B2EC1
:107E5000B8E03B2EA5EC4A2EA8E05A2EF2E56F2E94
:107E6000F3E07F2E4AC18E2DBE016F5F7F4F0E94CF
:107E70002B2D898182958370833039F48B818230F8
:107E800020F0CE0102960E94FE2B2DB73EB72A505D
:107E900030400FB6F8943EBF0FBE2DBFEDB7FEB712
:107EA0003196ADB7BEB71196FC92119712960C930E
:107EB00020EE38E0338322838981848315828A818E
:107EC000868317828B81808711860E9429100F90EC
:107ED0000F900F900F90EDB7FEB73196ADB7BEB7CC
:107EE0001196FC92119712960C93D382C2828C81C8
:107EF0009D81958384830E942910EDB7FEB731964A
:107F0000ADB7BEB71196FC92119712960C93D3821F
:107F1000C2828E819F81958384830E942910EDB750
:107F2000FEB73196ADB7BEB71196FC921197129677
:107F30000C93D382C28288859985958384830E941D
:107F40002910EDB7FEB73196ADB7BEB71196FC92CA
:107F5000119712960C9326ED38E0338322838A859D
:107F60009B85958384830E94291010E04DB75EB7EE
:107F70004A5F5F4F26C0E80DF91D80810E94844C46
:107F8000ADB7BEB718970FB6F894BEBF0FBEADBF62
:107F9000EDB7FEB731961196FC92119712960C939D
:107FA00022ED38E033832283A0E0B0E08483958320
:107FB000A683B7830E9429101F5F4DB75EB7485F45
:107FC0005F4F0FB6F8945EBF0FBE4DBFE12FF0E0DC
:107FD0008091A20790E00197E817F90764F2E80D95
:107FE000F91D80810E94844CADB7BEB718970FB6BB
:107FF000F894BEBF0FBEADBFEDB7FEB73196119678
:10800000AC9211971296BC922CEC38E03383228309
:10801000A0E0B0E084839583A683B7830E942910F3
:108020004DB75EB7485F5F4F0FB6F8945EBF0FBEA7
:108030004DBF82EF97E0BE01645C7F4F4CE050E0A3
:108040000E94FB061092FE0700D000D000D0EDB7D2
:10805000FEB73196ADB7BEB71196AC921197129696
:10806000BC9229EC38E03383228342EF57E05583FA
:1080700044830E9429102E2D30E08091830890E0E7
:108080000197ADB7BEB716960FB6F894BEBF0FBE38
:10809000ADBF2817390749F000D000D0EDB7FEB7C3
:1080A000F1820283548243820EC000D000D0ADB76B
:1080B000BEB71196FC92119712960C9312971496D4
:1080C0003C922E9213970E9429100F900F900F90C0
:1080D0000F9080917B0790917C07209179073091D8
:1080E0007A07821B930BF301E81BF90BEA3FF105BA
:1080F0001CF480E00E947238E39480918308E816B3
:1081000008F4B1CE00D000D085E797E0ADB7BEB798
:1081100012969C938E9311978FEB98E014969C93F4
:108120008E9313970E9429100F900F900F900F902D
:1081300061E070E080E090E00E94494F80E0C95B20
:10814000DF4F0FB6F894DEBF0FBECDBFCF91DF91EA
:108150001F910F91FF90EF90DF90CF90BF90AF9065
:108160009F908F907F906F905F904F903F902F9057
:1081700008958F929F92AF92BF92CF92DF92EF922B
:10818000FF920F931F93CF93DF9386EA99E069EAFA
:1081900077E00E94D62F8AE999E06FEA77E00E94A3
:1081A000D62F83E999E065EB77E00E94D62F8BE824
:1081B00099E06BEB77E00E94D62F85E899E061ECBF
:1081C00077E00E94D62F8DE799E067EC77E00E9478
:1081D000D62F00D000D005E717E0ADB7BEB7129696
:1081E0001C930E93119782E799E014969C938E93BB
:1081F00013970E942910FF240F900F900F900F905B
:10820000E02E012F32EF832E37E0932E2DE6A22EA3
:1082100029E0B22E9BE6C92E99E0D92EC2E5D3E023
:1082200051C08F2D62EF77E00E94D02400D000D0A3
:1082300000D0EDB7FEB73196ADB7BEB71196EC9250
:10824000119712960C93B382A282958284820E9427
:1082500029102F2D30E08091A20790E00197EDB713
:10826000FEB736960FB6F894FEBF0FBEEDBF2817C7
:108270003907A1F000D000D0ADB7BEB71196EC928F
:10828000119712960C9312971496DC92CE92139734
:108290000E9429100F900F900F900F9080917B07F4
:1082A00090917C072091790730917A07821B930B7C
:1082B000FE01E81BF90BE035F1051CF480E00E949B
:1082C0007238F3948091A207F81608F4AACF00D070
:1082D00000D000D0EDB7FEB7319685E797E0ADB797
:1082E000BEB712969C938E9311978CE599E0938379
:1082F000828380E190E0958384830E942910EDB70A
:10830000FEB736960FB6F894FEBF0FBEEDBF61E024
:1083100070E080E090E00E94494FDF91CF911F9183
:108320000F91FF90EF90DF90CF90BF90AF909F9014
:108330008F9008950E946F300E94B94080E00895A8
:10834000DF92EF92FF920F931F93CF93DF93D82E7C
:10835000862FBA01213041F4675F7F4F9B0140E0D7
:1083600050E0695070400EC0223029F020E030E02B
:1083700040E050E007C0625070409B0140E050E098
:108380006E5F7F4FE82EFF248AEE93E0E80EF91E21
:108390008B01E7010FC0F881E0E0898190E08E2B2E
:1083A0009F2BA0E0B0E0280F391F4A1F5B1F2296C9
:1083B000025010400230110570F7CB018E7FD701BB
:1083C000A80FB91F6817790779F08C9190E0A0E0A9
:1083D000B0E0BA2FA92F982F882702C040E050E0C4
:1083E000280F391F4A1F5B1FCA01AA27BB27009706
:1083F000A105B10599F7C90180959095ED2DF0E0A3
:10840000E651FC4F90838183DF91CF911F910F91B3
:10841000FF90EF90DF9008951092020410920304F1
:1084200080E48093FE031092FF038093000488E1B0
:108430006EE044E150E020E00E94A0410895282F22
:10844000662321F080910F048617E1F480911004D7
:108450008823C1F4809111048833A1F480910D0424
:108460008B3781F4E22FF92F80913C048383809134
:108470003D04828380913E04818380913F04808308
:1084800081E0089580E008958091400A8695809566
:10849000817008958091CE0380959091CA03892BB5
:1084A0008093D2038091CF0380959091CB03892B49
:1084B0008093D3038091D00380959091CC03892B36
:1084C0008093D4038091D10380959091CD03892B23
:1084D0008093D50308959093550A8093540A70931E
:1084E0005F0A60935E0A5093570A4093560A8CE3E2
:1084F0009BE09093590A8093580A10925B0A10925D
:108500005A0A30935D0A20935C0A309193012091BE
:1085100094018AED98E49093480A8093470A8AE18F
:1085200098E490934A0A8093490A2093430A30932F
:10853000440A81E08093410A8091420A8F5F8770EC
:108540008093420A8093530A08950F931F93BC01AE
:108550000AEE13E0C8010E94574EC801069664EC6B
:1085600073E00E94574E1F910F910895EF92FF9272
:108570000F931F937B010E94A54208E014E0C801FD
:10858000B7010E945F4EC80104976AEC73E00E9435
:108590005F4E1F910F91FF90EF900895EF92FF9221
:1085A0000F931F93CF93DF937C01EB018A018BE440
:1085B0009AE00E94B6428881807F803E49F088819F
:1085C0009981AA81BB818F5F9F4FAF4FBF4F31F41D
:1085D0008AEE93E061E473E00E94574E88E0809356
:1085E000F6031092F70388EF93E067E97AE049E039
:1085F00050E00E9498061092FA0381E180930104F2
:1086000010930E0400930F04F0920C04E0920D04FA
:10861000109210041092120410921304DF91CF9163
:108620001F910F91FF90EF900895EF92FF920F939B
:108630001F9300EF13E0C8010E94A54274E1E72EEA
:10864000F12CE00EF11EC8014896B7010E945F4E62
:10865000C7016AEC73E00E945F4E0E940C421F91BA
:108660000F91FF90EF900895BC011092E9031092D2
:10867000E80381E08093400A86ED93E00E945F4E1C
:1086800008950F931F938C0188969093FA0380931B
:10869000FB030E940C4210921C0410921D04045E05
:1086A0001F4F82E36AE1A80122E00E94A041C801B5
:1086B0004A960E94910E1F910F910895FF920F9379
:1086C0001F93CF93DF93EC01F62E042F10E08091DF
:1086D000600A9091610AA091620AB091630A2B2FFF
:1086E00033274427552720931004A0931104909317
:1086F000120480931304F0921904CE010E944143A6
:108700001F5F011720F79E0140E050E08091600A52
:108710009091610AA091620AB091630A820F931F3F
:10872000A41FB51F8093600A9093610AA093620A08
:10873000B093630ADF91CF911F910F91FF9008953D
:10874000CF93DF939C01862F80618093190464305E
:1087500029F02115310511F421E030E090910E044B
:1087600080910C0480930E0490930C0490910F045C
:1087700080910D0480930F0490930D04C3E1D4E025
:108780008881A901480F511D2C814C832883252FF6
:108790003327219754E0CF30D50791F71D861E86E9
:1087A00080E589871092FA0388E28093FB030E9498
:1087B000154384E08B871C8682E36AE14CE150E03C
:1087C00022E00E94A04186E390E00E94910EDF919A
:1087D000CF9108958091510A9091520A60E00E94D1
:1087E000A0438091100490E0A0E0B0E0BA2FA92F40
:1087F000982F882720911104820F911DA11DB11D72
:10880000BA2FA92F982F882720911204820F911D2B
:10881000A11DB11DBA2FA92F982F882720911304CD
:10882000820F911DA11DB11D8093600A9093610A72
:10883000A093620AB093630A0895E82F40910E0452
:1088400050E0292F30E04217530709F092C0809181
:108850000F048E1709F08DC080911904E82F81FF55
:108860004EC01092FA038CE28093FB030E941543E2
:1088700082E18093190490910E0480910C048093FE
:108880000E0490930C0490910F0480910D0480933A
:108890000F0490930D04E3E1F4E021E030E08081E7
:1088A000A901480F511D44831082252F332731978A
:1088B00054E0EF30F50799F715861686118212827B
:1088C0008091F202838314828D5F8093F20282E0B2
:1088D000818B84E0828B95E0938B148A80E681877C
:1088E000938788E7848782E36AE140E250E022E0F0
:1088F0000E94A0418AE390E00E94910E3AC084FF5A
:1089000038C09091FA0380E02091FB0330E0282BDF
:10891000392B80911804482F50E0A4E055954795D5
:10892000AA95E1F7CA01880F991F880F991F281B84
:10893000390B2451304037FF02C020E030E0309343
:10894000520A2093510A232B69F09A01220F331FF8
:10895000220F331F2E5D3F4F685070406217730720
:1089600040F009C0E0FF05C080E090E060E00E94B8
:10897000A04320E030E0C90108950F931F93DF93D7
:10898000CF930F92CDB7DEB78C01045E1F4F1093CB
:10899000FA030C511040802F845E8093FB0389837F
:1089A0000E940C42085F1F4F10931004898184516C
:1089B00080931104085F1F4F88E26AE1A80121E05B
:1089C0000E94A041C8014A960E94910E0F90CF913B
:1089D000DF911F910F910895FF920F931F939C01B8
:1089E000F62E8BE49AE0B9010E94B64206EF13E03E
:1089F00088E08093F6031092F703C801029667E9B6
:108A00007AE049E050E00E9498068CE48093FB03F2
:108A100081E1809301040E940C4210920E048BE7C6
:108A200080930F048AE080930C04F0920D0410925E
:108A3000100488E38093110410921204109213041E
:108A4000025E1F4F80E3F80111928A95E9F7C80191
:108A50006EE47BE04AE050E00E94980688E26AE11A
:108A600040E450E021E00E94A0418AE590E00E94AD
:108A7000910E1F910F91FF900895EF92FF920F9327
:108A80001F93BC018BE49AE00E94B64206EF13E00C
:108A900088E0F82EF092F6031092F703C8010296D0
:108AA00067E97AE049E050E00E94980684E5809307
:108AB000FB03EE24E394E09201040E940C42F09246
:108AC0000C0410920D0410920E0410920F0485E015
:108AD000809310048091CD038093110410921204AE
:108AE000E0921304C8014E9662E470E048E350E05F
:108AF0000E94C90684E262E240E450E020E00E9465
:108B0000A04182E690E00E94910E1F910F91FF908C
:108B1000EF900895DF92EF92FF920F931F93CF9300
:108B2000DF93EC018091E603882319F0CE010E94C7
:108B3000C508209709F0BFC08091400A8570F1F107
:108B40008091E8039091E903892BC1F50E94C90D3A
:108B50008823A1F181E493E00E94A54288E08093FC
:108B6000F603E6E0FE2EF092F70388EF93E06FE85D
:108B70007AE048E050E00E9498060AE014E0D8014C
:108B80001D92FA94E9F7C8010A9764EC73E00E9419
:108B9000574EC801069666ED73E00E945F4EC8010D
:108BA00004976AEC73E00E945F4E8091400A8860EF
:108BB0008093400A8AE290E00E94910E8091E8033F
:108BC0009091E90301969093E9038093E8038091E3
:108BD000410A813009F003C28091400A81FFFFC140
:108BE00002E00093410A8091F1028F5F8093F102CD
:108BF0008F711091420A1295110F107E182BE09080
:108C0000430AD090440A8BE49AE062EE73E00E943B
:108C1000B64278E0F72EF092F6031092F70388EF51
:108C200093E067E97AE049E050E00E9498068CE220
:108C30008093FB0386E0809301040E940C42E09243
:108C40000E04D0920F048BE080930C0410930D045B
:108C5000E0E1F4E0DF011D92FA94E9F78091F2027D
:108C6000809312048D5F8093F20280E68093180453
:108C70000093190483E080931A0410921B0410924D
:108C80001C0410921D0410921E0410921F040093E5
:108C9000200484E0809321040093220486E28093E0
:108CA000230482E36AE140E250E022E00E94A04116
:108CB0008AE390E0AFC0C932D10508F490C11091A9
:108CC000F603183009F096C18091F703863009F059
:108CD00091C180E194E06AEC73E044E050E00E94CE
:108CE000B306009709F086C18091FF03813029F512
:108CF00080EF93E00E94A5421092FE0382E08093F1
:108D0000FF038AE094E060E074E00E94574E80E048
:108D100094E064EC73E00E94574E80E194E066E0DA
:108D200074E00E945F4E86E094E06AEC73E00E947B
:108D30005F4E8AE290E00E94910E8091400A83FF8C
:108D40004EC11091FF03123009F049C186E094E052
:108D500066ED73E044E050E00E94B306009709F02E
:108D60003EC18BE49AE060E074E00E94574E10939D
:108D7000400A35C1183009F032C18091F7038823C9
:108D800009F02DC18091F803853409F028C188E0ED
:108D900094E06AEC73E044E050E00E94B306009770
:108DA000A9F088E094E062ED73E044E050E00E94B6
:108DB000B306009759F088E094E061E473E044E082
:108DC00050E00E94B306009709F009C180910104A8
:108DD000813019F580910C048830F9F4E091450A4E
:108DE000F091460A309719F084E094E009950E94CA
:108DF000154310920C0480910E04883F28F0809156
:108E00000F048F5F80930F0480910E04885F80931E
:108E10000E04CE010E94910EE2C00E94FB4B8823FB
:108E200051F080910104813131F4CE010E94004C57
:108E3000882309F0D4C0C633D10528F480910104F9
:108E4000863009F0CCC080910E048B3009F0BEC092
:108E500084E094E062EE73E044E050E00E94B306E8
:108E6000009709F0BCC080911904382F82FF13C00D
:108E7000E091470AF091480A309759F080910F0429
:108E800082958695877063E040E050E020E030E016
:108E9000099585E090C09091FA0380E02091FB0352
:108EA000022F10E0082B192B80911804482F50E056
:108EB00064E0559547956A95E1F7CA01880F991FB7
:108EC000880F991F081B190B0451104017FF02C08F
:108ED00000E010E08091410A823079F531FF21C035
:108EE00034FF1FC080E090E060E00E94A04388E172
:108EF00080931904E091490AF0914A0A309719F4D5
:108F000020E030E007C080910D048295869587703F
:108F100009959C0183E08093410AC9010E94414365
:108F20005EC081E08093410A34FF03C080E090E09E
:108F300002C0C801019664E046C0833081F5011586
:108F4000110579F1E091470AF091480A309749F10B
:108F5000440F551F440F551FCE0108974E5D5F4FBC
:108F60008417950708F4AC01C801840F951FC81732
:108F7000D90710F0980103C09E01241B350B809186
:108F80000F0482958695877060E009958091E703CC
:108F9000882319F0C80168E016C0C80108C08530F0
:108FA000F1F030FF0BC08330D1F0C801019669E0C9
:108FB0000E94A04386E08093410A11C0011511056B
:108FC00071F0C80160E00E94A04309C08091930144
:108FD00090919401BE010E941D449C0102C020E0BA
:108FE00030E0C901DF91CF911F910F91FF90EF9079
:108FF000DF900895CA32D10508F0BCCEF0CFBC0195
:10900000809101048130A1F480910C04882381F4C3
:1090100080911404823461F484E094E044E050E0F0
:109020000E94B3069C0180E0232B19F481E008958F
:1090300080E00895CF92DF92EF92FF920F931F93FB
:10904000DF93CF93CDB7DEB728970FB6F894DEBF86
:109050000FBECDBF20E234E03E832D8338872F83BF
:109060009091530A891709F08FC01C821B8282E1FC
:1090700093E09A83898340915A0A50915B0A411583
:109080005105A9F58DB79EB70C970FB6F8949EBF02
:109090000FBE8DBFEDB7FEB73196CE010196ADB7CD
:1090A000BEB712969C938E93119788E19BE09383B1
:1090B00082838091540A9091550A9583848380918C
:1090C0005E0A90915F0A978386838091560A9091F9
:1090D000570A918780878091580A9091590A9387FF
:1090E00082870E9429108DB79EB70C9648C02091A8
:1090F000580A3091590AE090540AF090550A0091AC
:10910000560A1091570A2115310519F06FE771E0E1
:1091100004C062E871E020EA3AE0DA010D90002034
:10912000E9F76D010894C108D108C41AD50A8DB7B2
:109130009EB740970FB6F8949EBF0FBE8DBFEDB798
:10914000FEB73196CE010196ADB7BEB712969C938D
:109150008E93119781EA9AE093838283F582E48269
:10916000178306833187208773876287D586C486F5
:10917000578746870E9429108DB79EB740960FB635
:10918000F8949EBF0FBE8DBF2F8138858D819E8143
:10919000281B390BC90128960FB6F894DEBF0FBE05
:1091A000CDBFCF91DF911F910F91FF90EF90DF9096
:1091B000CF9008950F931F93CF93DF9389019091E0
:1091C000530A891759F0E0915C0AF0915D0A84E036
:1091D00060E070E040E050E009952AC0662341F568
:1091E0002D30310528F1C0915C0AD0915D0A20979D
:1091F000F9F04D505C4F83E891E0BA0143E050E054
:109200000E94ED069C0180E0232B09F081E0609133
:10921000180470E0B4E075956795BA95E1F7660FAC
:10922000771F660F771F6E5D7F4FA801FE010995BE
:1092300080E0DF91CF911F910F9108958F929F92BF
:10924000AF92BF92CF92DF92EF92FF920F931F9354
:10925000CF93DF937B018C01EA012CE330E040E007
:1092600050E00E94BC6D6883C801B7012CE330E078
:1092700040E050E00E94BC6D122F032FF42EE52E2B
:10928000622F732F842F952F2CE330E040E050E0C5
:109290000E94BC6D6983612F702F8F2D9E2D2CE352
:1092A00030E040E050E00E94BC6D122F032FF42EFE
:1092B000E52E622F732F842F952F28E130E040E0B8
:1092C00050E00E94BC6D6A83612F702F8F2D9E2D00
:1092D00028E130E040E050E00E94BC6D79018A0155
:1092E000C801B7016C5F7F4F8F4F9F4F27E030E081
:1092F00040E050E00E94BC6D6F5F6B8320E0AA24C9
:10930000BB24650101C02F5F822E9924F401EE5425
:10931000F84FCF0183709070892B99F4CF0164E6E8
:1093200070E00E94A96D892B39F4CF0160E971E0EA
:109330000E94A96D892B29F48EE691E0A0E0B0E0AF
:1093400004C08DE691E0A0E0B0E0A80EB91ECA1EF0
:10935000DB1EC501A0E0B0E0E816F9060A071B070E
:1093600090F62E83F401EE54F84F83E0882E912C72
:109370008E229F228114910499F4CF0164E670E05B
:109380000E94A96D892B39F4CF0160E971E00E9438
:10939000A96D892B29F48EE691E0A0E0B0E004C02D
:1093A0008DE691E0A0E0B0E0A81AB90ACA0ADB0A8B
:1093B000980187010A191B092C093D09CF0164E6B0
:1093C00070E00E94A96D7C01CF0160E971E00E940C
:1093D000A96DAC01E7E4F3E060E0613051F4811481
:1093E000910449F4E114F10441F44115510529F0C7
:1093F00002C0808103C08CE101C08DE190E0A0E05B
:10940000B0E0081719072A073B0740F0081B190BA3
:109410002A0B3B0B6F5F31966C30F9F66F5F6D83F3
:10942000802F8F5F8C83DF91CF911F910F91FF90E1
:10943000EF90DF90CF90BF90AF909F908F90089566
:10944000EF92FF920F931F937B018C0180917B0A17
:1094500090917C0AA0917D0AB0917E0AE816F906E7
:109460000A071B0771F0C801B70140E75AE00E94E4
:109470001E49E0927B0AF0927C0A00937D0A1093C9
:109480007E0A1F910F91FF90EF9008950E94204A4D
:109490008091750A90E008950E94204A8091730A95
:1094A00090E008950E94204A8091740A90E0089507
:1094B0000E94204A8091710A90E008950E94204AFB
:1094C0008091720A90E008954F925F926F927F921E
:1094D0008F929F92AF92BF92CF92DF92EF92FF92C4
:1094E0000F931F93CF93DF934C01DC0116961C91D1
:1094F000612F70E080E090E020E833E341EE51E03E
:109500000E946A6D5B016C0122EB37E0E12FF0E015
:10951000EE54F84F1DC0C90183709070892BB1F4CF
:10952000C90164E670E00E94A96D892B39F4C90174
:1095300060E971E00E94A96D892B41F480E891E512
:10954000A1E0B0E0A80EB91ECA1EDB1E2F5F3F4F80
:109550002E173F0701F7D40115968C91482E5524FC
:10956000C90164E670E00E94A96D7C01C90160E94F
:1095700071E00E94A96D8C01C1E0D0E093E0692EFA
:10958000712C6222732227C0C230D10591F461147C
:10959000710479F4E114F10419F40115110549F489
:1095A00080E89BE3A6E2B0E0A80EB91ECA1EDB1E4F
:1095B00011C0FE01EA5BFC4F608170E080E090E04A
:1095C00020E831E541E050E00E946A6DA60EB71E2A
:1095D000C81ED91E2196C415D505B4F2D401129621
:1095E0006C9170E080E090E020E13EE040E050E0EF
:1095F0000E946A6D7B018C01F401618170E080E062
:1096000090E02CE330E040E050E00E946A6DE60E0E
:10961000F71E081F191FD4018C91E80EF11C011DC3
:10962000111D14966C9170E061507040882777FD91
:109630008095982F20E831E541E050E00E946A6D66
:10964000E60EF71E081F191FEA0CFB1C0C1D1D1D42
:10965000B701C801DF91CF911F910F91FF90EF905B
:10966000DF90CF90BF90AF909F908F907F906F9042
:109670005F904F9008956093F3027093F40280938B
:10968000F5029093F60208956093660A7093670A54
:109690008093680A9093690A2091F3023091F40252
:1096A0004091F5025091F602260F371F481F591FAF
:1096B00020936A0A30936B0A40936C0A50936D0AA8
:1096C00082E090E090936F0A80936E0A0E943B4F75
:1096D0006093770A7093780A8093790A90937A0A54
:1096E0000895EF92FF920F931F931CC02F5F3F4F7F
:1096F0004F4F5F4F2093660A3093670A4093680A82
:109700005093690A88EE93E0A0E0B0E0E80EF91EFD
:109710000A1F1B1FE092770AF092780A0093790AD9
:1097200010937A0A0E943B4FE090770AF090780AF3
:109730000091790A10917A0A6E197F09800B910BBA
:109740002091660A3091670A4091680A5091690A2F
:10975000685E73408040904048F680916A0A90911C
:109760006B0AA0916C0AB0916D0A281739074A0755
:109770005B07E8F0E091640AF091650A3097B9F070
:109780000995611571058105910519F00E94444BF9
:109790000EC020E030E080916E0A90916F0A892B14
:1097A00011F021E030E030936F0A20936E0A60914F
:1097B000660A7091670A8091680A9091690A1F9100
:1097C0000F91FF90EF9008959093650A8093640A3B
:1097D0008091660A9091670AA091680AB091690A1F
:1097E00080936A0A90936B0AA0936C0AB0936D0AF7
:1097F0000E94714B08958091A70A811181E008951C
:10980000CF92DF92EF92FF920F931F93CF93DF934C
:10981000CFE7DAE030E0CC24DD2429C02A814B8177
:1098200080910E0490E0042F10E080179107D9F486
:1098300090910F049217B9F48C818823A1F02091A4
:10984000110430E028503040F0901004EE242E0D2A
:109850003F1DE881F981892F942F64E074E044E191
:1098600054E0099531E00894C11CD11C25968091E3
:10987000A70A90E0C816D9068CF2832FDF91CF910A
:109880001F910F91FF90EF90DF90CF900895FC0112
:10989000CB01F999FECF92BD81BDF89A30B52081F8
:1098A000332349F0222339F00196321711F081E079
:1098B00008953196EECF80E0321381E008958C3325
:1098C000910510F4682F1EC02AE28033920730F40D
:1098D0006CE370E00E94956D655C14C021EE8130F0
:1098E000920730F460E17EE00E94956D64510AC0F9
:1098F0002FEF8E3F920729F08F5F9F4F11F46FEF8C
:1099000001C06EEF862F0895282F30E08C3338F198
:109910008F3E68F48CE390E0A901489F9001499F35
:10992000300D589F300D1124245D3D4018C08D3FEF
:1099300068F480E19EE0A901489F9001499F300DA5
:10994000589F300D1124205C364F09C08E3F29F0FE
:109950008F3F19F42FEF3FEF02C02EEF3FEFC90109
:1099600008952FEF8E3F920749F46091930770910D
:10997000940720919107309192070EC02FEF8F3FEF
:109980009207B9F4609191077091920760567A4FEF
:109990002091930730919407621B730B80E090E055
:1099A0002CE330E040E050E00E946A6D9B01AC0186
:1099B00003C09C0140E050E0B901CA010895CF9373
:1099C000DF93EC01D7FF04C0882799278C1B9D0BE0
:1099D0000E945F4C982FD7FD02C0805802C080E8DB
:1099E000891BDF91CF9108951F93182F90E0805825
:1099F000904097FF03C0909581959F4F0E94844CA3
:109A00009C0117FD03C0309521953F4FC9011F915F
:109A100008950F931F93DF93CF93CDB7DEB72897A9
:109A20000FB6F894DEBF0FBECDBF8091E20388234E
:109A300029F488E59BE060E00E94800A02EF17E0CD
:109A40001C821B8282E193E09A8389831E830D83AB
:109A500018870F838DB79EB70C970FB6F8949EBFEB
:109A60000FBE8DBFEDB7FEB73196CE010196ADB7F3
:109A7000BEB712969C938E9311978BE79BE09383CE
:109A8000828380915E028483158284E194E09783CF
:109A9000868384E894E0918780878091A4018287FF
:109AA00013860E942910D8010D900020E9F7119724
:109AB000A01BB10BA00FB11F29E638E0EDB7FEB730
:109AC0003C960FB6F894FEBF0FBEEDBF50E342E3E5
:109AD00095E213C08C91B90161507040803249F415
:109AE000F9015083FB01408392939F012150304044
:109AF00003C0F90180839B011197F7E0A23FBF07E4
:109B000049F78C91D9018C930091930110919401A4
:109B100080E590E0909394018093930182E79BE02D
:109B2000B90148E55BE026EA3DE40E946B421093F0
:109B300094010093930128960FB6F894DEBF0FBEF0
:109B4000CDBFCF91DF911F910F910895EF92FF92BA
:109B50000F93CF93DF93EB01C651DC4F01C02196E9
:109B60008881882309F49DC08632C9F78BC082EFB3
:109B700097E00E9450069C0185E0213A380720F4C6
:109B80003093920720939107CE0162EF77E048E788
:109B900023EA3BE001E0EE24FF240E94F12D88231C
:109BA00069F082EF97E00E9450069C0185E0213A1F
:109BB000380720F430939407209393070E9444249D
:109BC000CE0162EF77E048E72DE93BE001E0EE24CB
:109BD000FF240E94F12D882391F082EF97E00E94EC
:109BE00050069C018B3F910550F480912E0290E02D
:109BF0002817390721F020932E020E944323CE011B
:109C000062EF77E048E72AE93BE001E0EE24FF2439
:109C10000E94F12D882391F082EF97E00E94500678
:109C20009C018136910550F48091AA0190E028179B
:109C3000390721F02093AA010E944323CE0162EF4D
:109C400077E048E726E93BE001E0EE24FF240E94AC
:109C5000F12D882361F082EF97E00E946E066093F9
:109C6000ED077093EE078093EF079093F0070E9443
:109C700082296093E1077093E2078093E307909352
:109C8000E4070FC0CE0162EF77E048E72AEA3BE045
:109C900001E0EE24FF240E94F12D882309F474CF03
:109CA00066CFDF91CF910F91FF90EF900895DC0187
:109CB000FB0186E001900D928150E1F708959C012F
:109CC000FB0180819181A281B381F901808391831D
:109CD000A283B38308950E946A1B08950E94961977
:109CE0000895982F8E3008F09E5097708091F7025B
:109CF0008295880F880F807C892B80937C008091CF
:109D00007A00806480937A0080917A0086FDFCCF8F
:109D10002091780040917900942F80E030E0282B4A
:109D2000392BC90108951F93CF93DF93182FEB01AF
:109D300061E00E940050209709F44AC0CF3FD1054E
:109D400009F449C0E12FF0E0E05FF34F84918330E4
:109D5000C1F0843028F4813051F08230B1F50CC06C
:109D6000863019F1873049F1843079F514C084B513
:109D7000806884BDC7BD33C084B5806284BDC8BD62
:109D80002EC080918000806880938000D0938900ED
:109D9000C093880024C080918000806280938000FE
:109DA000D0938B00C0938A001AC08091B000806865
:109DB0008093B000C093B30012C08091B000806265
:109DC0008093B000C093B4000AC0C038D1051CF421
:109DD000812F60E002C0812F61E00E943F50DF913F
:109DE000CF911F9108951F920F920FB60F921124D9
:109DF0002F933F938F939F93AF93BF938091AC0A20
:109E00009091AD0AA091AE0AB091AF0A3091B00A1C
:109E10000196A11DB11D232F235D2D3720F02D5755
:109E20000196A11DB11D2093B00A8093AC0A9093B6
:109E3000AD0AA093AE0AB093AF0A8091A80A9091A0
:109E4000A90AA091AA0AB091AB0A0196A11DB11D61
:109E50008093A80A9093A90AA093AA0AB093AB0A88
:109E6000BF91AF919F918F913F912F910F900FBE16
:109E70000F901F9018958FB7F8942091AC0A3091ED
:109E8000AD0A4091AE0A5091AF0A8FBFB901CA0125
:109E90000895EF92FF920F931F937B018C019FB760
:109EA000F8942091A80A3091A90A4091AA0A5091E9
:109EB000AB0A86B5A89B06C08F3F21F02F5F3F4FAE
:109EC0004F4F5F4F9FBF542F432F322F2227280F12
:109ED000311D411D511DDA01C90162E0880F991F32
:109EE000AA1FBB1F6A95D1F7820F931FA41FB51F2E
:109EF000BC0135C09FB7F8942091A80A3091A90AF7
:109F00004091AA0A5091AB0A86B5A89B06C08F3F24
:109F100021F02F5F3F4F4F4F5F4F9FBF542F432F75
:109F2000322F2227280F311D411D511DDA01C90191
:109F3000E2E0880F991FAA1FBB1FEA95D1F7820F95
:109F4000931FA41FB51F861B970B885E934090F24A
:109F50000894E108F1080109110968517C4FE114E6
:109F6000F1040105110531F61F910F91FF90EF905B
:109F700008959C012150304039F0220F331F039780
:109F8000820F931F0197F1F70895789484B582604A
:109F900084BD84B5816084BD85B5826085BD85B58D
:109FA000816085BDEEE6F0E0808181608083E1E83C
:109FB000F0E0108280818260808380818160808374
:109FC000E0E8F0E0808181608083E1EBF0E0808177
:109FD00084608083E0EBF0E0808181608083EAE749
:109FE000F0E08081846080838081826080838081D2
:109FF000816080838081806880831092C100089591
:10A00000CF93DF93482F50E0CA018051944FFC0159
:10A0100034914053544FFA018491882369F190E0C0
:10A02000880F991FFC01EE54F44FA591B491FC01E7
:10A03000E454F44FC591D491662351F42FB7F894AA
:10A040008C91932F909589238C93888189230BC0C1
:10A05000623061F42FB7F8948C91932F90958923F7
:10A060008C938881832B88832FBF06C09FB7F89479
:10A070008C91832B8C939FBFDF91CF910895482FB4
:10A0800050E0CA01805F934FFC012491CA018051C6
:10A09000944FFC0194914053544FFA01349133236F
:10A0A00009F440C0222351F1233071F0243028F408
:10A0B0002130A1F0223011F514C02630B1F0273044
:10A0C000C1F02430D9F404C0809180008F7703C0A0
:10A0D000809180008F7D8093800010C084B58F7741
:10A0E00002C084B58F7D84BD09C08091B0008F7798
:10A0F00003C08091B0008F7D8093B000E32FF0E02B
:10A10000EE0FFF1FE454F44FA591B4912FB7F894CC
:10A11000662321F48C919095892302C08C91892B20
:10A120008C932FBF0895682F70E0CB01805F934F11
:10A13000FC012491CB018051944FFC014491605368
:10A14000744FFB019491992319F420E030E03CC056
:10A15000222351F1233071F0243028F42130A1F072
:10A16000223011F514C02630B1F02730C1F0243070
:10A17000D9F404C0809180008F7703C08091800063
:10A180008F7D8093800010C084B58F7702C084B526
:10A190008F7D84BD09C08091B0008F7703C080910E
:10A1A000B0008F7D8093B000892F90E0880F991FB9
:10A1B0008A53944FFC01A591B4918C9120E030E03A
:10A1C000842311F021E030E0C901089508951F9221
:10A1D0000F920FB60F9211242F933F934F938F93AB
:10A1E0009F93EF93FF934091C6002091F10A309125
:10A1F000F20A2F5F3F4F2F7330708091F30A9091D6
:10A20000F40A2817390759F0E091F10AF091F20A9F
:10A21000EF54F54F40833093F20A2093F10AFF91F7
:10A22000EF919F918F914F913F912F910F900FBE82
:10A230000F901F90189508951F920F920FB60F92CE
:10A2400011242F933F934F938F939F93EF93FF93FB
:10A250004091CE002091790B30917A0B2F5F3F4FC8
:10A260002F73307080917B0B90917C0B28173907EE
:10A2700059F0E091790BF0917A0BE75CF44F408351
:10A2800030937A0B2093790BFF91EF919F918F91EF
:10A290004F913F912F910F900FBE0F901F901895E7
:10A2A000E091CD0BF091CE0BE05CFF4F819191914D
:10A2B00020813181821B930B8F739070892B11F059
:10A2C0000E94E650E091EC0BF091ED0BE05CFF4F4B
:10A2D0008191919120813181821B930B8F739070BA
:10A2E000892B11F00E941B5108951F920F920FB6F7
:10A2F0000F9211242F933F938F939F93EF93FF938C
:10A300002091350B3091360B8091370B9091380BA3
:10A310002817390731F48091C1008F7D8093C100E7
:10A3200014C0E091370BF091380BEB50F54F2081C2
:10A330008091370B9091380B01968F7390709093AA
:10A34000380B8093370B2093C600FF91EF919F91BC
:10A350008F913F912F910F900FBE0F901F901895E6
:10A360001F920F920FB60F9211242F933F938F934A
:10A370009F93EF93FF932091BD0B3091BE0B809183
:10A38000BF0B9091C00B2817390731F48091C90099
:10A390008F7D8093C90014C0E091BF0BF091C00B7A
:10A3A000E358F44F20818091BF0B9091C00B019630
:10A3B0008F7390709093C00B8093BF0B2093CE004F
:10A3C000FF91EF919F918F913F912F910F900FBE31
:10A3D0000F901F901895DC011C96ED91FC911D9734
:10A3E000E05CFF4F2191319180819181281B390BD5
:10A3F0002F733070C9010895DC011C96ED91FC911A
:10A400001D97E05CFF4F20813181E054F040DF0177
:10A41000AE5BBF4F8D919C9111972817390719F4A6
:10A420002FEF3FEF07C08D919C91E80FF91F8081BE
:10A43000282F30E0C9010895DC011C96ED91FC91B4
:10A440001D97E05CFF4F20813181E054F040DF0137
:10A45000AE5BBF4F8D919C9111972817390719F466
:10A460002FEF3FEF10C08D919C911197E80FF91FCE
:10A4700020818D919C91119701968F739070119608
:10A480009C938E9330E0C9010895FC0186859785E1
:10A49000DC01A05CBF4FFC01EE5BFF4F2D913C91B6
:10A4A00011978081918128173907C1F70895CF93BB
:10A4B000DF93EC01EE85FF85E05CFF4F2081318169
:10A4C000E054F0402F5F3F4F2F733070DF01AE5BE1
:10A4D000BF4F8D919C91119728173907D1F3E05CFC
:10A4E000FF4F80819181E054F040E80FF91F6083B5
:10A4F000EE85FF85E05CFF4F31832083EE89FF8985
:10A50000208181E090E00D8C02C0880F991F0A9491
:10A51000E2F7282B208381E090E0DF91CF9108952E
:10A520001F931092C40B1092C30B28EE33E040E04F
:10A5300050E02093C50B3093C60B4093C70B50934C
:10A54000C80B67E573E07093C20B6093C10B81EB9E
:10A550009AE09093CE0B8093CD0B85EF9AE0909389
:10A56000D00B8093CF0B85EC90E09093D20B80932F
:10A57000D10B84EC90E09093D40B8093D30B80ECC0
:10A5800090E09093D60B8093D50B81EC90E0909364
:10A59000D80B8093D70B86EC90E09093DA0B8093E6
:10A5A000D90B14E01093DB0BB3E0B093DC0BA7E006
:10A5B000A093DD0BF5E0F093DE0BE1E0E093DF0B21
:10A5C0001092E30B1092E20B2093E40B3093E50B17
:10A5D0004093E60B5093E70B7093E10B6093E00B15
:10A5E00089E39BE09093ED0B8093EC0B8DE79BE070
:10A5F0009093EF0B8093EE0B8DEC90E09093F10B2A
:10A600008093F00B8CEC90E09093F30B8093F20B23
:10A6100088EC90E09093F50B8093F40B89EC90E03C
:10A620009093F70B8093F60B8EEC90E09093F90BE0
:10A630008093F80B1093FA0BB093FB0BA093FC0BD9
:10A64000F093FD0BE093FE0B1F910895CF93DF93E2
:10A650000E94C54F0E946E4EC0E5D1E50E946B4E30
:10A660002097E1F30E945051F9CFCF92DF92EF9201
:10A67000FF920F931F93CF93DF937C016B018A01AD
:10A68000C0E0D0E00FC0D6016D916D01D701ED9112
:10A69000FC910190F081E02DC7010995C80FD91FE9
:10A6A000015010400115110571F7CE01DF91CF91D6
:10A6B0001F910F91FF90EF90DF90CF900895DC01F4
:10A6C000ED91FC910190F081E02D09950895CF93D3
:10A6D000DF93DB010D900020E9F71197A61BB70B64
:10A6E000EC01E881F9810280F381E02DAD0109954B
:10A6F000DF91CF9108954F925F927F928F929F92B8
:10A70000AF92BF92CF92DF92EF92FF920F931F937F
:10A71000DF93CF93CDB7DEB7A1970FB6F894DEBF26
:10A720000FBECDBF2C01742ECB01223008F42AE0DD
:10A7300019A231E2C32ED12CCC0EDD1E822E99241B
:10A74000AA24BB24672D752FA50194010E94BC6D1E
:10A7500079018A01C801B701A50194010E946A6DBF
:10A76000472D461B0894C108D1084A3014F4405DB7
:10A7700001C0495CF6014083E114F10401051105B3
:10A7800021F07E2C5F2DC801DDCFC201B6010E94F1
:10A790006753A1960FB6F894DEBF0FBECDBFCF9121
:10A7A000DF911F910F91FF90EF90DF90CF90BF90BE
:10A7B000AF909F908F907F905F904F900895DC01B5
:10A7C0002115310541F4ED91FC910190F081E02DCE
:10A7D000642F099508950E947B530895EF92FF928C
:10A7E0000F931F939A017B0100E010E0B801A701CD
:10A7F0000E94DF531F910F91FF90EF900895CF9229
:10A80000DF92EF92FF920F931F93CF93DF93EC01B0
:10A810006A017B012115310541F4E881F98101903C
:10A82000F081E02D642F09951FC02A303105D1F445
:10A8300077FF17C0E881F9810190F081E02D6DE28A
:10A8400009958C0144275527BA014C195D096E09F9
:10A850007F09CE012AE00E947B539801280F391FFF
:10A8600004C02AE00E947B539C01C901DF91CF9173
:10A870001F910F91FF90EF90DF90CF900895EF928E
:10A88000FF920F931F937B019A010027F7FC00951D
:10A89000102FB801A7010E94FF531F910F91FF9045
:10A8A000EF9008950E946753089581E08093440CCF
:10A8B0006093210C1092420C1092430C0895209149
:10A8C000200C30E080911F0C281B3109C90108952C
:10A8D00040911F0C8091200C481718F02FEF3FEF8C
:10A8E0000AC0E42FF0E0E150F44F8081282F30E0DF
:10A8F0004F5F40931F0CC9010895E0911F0C809198
:10A90000200CE81718F0EFEFFFEF06C0F0E0E15081
:10A91000F44F8081E82FF0E0CF0108950895109260
:10A92000480C1092470C88EE93E0A0E0B0E08093D2
:10A93000490C90934A0CA0934B0CB0934C0C87E6B7
:10A9400093E09093460C8093450C0895CF92DF924C
:10A95000EF92FF920F931F93CF93DF937C016B01D4
:10A960008A018091440C8823A1F0C0E0D0E00DC0A2
:10A97000D701ED91FC91D601AC0FBD1F0190F08184
:10A98000E02DC7016C9109952196C017D10780F37E
:10A9900004C0CB01642F0E94A06BC801DF91CF914E
:10A9A0001F910F91FF90EF90DF90CF900895DF936C
:10A9B000CF930F92CDB7DEB7FC0169838091440C31
:10A9C0008823C9F08091430C803238F081E090E018
:10A9D0009383828320E030E015C08091420CE82F01
:10A9E000F0E0EE5DF34F998190838F5F8093420C8E
:10A9F0008093430C05C0CE01019661E00E94A06BDC
:10AA000021E030E0C9010F90CF91DF9108950F93BD
:10AA1000062F8091210C62E27CE04091430C21E002
:10AA20000E944B6B1092420C1092430C1092440CFB
:10AA30000F91089561E00E9407550895413208F092
:10AA400040E2862F6FEF7BE00E94026B10921F0C9A
:10AA50008093200C089521E00E941E5508951092C5
:10AA60001F0C1092200C1092420C1092430C0E946A
:10AA70004C6D08950F931F93CF93DF93DC01EB018F
:10AA80008A0180E090E020E2FE01E80FF91F2083B8
:10AA900001968B309105C1F757E040E024C0622F4A
:10AAA0002E3219F080E39CE007C05A3051F15AE091
:10AAB00048E018C0321729F1FC0101963491332384
:10AAC000C9F75417F0F02132E0F02F37D0F4822F7D
:10AAD00081568A3110F4622F6052FE01E40FF11D9D
:10AAE00060834F5F11962C91222311F02F32B9F61B
:10AAF000F801B183A08390E08881803219F091E061
:10AB000001C090E0892FDF91CF911F910F9108959F
:10AB1000CF92DF92EF92FF920F931F93DF93CF9329
:10AB200000D000D0CDB7DEB77C01FC0186899789C3
:10AB3000A08DB18D89839A83AB83BC8300E010E044
:10AB40006E010894C11CD11C49815A816B817C81A2
:10AB5000D70114968D919C91159796010E94876557
:10AB6000882379F1D7011496ED91FC911597848192
:10AB7000080F111DB0E100301B0718F529813A813B
:10AB80004B815C818389803131F4285F3F4F4040A5
:10AB90005040D0F205C0285F3F4F4F4F5F40A0F2BA
:10ABA000C801A0E0B0E029E0880F991FAA1FBB1FD1
:10ABB0002A95D1F7F701828B938BA48BB58B81E01B
:10ABC00001C080E00F900F900F900F90CF91DF9118
:10ABD0001F910F91FF90EF90DF90CF900895CF934A
:10ABE000DF93EC01FB018A818823D1F57D836C839F
:10ABF00083898031C9F582E08A831E8A1F8A188E74
:10AC0000198E84899589A0E0B0E035E0880F991FFE
:10AC1000AA1FBB1F3A95D1F78A8B9B8BAC8BBD8B40
:10AC20000FC083E08A8386899789A08DB18D8E8B32
:10AC30009F8BA88FB98FCE010E948855882381F001
:10AC400081E089831E821F82188619861A861B86D8
:10AC50001C861D861E861F86188A198A1B8201C0C3
:10AC600080E0DF91CF9108958032D1F7DACF6F92F3
:10AC70007F928F929F92AF92BF92CF92DF92EF928C
:10AC8000FF920F931F93CF93DF93EC017A018B0117
:10AC90002A81222309F480C08A899B89AC89BD89D5
:10ACA00084179507A607B70708F476C085C0E11496
:10ACB000F1040105110551F41E821F8218861986C0
:10ACC0001A861B861C861D8681E067C02A853B8507
:10ACD0004C855D85EC81FD81828590E0099621504F
:10ACE00030404040504039014A01082E04C096943B
:10ACF0008794779467940A94D2F72F5F3F4F4F4F12
:10AD00005F4F0894E108F108010911095701680132
:10AD100004C0D694C794B794A7948A95D2F70894A0
:10AD2000E11CF11C011D111DA614B704C804D904AF
:10AD300028F0211531054105510549F48E899F8977
:10AD4000A88DB98D8E839F83A887B98716C0A61852
:10AD5000B708C808D90811C04E815F816885798518
:10AD60008C819D8194010E9487650894A108B10897
:10AD7000C108D108882331F40FC046E0842E912CFD
:10AD80008C0E9D1EA114B104C104D10429F7EA86DA
:10AD9000FB860C871D8798CF80E0DF91CF911F91B4
:10ADA0000F91FF90EF90DF90CF90BF90AF909F906A
:10ADB0008F907F906F900895223009F078CFE7CF81
:10ADC000CF93DF93EC01462F6E857F858889998923
:10ADD0000E949A63AC01009719F420E030E00AC0A9
:10ADE0008B81282F30E065E0220F331F6A95E1F751
:10ADF000240F351FC901DF91CF9108950F931F9341
:10AE0000CF93DF938C01FC0182818823F1F1818152
:10AE100087FF38C0C80161E00E94E056EC0100974E
:10AE2000A1F18881853E89F1F8018281823040F468
:10AE300082899389A489B5898C8F9D8FAE8FBF8FAE
:10AE4000F801868997899B8F8A8F86899789A08D3B
:10AE5000B18DCD01AA27BB279D8B8C8BE091530C24
:10AE6000F091540C309751F0BE016A5E7F4FCE01D5
:10AE700048960995888D998D9B8B8A8BF8018181E5
:10AE80008F7781830E94526304C081E0F801808340
:10AE900080E0DF91CF911F910F9108956F927F9283
:10AEA0008F929F92AF92BF92CF92DF92EF92FF92DA
:10AEB0000F931F93DF93CF9300D000D0CDB7DEB7B1
:10AEC0007C015A016B01DC0112968C911297813042
:10AED00009F091C011968C9181FF8DC0A0C00097A0
:10AEE000A105B10511F481E087C0F7016284738484
:10AEF00084849584C701B601A5010E943756882332
:10AF000009F479C0D70114968D919C911597A114DD
:10AF1000B104C104D10489F456964D915D916D91AF
:10AF20007C9159970E94F665882309F464C0F70163
:10AF3000168A178A108E118E44C0D70116964D912D
:10AF40005D916D917C9119979E012F5F3F4F0E94FB
:10AF50008765882309F44FC0D7011496ED91FC91C1
:10AF6000159749815A816B817C818389803149F4AD
:10AF7000483FBFEF5B07B0E06B07B0E07B0748F0EE
:10AF800020C0483F8FEF58078FEF68078FE07807A2
:10AF9000C0F4CF010E94F665882369F1D7011696A7
:10AFA0004D915D916D917C91199714968D919C9125
:10AFB00015970FEF1FEF2FEF3FE00E9417658823D3
:10AFC000D1F0F701A28AB38AC48AD58A81818068C8
:10AFD0008183C7010E94FE56882369F0B601A5014E
:10AFE0006A147B048C049D0410F4B401A301C7010E
:10AFF0000E94375601C080E00F900F900F900F9085
:10B00000CF91DF911F910F91FF90EF90DF90CF9044
:10B01000BF90AF909F908F907F906F900895F701B1
:10B0200082899389A489B58984179507A607B707EC
:10B0300008F055CFE0CF1F93CF93DF93EC01142F8F
:10B04000262F30E0F90185E0EE0FFF1F8A95E1F72A
:10B05000E65AF34F8385817121F0842F827109F0C4
:10B0600064C080915A0E90915B0EA0915C0EB091DD
:10B070005D0E8E879F87A88BB98B6B83F901B5E036
:10B08000EE0FFF1FBA95E1F7E65AF34F2489358991
:10B0900040E050E0A901332722272E8B3F8B488FB9
:10B0A000598F828D938DA0E0B0E0282B392B4A2B4D
:10B0B0005B2B2E8B3F8B488F598F838590E0887157
:10B0C0009070009751F4848D958DA68DB78D8A8BE5
:10B0D0009B8BAC8BBD8B81E008C0409731F5CE01D6
:10B0E0000E948855882309F184E08A83812F8F701C
:10B0F00089831E821F82188619861A861B861C86E3
:10B100001D8614FF18C0CE0140E050E060E070E002
:10B110000E944E57882379F408C04A895B896C895C
:10B120007D89CE010E94375602C01A8280E0DF91ED
:10B13000CF911F91089515FDF0CF81E0F8CF0F93C7
:10B140001F938C010E94FE56F80112821F910F91ED
:10B150000895CF93DF93EC0140E050E060E070E0B1
:10B160000E944E57882369F0CE0161E00E94E056AC
:10B17000FC01009731F085EE80831A820E945263B1
:10B1800001C080E0DF91CF9108953F924F925F928E
:10B190006F927F928F929F92AF92BF92CF92DF92E7
:10B1A000EF92FF920F931F93DF93CF93CDB7DEB74C
:10B1B00028970FB6F894DEBF0FBECDBF98878F8358
:10B1C0005E834D83DC0112968C911297882309F4DB
:10B1D0001DC111968C9180FF19C133C1F501EE1983
:10B1E000FF09FE83ED837A8369838F8198850696B4
:10B1F0009C838B836D807E8002C1AF81B8851A9657
:10B200002D913D914D915C911D978FEF482E81E0DE
:10B21000582E422253221496ED91FC911597590114
:10B220006A0109E0D694C794B794A7940A95D1F718
:10B2300035803A2012968C91823049F4E688F7885E
:10B24000008D118DEA0CFB1C0C1D1D1D35C0411419
:10B25000510411F5332001F5211531054105510542
:10B2600059F4EF81F88586899789A08DB18D868301
:10B270009783A087B18710C0AF81B88516964D918E
:10B280005D916D917C911997CF012B813C810E943A
:10B290008765882309F4BAC0EF81F8854681578114
:10B2A00060857185848195810E9438637B018C0162
:10B2B000E30CF11C011D111D4114510499F4F0E03F
:10B2C0006F16F2E07F0670F020915A0E30915B0EFF
:10B2D00040915C0E50915D0EE216F30604071507CF
:10B2E00009F0CFC0C801B70140E00E949A630097FF
:10B2F00009F48CC040E052E0441955094301461559
:10B30000570508F44A019C01240D351D89819A8155
:10B31000B901A4010E94C00659C080915F0E9091AE
:10B32000600EB801A70129813A810E94DB69882358
:10B3300009F46CC0812C12E0912E48C0D72CD69411
:10B34000AF81B88512968C911297823049F014968D
:10B35000ED91FC911597848183198D1508F4D82EF1
:10B36000E216F3060407150770F02D0D311D411D7F
:10B37000511DE216F3060407150728F40E945263D4
:10B38000882309F443C080915F0E9091600EB8014C
:10B39000A7010E943F698823C9F109811A81FF240E
:10B3A00008C0B8010E94C86900501E4F882371F17F
:10B3B000F39480915F0E9091600EFD1490F30E94C3
:10B3C0002569882319F19D2C990C8824E981FA813B
:10B3D000E80DF91DFA83E983940140E050E0EF8124
:10B3E000F88582859385A485B585820F931FA41F58
:10B3F000B51F82879387A487B58768187908611479
:10B40000710409F0FACE4D815E8102C04FEF5FEF0B
:10B41000CA0128960FB6F894DEBF0FBECDBFCF91FC
:10B42000DF911F910F91FF90EF90DF90CF90BF9031
:10B43000AF909F908F907F906F905F904F903F90D4
:10B440000895AF81B8855296AD90BD90CD90DC90B7
:10B4500055971A96ED90FD900D911C911D97ED81D9
:10B46000FE819F0140E050E0D601C5018E199F0981
:10B47000A00BB10B281739074A075B0708F0AECEBF
:10B48000B2CEF0E06F16F4E07F0608F057CF45CF5C
:10B49000DF93CF930F92CDB7DEB7BE016F5F7F4FC3
:10B4A00041E050E00E94C558019719F02FEF3FEF9F
:10B4B00003C08981282F30E0C9010F90CF91DF911F
:10B4C0000895EF92FF920F931F93CF93DF93EC01B8
:10B4D0008A81823038F1EA84FB840C851D85CE0197
:10B4E0000E94485A97FD1EC08A859B85AC85BD8504
:10B4F0004F96A11DB11D8A879B87AC87BD8725E02C
:10B5000016950795F794E7942A95D1F72E2D30E0FC
:10B510002F70307095E0220F331F9A95E1F7265A6D
:10B52000334F02C020E030E0C901DF91CF911F917D
:10B530000F91FF90EF900895CF93DF93EC018A81F4
:10B54000843071F5CE0140E050E060E070E00E9490
:10B55000375610C0CE010E94615AFC01009701F1DC
:10B5600080818823A1F0853E29F08E3219F08385F1
:10B5700083FF16C02A853B854C855D858A899B891A
:10B58000AC89BD89281739074A075B0718F381E0A2
:10B590008A83898182608983CE010E94A95801C073
:10B5A00080E0DF91CF910895DF92EF92FF920F93A9
:10B5B0001F93CF93DF938C01EB017A01D22E8C8104
:10B5C0009D81F801958384838281882329F5611503
:10B5D000710559F521C0A70165E0440F551F6A9513
:10B5E000E1F760E070E0CE010E9437568823A1F0B9
:10B5F000CE010E94615AFC01009771F0808188237E
:10B6000059F0853E49F08E3239F06E2D6F70C801C9
:10B610004D2D0E941B5801C080E0DF91CF911F91FA
:10B620000F91FF90EF90DF90089527FFD4CFF4CFD4
:10B63000AF92BF92CF92DF92EF92FF920F931F9340
:10B64000DF93CF93CDB7DEB76A970FB6F894DEBF1E
:10B650000FBECDBF8C0119821B8240E050E060E03C
:10B6600070E00E9437565E010894A11CB11C52C0C4
:10B67000C8010E94615AFC01009709F466C08081EC
:10B68000882309F456C0853E09F444C08E3209F47B
:10B6900041C0838583FD3EC0A7019601F5E0569524
:10B6A000479537952795FA95D1F77901C501B801E6
:10B6B000A90121E00E94D45A882309F446C08B8155
:10B6C000843021F4C5010E94185B06C08A81826023
:10B6D0008A83C5010E94A9588823B9F10894E11C06
:10B6E000F11CA70160E070E0E5E0440F551F661F04
:10B6F000771FEA95D1F7F80182859385A485B585F2
:10B7000084179507A607B70729F0C8010E94375686
:10B710008823D9F0F801C284D384E484F584828933
:10B720009389A489B589C816D906EA06FB0608F4E8
:10B730009FCFF80182818250823028F0C8010E9498
:10B740009C5A882319F081E001C080E06A960FB608
:10B75000F894DEBF0FBECDBFCF91DF911F910F9147
:10B76000FF90EF90DF90CF90BF90AF9008952F9211
:10B770003F924F925F926F927F928F929F92AF9281
:10B78000BF92CF92DF92EF92FF920F931F93DF93BE
:10B79000CF930F92CDB7DEB72C015B013A0149017F
:10B7A00000E010E0EE24EA94FE2C1E010894211C17
:10B7B000311C13C00A0D1B1DF80160838114910414
:10B7C00019F46A3049F41EC0772767FD7095C401EB
:10B7D0000E94DB060097B1F4860168010894C11C41
:10B7E000D11CC614D70444F5C201B10141E050E0B8
:10B7F0000E94C5587C0181309105F1F469816D305A
:10B80000C9F6EBCF8601A00EB11EF5011082C8016A
:10B810000F90CF91DF911F910F91FF90EF90DF90EC
:10B82000CF90BF90AF909F908F907F906F905F90E0
:10B830004F903F902F900895F7FEE5CF0FEF1FEF49
:10B84000E6CFCF93DF93EC019C012A5F3F4F8C81C1
:10B850009D8141E050E060E070E00E945D668823D9
:10B86000A1F08E899F89A88DB98D0097A105B1059A
:10B8700059F48E819F81A885B9858E8B9F8BA88F67
:10B88000B98F89818068898381E0DF91CF910895A4
:10B890002F923F924F925F926F927F928F929F92E0
:10B8A000AF92BF92CF92DF92EF92FF920F931F93CE
:10B8B000DF93CF93CDB7DEB729970FB6F894DEBFED
:10B8C0000FBECDBF4C01162F072F59874887DC01CB
:10B8D00012968C911297813009F0BDC111968C910E
:10B8E00081FFB9C1D7C1F40142895389648975893F
:10B8F00082859385A485B58584179507A607B70724
:10B9000031F0C4010E943756882309F4A4C1888508
:10B9100099859C0140E050E0F40182859385A485DF
:10B92000B58580959095A095B09582179307A4074B
:10B93000B50708F490C1812F902F9C013F832E837F
:10B94000288439844CC1D4011496ED91FC9115974B
:10B95000DA01C90119E0B695A795979587951A95CB
:10B96000D1F715811823AFEFEA2EA1E0FA2EE222DB
:10B97000F322112309F052C0E114F10409F04EC082
:10B98000D40116964D915D916D917C911997411559
:10B9900051056105710571F1CF019E012F5F3F4F88
:10B9A0000E948765882309F456C129813A814B8119
:10B9B0005C81D4011496ED91FC91159783898031B7
:10B9C00049F4283FBFEF3B07B0E04B07B0E05B070F
:10B9D00048F019C0283FEFEF3E07EFEF4E07EFE0CA
:10B9E0005E0788F4D40116962D933D934D935C9396
:10B9F000199714C0F40186899789A08DB18D00979D
:10BA0000A105B10531F4C4010E94215C882331F401
:10BA100022C1F40186839783A087B187D40116964B
:10BA20004D915D916D917C91199714968D919C919A
:10BA300015970E9438635B016C01A10EB11CC11CFB
:10BA4000D11CE114F104A9F4B0E02B16B2E03B06DE
:10BA5000A0F5F40122853385448555858289938933
:10BA6000A489B589281739074A075B0710F045E014
:10BA700001C041E0C601B5010E949A63009709F434
:10BA8000EAC000E012E00E191F092101021513059A
:10BA900008F428019C012E0D3F1DC9016E817F8194
:10BAA000A2010E94C0064016510609F080C00E9403
:10BAB0009763882309F07BC0CEC0F0E02F16F4E036
:10BAC0003F0600F580915A0E90915B0EA0915C0E9E
:10BAD000B0915D0E8A159B05AC05BD0511F40E9461
:10BAE000296380915F0E9091600EB601A5012E81B1
:10BAF0003F810E94EB68882309F4ADC0412CF2E03D
:10BB00005F2E55C0D4011496ED91FC911597848158
:10BB1000811BB32DB695BD838B1708F48D83ED8102
:10BB20000E2F10E020E030E080915F0E9091600ECB
:10BB3000B601A5010E943E68882309F48CC06E807E
:10BB40007F808601750122C080915A0E90915B0E14
:10BB5000A0915C0EB0915D0EE816F9060A071B076E
:10BB600011F40E94296380915F0E9091600EB301E1
:10BB70000E94C56820E032E0620E731E0894E11C4A
:10BB8000F11C011D111D882309F465C08E2D8A1931
:10BB90003D818317C8F280915F0E9091600E0E94E4
:10BBA0001868882309F457C05D80550C442492011D
:10BBB00040E050E0F40182859385A485B585820F2D
:10BBC000931FA41FB51F82879387A487B5872E81F3
:10BBD0003F81240D351D3F832E8324183508D40161
:10BBE0001A962D913D914D915C911D972114310430
:10BBF00009F0A9CE52968D919D910D90BC91A02DEA
:10BC000082179307A407B50748F4F401228B338BFE
:10BC1000448B558B81818068818311C08091530C46
:10BC20009091540C892B59F028853985232B39F0B4
:10BC3000D40111968C911197806811968C93F40120
:10BC4000818183FF05C0C4010E94FE56882319F03C
:10BC50004885598505C081E0D4018C934FEF5FEF93
:10BC6000CA0129960FB6F894DEBF0FBECDBFCF91A3
:10BC7000DF911F910F91FF90EF90DF90CF90BF90D9
:10BC8000AF909F908F907F906F905F904F903F907C
:10BC90002F90089582FD27CE3ACE9F92AF92BF9209
:10BCA000CF92DF92EF92FF920F931F93CF93DF9388
:10BCB0008C01FC0182899389A489B589805E9F4F9C
:10BCC000AF41B04008F05CC0C8010E94215C8823ED
:10BCD00009F456C0D80116964D915D916D917C91F5
:10BCE000199714968D919C9115970E9438635B016A
:10BCF0006C0145E00E949A63EC01009709F442C090
:10BD000080E092E0FE019C01119221503040E1F769
:10BD10009C2EED2EFF24F39411C0B601A5014F0D0A
:10BD2000511D611D711D80915F0E9091600E292D36
:10BD30003E2D0E94EB68882319F1F394D8011496E4
:10BD4000ED91FC9115972481F21638F330E040E034
:10BD500050E089E0220F331F441F551F8A95D1F709
:10BD600052968D919D910D90BC91A02D820F931FA5
:10BD7000A41FB51FF801828B938BA48BB58B02C0D7
:10BD8000C0E0D0E0CE01DF91CF911F910F91FF90E5
:10BD9000EF90DF90CF90BF90AF909F9008953F922B
:10BDA0004F925F926F927F928F929F92AF92BF92CB
:10BDB000CF92DF92EF92FF920F931F93CF93DF9377
:10BDC0004C01EB01442E352E522E8C819D81F401C5
:10BDD00095838483CB0140E050E060E070E00E94F6
:10BDE000375677244FC0CE010E94485A97FDABC00A
:10BDF0008A859B85AC85BD8581509E4FAF4FBF4FD7
:10BE00008A879B87AC87BD87A0905A0EB0905B0E47
:10BE1000C0905C0ED0905D0E2AE5E22E2CE0F22E52
:10BE200000E010E0602EF7018081882311F0853E4C
:10BE300079F4772041F4F401A686B786C08AD18AC6
:10BE4000638277247394F7018081882391F428C05A
:10BE5000B80195E0660F771F9A95E1F7665A734F20
:10BE6000842D932D4BE050E00E94B306009709F417
:10BE70007DC00F5F1F4F80E290E0E80EF91E003199
:10BE8000110581F62A853B854C855D858A899B89CC
:10BE9000AC89BD89281739074A075B0708F4A3CF87
:10BEA00056FE51C051FE4FC0772051F0F40163801F
:10BEB000C40161E00E94E056EC01009761F443C0C8
:10BEC0008A81823009F43FC0CE010E944D5E009706
:10BED000D1F1EC01662480E2FE0111928A95E9F726
:10BEE000DE01242D332DC901FC018BE001900D9260
:10BEF0008150E1F7E091530CF091540C309739F0F8
:10BF0000BE01625F7F4FCE014096099508C081E275
:10BF100098E2998B888B80E098E09F878E8788894C
:10BF200099899B8B8A8B998F888F8E859F859F8B14
:10BF30008E8B0E945263882331F0C401662D452DFB
:10BF40000E941B5801C080E0DF91CF911F910F919B
:10BF5000FF90EF90DF90CF90BF90AF909F908F9029
:10BF60007F906F905F904F903F90089557FEE5CF80
:10BF7000EACF2F923F924F925F926F927F928F9271
:10BF80009F92AF92BF92CF92DF92EF92FF920F9368
:10BF90001F93DF93CF93CDB7DEB7C454D0400FB615
:10BFA000F894DEBF0FBECDBF4C016B01DE01A05C7B
:10BFB000BF4F11965C934E9323962FAF2397611535
:10BFC000710509F48AC01E8618A6FC0182818823A7
:10BFD00009F083C01C861EA2FA0180818F32F1F025
:10BFE00086015CE0E52EF12CEC0EFD1E40E4A42E53
:10BFF000B12CAC0EBD1E3E010894611C711C25962F
:10C00000FFAEEEAE259736E2232E312C2C0E3D1ED0
:10C0100027012BC01196B183A08301C0FD01A0812F
:10C02000B1818C918F32B1F3882349F4D6011496F3
:10C030006D917C911597C4010E94EF554FC0F60198
:10C0400082818250823060F28E010A5D1F4F6481CE
:10C050007581C8010E94EF55882319F63EC0342D22
:10C06000252D8701832F922F7C01D5018D919C91E5
:10C07000B301A5010E943A55882329F42EC03196B8
:10C08000D501ED93FC93D501ED91FC9180818F3228
:10C09000B1F38823C9F0C701B801A30121E00E94D0
:10C0A000CF5E8823D1F00C151D0519F0C8010E9440
:10C0B0009F582596EEADFFAD2597EE16FF0679F653
:10C0C000C101322D292FCDCFC401B801A301239680
:10C0D0002FAD23970E94CF5E01C080E0CC5BDF4F85
:10C0E0000FB6F894DEBF0FBECDBFCF91DF911F9189
:10C0F0000F91FF90EF90DF90CF90BF90AF909F9007
:10C100008F907F906F905F904F903F902F90089509
:10C110000F931F93DF93CF93CDB7DEB76A970FB618
:10C12000F894DEBF0FBECDBF9C01AB0119821B820C
:10C130008E010F5F1F4FC801B90122E00E94B95F55
:10C14000882319F0C8010E94A9586A960FB6F8947E
:10C15000DEBF0FBECDBFCF91DF911F910F9108952C
:10C16000FB01242F6091510C7091520CAF010E9481
:10C17000B95F0895FC01128210820E94B060089598
:10C18000DF93CF93CDB7DEB76A970FB6F894DEBFD3
:10C190000FBECDBF9C01AB0119821B82CE0101965F
:10C1A000B90121E00E94B95F6A960FB6F894DEBF2C
:10C1B0000FBECDBFCF91DF910895EF92FF920F9305
:10C1C0001F93DF93CF93CDB7DEB7A0970FB6F89448
:10C1D000DEBF0FBECDBF8C017B01FB0182818230AF
:10C1E00008F46FC0C80123EC0E94CF5E882309F4D5
:10C1F00068C081E0F801818384E08283C8010E94E5
:10C200004D5E892B09F45DC0C8010E94FE5688234B
:10C2100009F457C0C80161E00E94E056FC01009794
:10C2200009F44FC080E18387DE01119680E201901E
:10C230000D928150E1F78EE28983FE01329620E271
:10C24000CE010C962193E817F907E1F7F80146892A
:10C250005789608D718D848195810E94386341E09A
:10C260000E949A639C01009761F1DC01FE01319606
:10C2700080E201900D928150E1F78EE28A83F7010E
:10C2800082818250823028F41C8E1B8E1E8A1D8A69
:10C290000CC0F70186899789A08DB18D9C8F8B8FFB
:10C2A000CD01AA27BB279E8B8D8BD9019096FE01CD
:10C2B000319680E201900D928150E1F70E94526325
:10C2C00001C080E0A0960FB6F894DEBF0FBECDBFD0
:10C2D000CF91DF911F910F91FF90EF9008952F92D2
:10C2E0003F924F925F926F927F928F929F92AF9206
:10C2F000BF92CF92DF92EF92FF920F931F93DF9343
:10C30000CF93CDB7DEB7C454D0400FB6F894DEBF9C
:10C310000FBECDBF3C016B01DE01A05CBF4F11968B
:10C320005C934E9323962FAF23976115710509F403
:10C3300087C01E8618A6FC018281882309F080C070
:10C340009AC08601FCE0EF2EF12CEC0EFD1EE0E41D
:10C35000AE2EB12CAC0EBD1E4E010894811C911C5A
:10C360002596FFAEEEAE259776E2272E312C2C0EC9
:10C370003D1E270124C01196B183A08301C0FD0199
:10C38000A081B1818C918F32B1F3D60112968C913C
:10C39000129782508230A8F28E010A5D1F4F1496C8
:10C3A0006D917C911597C8010E94EF55882351F635
:10C3B00047C0342D252D8701832F922F7C01F50155
:10C3C00080819181B401A5010E943A55882329F406
:10C3D00037C03196D501ED93FC93D501ED91FC91D9
:10C3E00080818F32B1F3882329F1C701B801A401FC
:10C3F00021E00E94CF5E882361F42396BFAD23978E
:10C40000BB23F1F0C701B801A4010E94DD608823BD
:10C41000B9F00C151D0519F0C8010E949F5825960A
:10C42000EEADFFAD2597EE16FF0619F6C101322DD0
:10C43000292FC1CFC301B801A4010E94DD6001C052
:10C4400080E0CC5BDF4F0FB6F894DEBF0FBECDBFF0
:10C45000CF91DF911F910F91FF90EF90DF90CF90E0
:10C46000BF90AF909F908F907F906F905F904F9014
:10C470003F902F9008951C861EA2ED91FC9111977C
:10C4800080818F3209F05DCF7ACF4F960E9488600D
:10C490000895DF93CF93CDB7DEB76A970FB6F894C0
:10C4A000DEBF0FBECDBFFB01242F19821B82BC0152
:10C4B000615E7F4FCE010196AF010E946F616A9667
:10C4C0000FB6F894DEBF0FBECDBFCF91DF910895B8
:10C4D0004F960E94C0600895DF92EF92FF920F93F3
:10C4E0001F93DF93CF93CDB7DEB76A970FB6F8945B
:10C4F000DEBF0FBECDBF9B01D42E19821B828C01E3
:10C50000015E1F4F7E010894E11CF11CC701B801B8
:10C51000A90121E00E94B95F8B81823010F480E094
:10C520000EC0D801F7018AE101900D928150E1F728
:10C53000DD2021F01093520C0093510C81E06A969B
:10C540000FB6F894DEBF0FBECDBFCF91DF911F9124
:10C550000F91FF90EF90DF900895CF93DF93EC0160
:10C56000662331F06F96D093520CC093510C6F97A5
:10C5700089A1882321F0CE014F960E949F58CE01B9
:10C580004F962596BE010E94EF55DF91CF910895F9
:10C590000F931F93CF93DF93EC010E940F6A8823C0
:10C5A000C9F08E010B5F1F4FC801BE0141E00E9420
:10C5B000DE63882339F4C801BE0140E00E94DE63D7
:10C5C000882341F0CE0161E00E94AD62882319F01A
:10C5D00081E001C080E0DF91CF911F910F9108951C
:10C5E00004960E94485C0895DF93CF930F92CDB7D5
:10C5F000DEB769830496BE016F5F7F4F41E050E074
:10C600000E94485C20E030E0019711F421E030E026
:10C61000C9010F90CF91DF910895DB010D900020AB
:10C62000E9F71197A61BB70B0496AD010E94485C71
:10C6300008950F931F938C0104960E94BA60F8012D
:10C640001382128287E793E0918380831F910F9179
:10C6500008958FEF9FEFAFEFBFEF80935A0E909347
:10C660005B0EA0935C0EB0935D0E10925E0E08956B
:10C67000FC019A01AB0122503040404050400284FE
:10C6800004C0220F331F441F551F0A94D2F783851D
:10C690009485A585B685280F391F4A1F5B1FB901F0
:10C6A000CA01089580915E0E80FF3DC040915A0EF0
:10C6B00050915B0E60915C0E70915D0E80915F0EEB
:10C6C0009091600E2AE53CE00E94EB68882369F1B6
:10C6D00080915E0E81FF22C08091550C8230F0F077
:10C6E0004091560C5091570C6091580C7091590C18
:10C6F00080915A0E90915B0EA0915C0EB0915D0EF0
:10C70000480F591F6A1F7B1F80915F0E9091600E2A
:10C710002AE53CE00E94EB68882339F080915E0EA8
:10C720008E7F80935E0E81E0089580E008950E94E0
:10C7300052630895DF92EF92FF920F931F937B0154
:10C740008C01D42E80915A0E90915B0EA0915C0EBC
:10C75000B0915D0E8E159F05A007B107E1F00E9414
:10C760005263882311F1D2FC0CC080915F0E90912E
:10C77000600EB801A7012AE53CE00E94DB6988232E
:10C78000A1F010925E0EE0925A0EF0925B0E0093B2
:10C790005C0E10935D0E83E0D82280915E0E8D2991
:10C7A00080935E0E2AE53CE002C020E030E0C90143
:10C7B0001F910F91FF90EF90DF9008956F927F92FD
:10C7C0008F929F92AF92BF92CF92DF92EF92FF92A1
:10C7D0000F931F93CF93DF93EC01142F7093600E90
:10C7E00060935F0E1B8A82E090E0A0E0B0E0888357
:10C7F0009983AA83BB8310925E0E8FEF9FEFAFEFFA
:10C80000BFEF80935A0E90935B0EA0935C0EB09393
:10C810005D0E442321F466247724430136C045305D
:10C8200008F0F1C060E070E080E090E040E00E943D
:10C830009A63DC01009709F4E6C0412F50E04150B3
:10C840005040FA0174E0EE0FFF1F7A95E1F7E80F10
:10C85000F91FE254FE4F808190E08F779070892B12
:10C8600009F0D1C064E0440F551F6A95E1F7A40FA9
:10C87000B51FAA53BE4F6D907D908D909C90611412
:10C8800071048104910409F4BEC0C401B30140E005
:10C890000E949A635C01009709F4B5C0FC0183858E
:10C8A00094858050924009F0AEC0F5012089222382
:10C8B00009F4A9C0468557854115510509F4A3C05F
:10C8C0002093550C85858C8381508D831A8691E049
:10C8D00060E070E00AC0990F6F5F7F4F68307105AC
:10C8E00009F491C08A858F5F8A878C81891799F7AF
:10C8F000F501668977896115710519F080E090E08E
:10C9000005C0F50164A175A186A197A16093560C9D
:10C910007093570C8093580C9093590C6A01EE2435
:10C92000FF24C60CD71CE81CF91CCF86D88AE98ADC
:10C93000FA8AF501018912891D8B0C8B30E040E0E9
:10C9400050E00E946A6D6C0D7D1D8E1D9F1D6E8BCB
:10C950007F8B888F998F35E0000F111F3A95E1F793
:10C9600001501E4F012F11270695980140E050E01D
:10C97000260F371F481F591F2B873C874D875E871F
:10C98000F50183899489009721F07C0100E010E093
:10C9900005C0F501E0A0F1A002A113A1C401B301FB
:10C9A000621B730B840B950B6E0D7F1D801F911FF7
:10C9B0000A8404C096958795779567950A94D2F76F
:10C9C0006E837F8388879987653FFFE07F07F0E06C
:10C9D0008F07F0E09F0718F48CE08B8B14C0655F25
:10C9E0007F4F8040904010F480E10AC0F50184A59B
:10C9F00095A5A6A5B7A58E8B9F8BA88FB98F80E232
:10CA00008B8B81E001C080E0DF91CF911F910F916E
:10CA1000FF90EF90DF90CF90BF90AF909F908F905E
:10CA20007F906F90089542600E949A6308958F925C
:10CA30009F92AF92BF92CF92DF92EF92FF920F93AD
:10CA40001F93CF93DF93EC016A017B0148015901E9
:10CA5000423051056105710508F44BC08E819F81FC
:10CA6000A885B9850196A11DB11D84179507A60754
:10CA7000B70708F43EC08B89803129F4252F362F63
:10CA8000472F55270BC08032A1F59A01AB0117E063
:10CA900056954795379527951A95D1F78F8598899B
:10CAA000A989BA89280F391F4A1F5B1FCA01B9011A
:10CAB00041E00E9413659C010097D9F08B89803179
:10CAC00049F4F601F070EE0FFF1FE20FF31F9182A1
:10CAD00080820DC0F601EF77F070EE0FFF1FEE0FB2
:10CAE000FF1FE20FF31F80829182A282B38281E056
:10CAF00001C080E0DF91CF911F910F91FF90EF90E7
:10CB0000DF90CF90BF90AF909F908F900895CF927D
:10CB1000DF92EF92FF920F931F93CF93DF93EC017D
:10CB20007A018B016901423051056105710508F4F4
:10CB300053C08E819F81A885B9850196A11DB11D25
:10CB400084179507A607B70708F446C08B8980317C
:10CB500029F45527412F302F2F2D0BC08032E1F5BE
:10CB60009A01AB0167E056954795379527956A95E9
:10CB7000D1F78F859889A989BA89280F391F4A1F4B
:10CB80005B1FCA01B90140E00E9413659C01009738
:10CB900019F18B89803159F4F701F070EE0FFF1F06
:10CBA000E20FF31F80819181A0E0B0E00EC0F70199
:10CBB000EF77F070EE0FFF1FEE0FFF1FE20FF31F76
:10CBC00080819181A281B381BF70F60180839183BE
:10CBD000A283B38381E001C080E0DF91CF911F91F8
:10CBE0000F91FF90EF90DF90CF9008958F929F92DA
:10CBF000AF92BF92CF92DF92EF92FF920F931F936B
:10CC0000DF93CF9300D000D0CDB7DEB75C016A01CF
:10CC10007B014E010894811C911CC501B701A6013E
:10CC200094010E9487658823B1F1C501B701A6016F
:10CC300000E010E020E030E00E941765882359F101
:10CC4000F50180819181A281B381C816D906EA06D7
:10CC5000FB0620F4C082D182E282F382C980DA80AE
:10CC6000EB80FC80F5018389803151F4F8EFCF1619
:10CC7000FFEFDF06F0E0EF06F0E0FF0670F209C01C
:10CC800088EFC8168FEFD8068FEFE8068FE0F8061A
:10CC900020F281E001C080E00F900F900F900F9084
:10CCA000CF91DF911F910F91FF90EF90DF90CF9088
:10CCB000BF90AF909F908F9008952F923F924F9288
:10CCC0005F926F927F928F929F92AF92BF92CF921C
:10CCD000DF92EF92FF920F931F93DF93CF93CDB725
:10CCE000DEB766970FB6F894DEBF0FBECDBF1C014E
:10CCF00049875A876B877C873E872D87DC0116968C
:10CD00002D913D914D915C9119972F5F3F4F4F4F62
:10CD10005F4F2D833E834F835887ED85FE850081CD
:10CD2000118122813381011511052105310549F059
:10CD3000480159010894811C911CA11CB11C10E0F0
:10CD400006C0DC018D909D90AD90BC9011E0750106
:10CD50006401442455243201F10186819781A08524
:10CD6000B185481659066A067B0608F09DC02D81DC
:10CD70003E814F8158852C153D054E055F0550F4C9
:10CD8000F2E08F2E912CA12CB12CE2E0CE2ED12CF2
:10CD9000E12CF12CC101B701A6019E012F5F3F4F8D
:10CDA0000E948765882309F47FC089819A81AB81BD
:10CDB000BC810097A105B10571F08C149D04AE04EF
:10CDC000BF0409F010E0460157010894811C911C32
:10CDD000A11CB11C16C0D701C6010196A11DB11D31
:10CDE0008B8B9C8BAD8BBE8B88199909AA09BB09CB
:10CDF00029853A854B855C8582179307A407B5077B
:10CE000059F00894411C511C611C711C0894C11CF0
:10CE1000D11CE11CF11CA0CF112349F08B899C8906
:10CE2000AD89BE89F10180839183A283B383C1015F
:10CE3000B701A6010FEF1FEF2FEF3FE00E9417652C
:10CE4000882399F431C0260137010894410851081C
:10CE500061087108C101B301A201970186010E9416
:10CE60001765882309F1730162018C149D04AE04D7
:10CE7000BF0448F3AD85BE854D915D916D917C9168
:10CE8000411551056105710539F0C1019501840114
:10CE90000E941765882341F0ED85FE85808291828E
:10CEA000A282B38281E001C080E066960FB6F8945A
:10CEB000DEBF0FBECDBFCF91DF911F910F91FF90CD
:10CEC000EF90DF90CF90BF90AF909F908F907F902A
:10CED0006F905F904F903F902F9008958091C10088
:10CEE00085FDFCCF8091C00085FFF8CF6093C60020
:10CEF00081E090E008951092640E1092630E8FE727
:10CF000093E09093620E8093610E0895FF920F93C9
:10CF10001F93CF93DF938B010E943B4FEB01FF24C4
:10CF2000FA9409C00E943B4F6C1B7D0B6017710780
:10CF300010F080E008C0FEBC0DB407FEFDCF8EB53A
:10CF40008F3F81F781E0DF91CF911F910F91FF908B
:10CF500008950F931F938C0185E69EE0F80162818E
:10CF60000E94D36AF801808160E00E943F501F91C7
:10CF70000F910895FF920F931F93DF93CF9300D0EB
:10CF800000D0CDB7DEB78C01F62E29833A834B83D0
:10CF90005C830E94A967C80168E572E00E94866709
:10CFA0008F2D80648EBD0DB407FEFDCFFE0131963E
:10CFB0009E012350304083818EBD0DB407FEFDCF0E
:10CFC0003197E217F307B9F7FF2011F087E801C0A6
:10CFD00085E98EBD0DB407FEFDCF8CE0F81631F467
:10CFE0008FEF8EBD0DB407FEFDCF8EB590E02FEF15
:10CFF0002EBD0DB407FEFDCF8EB587FF02C0915048
:10D00000B9F7F80183830F900F900F900F90CF9195
:10D01000DF911F910F91FF900895FC01808161E0E5
:10D020000E943F508FEF8EBD0DB407FEFDCF0895D7
:10D03000CF93DF93EC010E94A967CE0168E572E00F
:10D040000E948667882389F08DEF8EBD0DB407FEA0
:10D05000FDCFCE0168E572E00E948667882329F043
:10D06000CE010E940D6881E006C082E18983CE0175
:10D070000E940D6880E0DF91CF910895AF92BF923A
:10D08000CF92DF92EF92FF920F931F93CF93DF9394
:10D09000EC015A016B017801890167E320E030E07F
:10D0A00040E050E00E94BA67CE0167E1A801970115
:10D0B0000E94BA67882311F089E013C08C81833005
:10D0C00039F089E0AA0CBB1CCC1CDD1C8A95D1F779
:10D0D000CE0169E1A60195010E94BA67882339F063
:10D0E00087E08983CE010E940D6880E004C0CE01F4
:10D0F0000E940D6881E0DF91CF911F910F91FF9009
:10D10000EF90DF90CF90BF90AF900895CF93DF93D3
:10D11000EC01DA016EBD0DB407FEFDCF8C918EBD22
:10D120001196EC91119782E090E00DB407FEFDCFCF
:10D13000EEBD22E08030920731F0FD01E80FF91FCB
:10D14000E0810196F2CF0DB407FEFDCF8FEF8EBDCB
:10D150000DB407FEFDCF8FEF8EBD0DB407FEFDCFE2
:10D160008FEF8EBD0DB407FEFDCF8EB58B838F7113
:10D17000853011F481E006C083E18983CE010E94ED
:10D180000D6880E0DF91CF9108950F931F93CF93A7
:10D19000DF93EC018B010E94A967CE0168E572E084
:10D1A0000E948667882361F0CE016CEFA8010E947F
:10D1B0008668882329F0CE010E940D6881E006C0B0
:10D1C00085E18983CE010E940D6880E0DF91CF91D7
:10D1D0001F910F910895CF92DF92EF92FF920F93DC
:10D1E0001F93CF93DF93EC017A018B0169018C814E
:10D1F000833039F099E0EE0CFF1C001F111F9A9547
:10D20000D1F7CE0168E1A80197010E94BA6788238F
:10D2100019F086E089830CC0CE016EEFA6010E9452
:10D220008668882329F0CE010E940D6881E004C041
:10D23000CE010E940D6880E0DF91CF911F910F9188
:10D24000FF90EF90DF90CF900895CF93DF93EC01A4
:10D250006CE020E030E040E050E00E94BA678823B4
:10D2600039F083E08983CE010E940D6880E004C01C
:10D27000CE010E940D6881E0DF91CF910895CF9398
:10D28000DF93EC019A01AB018C81833039F069E0C6
:10D29000220F331F441F551F6A95D1F7CE0162E15B
:10D2A0000E94BA67882339F085E08983CE010E9405
:10D2B0000D6880E004C0CE010E940D6881E0DF911E
:10D2C000CF910895BF92CF92DF92EF92FF920F938A
:10D2D0001F93CF93DF93EC016B017A010E943B4FC8
:10D2E0008B01BB24BA9409C00E943B4F601B710B99
:10D2F0006D52714010F081E10BC0BEBC0DB407FE51
:10D30000FDCF8EB58B838F3F79F38E3F39F08FE061
:10D310008983CE010E940D6880E030C0D70111974B
:10D32000EF28D9F08FEF8EBD20E030E09FEF0BC0EB
:10D330000DB407FEFDCF8EB59EBDF601E20FF31FC3
:10D3400080832F5F3F4F2A173B0790F30DB407FEF2
:10D35000FDCF8EB5AC0DBD1D8C931B828FEF8EBDA6
:10D360000DB407FEFDCF8EB58FEF8EBD0DB407FE59
:10D37000FDCF8EB5CE010E940D6881E0DF91CF9187
:10D380001F910F91FF90EF90DF90CF90BF90089585
:10D39000EF92FF920F931F938C017B010E94A9676C
:10D3A000C801B70140E052E00E9462691F910F91ED
:10D3B000FF90EF900895CF92DF92EF92FF920F933C
:10D3C0001F93CF93DF93EC017A018B0169018C816C
:10D3D000833039F0B9E0EE0CFF1C001F111FBA9525
:10D3E000D1F7CE0161E1A80197010E94BA678823B5
:10D3F00039F084E08983CE010E940D6880E006C088
:10D40000CE01B60140E052E00E946269DF91CF9107
:10D410001F910F91FF90EF90DF90CF900895BF92F2
:10D42000CF92DF92EF92FF920F931F93CF93DF93F0
:10D43000EC01B42E1C82198268830E943B4F6B0161
:10D44000888161E00E940050888161E00E943F5025
:10D4500085E69EE00E94ED6A80E48A8385E69EE090
:10D4600060E40E94D36A80E09FEF9EBD0DB407FE8A
:10D47000FDCF8F5F8A30C9F709C00E943B4F6C19FE
:10D480007D09615D774010F081E063C0CE0160E00E
:10D4900020E030E040E050E00E94BA67813069F758
:10D4A0001FEFCE0168E02AEA31E040E050E00E9440
:10D4B000BA67853011F481E00DC080E01EBD0DB467
:10D4C00007FEFDCF9EB58F5F8430C1F79B839A3AEC
:10D4D00031F482E08C838C81823051F40DC00E9443
:10D4E0003B4F6C197D09615D7740D8F282E031C015
:10D4F000EE24FF2487010FC0E12CF12C012D80E4E4
:10D50000182F09C00E943B4F6C197D09615D77405F
:10D5100010F08AE01EC0CE0167E320E030E040E07A
:10D5200050E00E94BA67CE0169E2A80197010E940B
:10D53000BA67882339F78C81823031F5CE016AE3EE
:10D5400020E030E040E050E00E94BA67882339F0E4
:10D5500088E08983CE010E940D6880E01AC08FEFB9
:10D560008EBD0DB407FEFDCF8EB5807C803C11F4DE
:10D5700083E08C8380E09FEF9EBD0DB407FEFDCF5E
:10D580002EB58F5F8330C1F7CE010E940D68BA823D
:10D5900081E0DF91CF911F910F91FF90EF90DF908D
:10D5A000CF90BF90089540E082E002C0880F4F5FA7
:10D5B000861710F44630D1F7242F30E0C901959535
:10D5C000879580658CBD40FF02C080E004C080E08C
:10D5D000463009F081E08DBD089584E061E00E944D
:10D5E0003F5084E061E00E94005086E060E00E94CD
:10D5F000005085E061E00E94005087E061E00E94F9
:10D6000000500895382F413210F040E042C0809120
:10D61000660E8823E1F791E09093660E2093680EE2
:10D620008FEF8093D30E10928E0E415040938F0E49
:10D630004F5F9093670E8091670E330F832B80931B
:10D64000670E8091690E813041F41092690E8091CD
:10D65000670E8093BB0085EC01C085EE8093BC0013
:10D660008091660E8130E1F380918E0E841710F464
:10D6700040918E0E20E030E00AC0FB01E20FF31F64
:10D68000D901A259B14F8C9180832F5F3F4F24174E
:10D69000A0F3842F08950F931F93582F122F413218
:10D6A00010F081E04AC08091660E8823E1F782E0A5
:10D6B0008093660E0093680E8FEF8093D30E1092C6
:10D6C0008E0E40938F0EAEE6BEE0FB0102C081914C
:10D6D0008D938E2F861B8417D0F31092670E809146
:10D6E000670E550F852B8093670E8091690E8130F0
:10D6F00041F41092690E8091670E8093BB0085EC17
:10D7000001C085EE8093BC00112321F08091660E4C
:10D710008230E1F38091D30E8F3F11F480E00DC091
:10D720008091D30E803211F482E007C08091D30E35
:10D73000803311F084E001C083E01F910F910895C0
:10D74000482F613210F081E008958091660E843098
:10D7500011F082E008956093B10EA0E9BEE0842F3D
:10D760009C01F90102C081918D938E2F841B861735
:10D77000D0F380E008951F920F920FB60F921124FC
:10D780002F933F934F935F936F937F938F939F93C9
:10D79000AF93BF93EF93FF938091B90090E0887FA0
:10D7A00090708036910509F4F2C081369105CCF570
:10D7B0008832910509F47BC089329105B4F4803137
:10D7C000910509F46FC0813191053CF4009709F48B
:10D7D00047C1089709F04FC165C08831910509F428
:10D7E00066C0809709F047C182C08034910509F472
:10D7F000A4C08134910544F48033910509F482C0BA
:10D80000C89709F038C189C08035910509F489C0ED
:10D810008835910509F496C08834910509F02BC12B
:10D82000AEC08839910509F413C189399105ECF42A
:10D830008837910509F4ABC0893791054CF48836D7
:10D84000910509F4A4C08037910509F014C19FC067
:10D850008838910509F4FCC08039910509F49DC010
:10D860008038910509F007C198C0803B910509F403
:10D87000C6C0813B91054CF4803A910509F49FC0E4
:10D88000883A910509F0F7C0BAC0803C910509F4C7
:10D89000E3C0883C910509F4DFC0883B910509F09D
:10D8A000EAC0C2C08091670E8093BB00CFC0909148
:10D8B0008E0E80918F0E981768F490918E0EE92F3E
:10D8C000F0E0E259F14F80818093BB009F5F90931D
:10D8D0008E0EBCC08091680E882309F44BC085ED84
:10D8E0008093BC008091BC0084FDFCCFC2C080E26C
:10D8F0008093D30E85ED8093BC008091BC0084FDA5
:10D90000FCCFB7C080E38093D30E85ED8093BC003D
:10D910008091BC0084FDFCCFACC088E38093D30E23
:10D920009BC080918E0E9091BB00E82FF0E0E259F1
:10D93000F14F90838F5F80938E0E90918E0E809129
:10D940008F0E82C080918E0E9091BB00E82FF0E088
:10D95000E259F14F90838F5F80938E0E8091680E15
:10D96000882341F085ED8093BC008091BC0084FD4C
:10D97000FCCF7FC081E08093690E84EA6EC085EDA4
:10D980008093BC008091BC0084FDFCCF72C083E01A
:10D990008093660E1092D20E59C08091D20E8032C2
:10D9A00008F056C08091D20E9091BB00E82FF0E0B5
:10D9B000EE54F14F90838F5F8093D20E47C08091D9
:10D9C000D20E803230F4E091D20EF0E0EE54F14FFE
:10D9D000108285ED8093BC008091BC0084FDFCCF5B
:10D9E0001092660E6091D20EE0916C0EF0916D0E69
:10D9F00082EB9EE070E009951092D20E2DC084E07B
:10DA00008093660E1092B00E1092B10EE0916A0EE5
:10DA1000F0916B0E09958091B10E882329F481E075
:10DA20008093B10E1092900E9091B00EE92FF0E01D
:10DA3000E057F14F80818093BB009F5F9093B00EC1
:10DA40009091B00E8091B10E981710F485EC01C042
:10DA500085E88093BC000FC085EC8093BC0009C0B2
:10DA60001092D30E85ED8093BC008091BC0084FDA4
:10DA7000FCCF1092660EFF91EF91BF91AF919F91F5
:10DA80008F917F916F915F914F913F912F910F9067
:10DA90000FBE0F901F9018951092660E81E0809334
:10DAA000680E1092690E81E161E00E943F5080E1B2
:10DAB00061E00E943F50E9EBF0E080818E7F80833F
:10DAC00080818D7F808384E38093B80085E4809398
:10DAD000BC000895629FD001739FF001829FE00D0A
:10DAE000F11D649FE00DF11D929FF00D839FF00DDD
:10DAF000749FF00D659FF00D9927729FB00DE11D89
:10DB0000F91F639FB00DE11DF91FBD01CF01112465
:10DB10000895991B79E004C0991F961708F0961B89
:10DB2000881F7A95C9F780950895AA1BBB1B51E100
:10DB300007C0AA1FBB1FA617B70710F0A61BB70B7D
:10DB4000881F991F5A95A9F780959095BC01CD0122
:10DB5000089597FB092E07260AD077FD04D0E5DF4C
:10DB600006D000201AF4709561957F4F0895F6F75E
:10DB7000909581959F4F0895A1E21A2EAA1BBB1B79
:10DB8000FD010DC0AA1FBB1FEE1FFF1FA217B30789
:10DB9000E407F50720F0A21BB30BE40BF50B661F9F
:10DBA000771F881F991F1A9469F760957095809563
:10DBB00090959B01AC01BD01CF01089597FB092E03
:10DBC00005260ED057FD04D0D7DF0AD0001C38F44C
:10DBD00050954095309521953F4F4F4F5F4F089599
:10DBE000F6F790958095709561957F4F8F4F9F4F79
:10DBF00008952F923F924F925F926F927F928F92F1
:10DC00009F92AF92BF92CF92DF92EF92FF920F93CB
:10DC10001F93CF93DF93CDB7DEB7CA1BDB0B0FB6D5
:10DC2000F894DEBF0FBECDBF09942A883988488892
:10DC30005F846E847D848C849B84AA84B984C88428
:10DC4000DF80EE80FD800C811B81AA81B981CE0F1F
:10DC5000D11D0FB6F894DEBF0FBECDBFED01089504
:10DC6000EE0FFF1F0590F491E02D0994F894FFCF7B
:10DC70002F00616C6C0000727300726400776C009E
:10DC80002E0076006F70656E646F6F7200426F7366
:10DC9000746F6E2C4D410068747470733A2F2F7539
:10DCA000692E6F70656E737072696E6B6C65722E23
:10DCB000636F6D2F6A73000068747470733A2F2F4E
:10DCC00075692E6F70656E737072696E6B6C6572BC
:10DCD0002E636F6D2F6A7300763D5B00743D5B00B1
:10DCE0002F002E63677A002E6A677A00776C000D2A
:10DCF0000A0000323030004F532D30300063825321
:10DD000063350150002F6C6F67732F000601070108
:10DD10000A010D01D600C60118011C6CCA011C01C4
:10DD20000101D1011F010101D601230100FFDC0126
:10DD3000280100FFE4012C0100FFEA01300100FF8F
:10DD4000F001340100FFF601380100FFFE013C0143
:10DD500000FF0402400100FF0A02440150FF1002CC
:10DD6000480100FF16024C01150017025001000582
:10DD70001C02540101012802580180F729025A01AE
:10DD8000003034025E01003C3A0262013C784802F5
:10DD90006701000156026C0101016302700164FA1F
:10DDA0007202740101017E02770100018B027B0186
:10DDB00000FF940280016EFF9D02860164FFA702AE
:10DDC0008A010FFFB1028E0100C8BB02920100FF61
:10DDD000BC02940132FFC902980161FFD2029D0189
:10DDE000D2FFD802A201A9FFDE02A7010101E402CD
:10DDF000AC010030E902AF01003CEF02B4013C7815
:10DE0000FD02BA0100010B03C00116031A031E0331
:10DE1000220326032A032E03F403783CF703BF3EB4
:10DE2000FA030A37FD03C435000437370304E1362B
:10DE30000604C53E090486330C04BE350F04E632E1
:10DE40001204A130150434321804BD371B049A4162
:10DE50001E04D73A2104383124040B3127045033EF
:10DE60007B010A100E000001FFFFFFFFFFFF000013
:10DE70000000BB11355300004000140054000000A6
:10DE80000000EC1235532E6F4F00000703050810F9
:10DE900000000006091F00151500001F111F1113B7
:10DEA0001E00140815010505156F00000000000094
:10DEB00000FFFFFFFFFFFF1F1C1F1E1F1E1F1F1E57
:10DEC0001F1E1F0000000057523553EB511C52FC1F
:10DED00051455200000000D754A6545F5468547D49
:10DEE000548E5400000000F462F062000000006EE6
:04DEF000673553003F
:00000001FF
